:100000000C9492190C94C3190C94C3190C94C31931
:100010000C94C3190C94C3190C94C3190C94C319F0
:100020000C94C3190C94C3190C94C3190C94C319E0
:100030000C94C3190C94C3190C94C3190C94C319D0
:100040000C94C3190C9474680C94C3190C94C319C0
:100050000C94C3190C94C3190C94F18C0C94BFFB31
:100060000C94C3190C94AA540C94A0540C94C31966
:100070000C94C3190C94C3190C94C3190C94C31990
:100080000C94C3190C94C3190C94C3190C94C31980
:100090000C94C3190C94C3190C94C3190C94C31970
:1000A0000C94C3190C94C3190C94C3190C94C31960
:1000B0000C94C3190C94C3190C94C3190C94C31950
:1000C0000C94C3190C94C3190C94C3190C944E5777
:1000D0000C9424570C94C3190C94C3190C94C31991
:1000E0000C94C319721BB81BBE1BE51BF21BFB1B38
:1000F000061CCC23DE24BB25EE25B631B6310927FC
:10010000AA27BA24B631B6314929E32A1B2BB631C6
:10011000412DB631B631912EB631B6311B2F4E2F4F
:10012000B6310E30C930DD54E354F55405550D5544
:100130003A5511553A55155519553A551D552155EC
:1001400025552D553A553755375E3A5E295E2D5E59
:10015000335E715E3E5E425E485E4C5E505E565E51
:100160005A5E5E5E715E645E685E6C5E3A673F67B3
:1001700044674E675867D16762676A6772677C67D2
:10018000866790679F67A967D167B367BD67C767D1
:10019000D2A1F4A114A239A25EA215A483A2A6A2A0
:1001A000C9A2EEA213A338A35DA382A315A4A7A39B
:1001B000CCA3F1A3A3A5A6A5AAA5ADA5B0A5DAA534
:1001C000B4A5B7A5BBA5BEA5C1A5C5A5C8A5CBA50A
:1001D000DAA5CFA5D2A5D5A5084AD73B3BCE016E5F
:1001E00084BCBFFDC12F3D6C74319ABD56833DDA8E
:1001F0003D00C77F11BED9E4BB4C3E916BAAAABE9D
:10020000000000803F05A84CCDB2D44EB93836A9C5
:10021000020C50B9918688083CA6AAAA2ABE000002
:1002200000803F000C94A7A30C94E51B0C94FB1BCF
:100230000C9419550C94715E0C94B7A50C947C67C2
:100240000C94ADA50C94D1670C9421550C94F055E9
:100250000C94EEA20C94D2A50C9425550C94BE1BC4
:100260000C942D5E0C94B81B0C94BD670C94D2A119
:100270000C94061C0C94E32A0C943E5E0C94092703
:100280000C94BBA50C946C5E0D946D040C94B0A5FD
:100290000C945A5E0C94F21B0C94B3670C94412D91
:1002A0000C94AAA50C94C8A50C9449290C9413A3EA
:1002B0000C9436560C94C5A50C94565E0C943F676E
:1002C0000C94F1A30C946A670C9415550C945E5E23
:1002D0000C9414A20C94B4A50C943A5E0C94CD55D5
:1002E0000C945EA20C9439A20C94C9A20D94ED0654
:1002F0000C94BB250C9490670C94CCA30C941155D2
:100300000C94A6A50C94F4A10C942D550C9483A2E6
:100310000C943A670C943A550C949F550C94DE2437
:100320000C94F5540C94DC550C941D550C94E3542A
:100330000C94375E0C9458670C9405550C94505EE1
:100340000C9482A30C94EE250C941B2F0C94BA24CD
:100350000C94CFA50C9462670C94A3A50C94335E07
:100360000C94A9670C940E300C944C5E0C94FE55C2
:100370000C9483560C9472670C94DAA50C94AA27FB
:100380000C940D550C9486670C9444670C94CC2304
:100390000C949F670C94485E0C94C1A50C94C930D2
:1003A0000C94912E0C94BEA50C94645E0C94721B5C
:1003B0000C94295E0C94D5A50C94CBA50C945DA34C
:1003C0000C94C7670C941B2B0C9437550C94A6A265
:1003D0000C944E2F0C94685E0C94DD540C94425E89
:1003E0000C944E670C9438A30C94B6310C9415A45D
:1003F0004E414E494E495459494E46CDCCCC3D0A0A
:10040000D7233C17B7D13877CC2B329595E6241FEC
:10041000B14F0A000020410000C84200401C4620A5
:10042000BCBE4CCA1B0E5AAEC59D7400407A10F378
:100430005A00A0724E18090010A5D4E80000E87612
:1004400048170000E40B54020000CA9A3B00000069
:10045000E1F505000080969800000040420F000082
:1004600000A08601000000102700000000E8030043
:100470000000006400000000000A0000000000010D
:1004800000000000002C76D888DC674F0823DFC10D
:10049000DFAE59E1B1B796E5E3E453C63AE65199C8
:1004A0007696E8E6C28426EB898C9B62ED407C6FF1
:1004B000FCEFBC9C9F40F2BAA56FA5F490055A2AA8
:1004C000F75C936B6CF9676DC11BFCE0E40D47FEB4
:1004D000F520E6B500D0ED902E03009435770500A9
:1004E00080841E080000204E0A000000C80C333330
:1004F00033330F986E12831141EF8D2114893BE63F
:100500005516CFFEE6DB18D1844B381BF77C1D90C7
:100510001DA4BBE424203284725E228100C9F12430
:10052000ECA1E53D274D323520500A4D32340050C4
:1005300072696E74205061757365640052657375DD
:100540006D65005549205061757365004E6F204DF3
:1005500061746368203A004D333033452D31533692
:1005600035433455004D393939004D3530320A4D57
:10057000353030004D333033453053323135433828
:1005800055000A202A2A2A7265636461742E646108
:1005900074615B305D203D004732380A47312046A8
:1005A00031303030205A313000556E737570706FB5
:1005B00072746564204F7074696F6E2053656C654A
:1005C000637465640047323800473120463130306B
:1005D00030205A302E30004732380A473120463119
:1005E000303030205A302E30004D353030005A2017
:1005F0004F6666736574203A202573004D353030A0
:10060000005A204F6666736574203A2025730047B0
:1006100032385A0A473146313530305A302E3000A0
:100620004732380A473146313530305A302E3000A3
:100630004D383400473146313030305A302E30009A
:100640004732380A473146313030305A302E300088
:100650005A204F6666736574203A202573004D3525
:100660003030004D383400426567696E53776974E5
:100670006368007265636461742E61646472203D16
:100680003D007265636461742E646174615B305D0A
:10069000203D3D0077616974776179203D3D000A16
:1006A000202A2A2A4E6F7A7A6C6554656D705374CD
:1006B000617475735B325D203D00434F4D4D554E67
:1006C00049434154494F4E0044525952554E0045FA
:1006D00052524F525300494E464F004543484F0037
:1006E00047322F47332062616420706172616D650B
:1006F000746572730A00536C6565702E2E2E004867
:100700006F6D652058592046697273740A00486FEE
:100710006D65205859204669727374004F46460033
:100720004F4E00206F6620004D424C20473239204A
:10073000706F696E742000290A004A206F7574205A
:100740006F662072616E67652028302D00290A00CF
:1007500049206F7574206F662072616E676520286E
:10076000302D004D6573682070726F62696E67206E
:10077000646F6E652E0A005374617274206D657328
:10078000682070726F62696E6720776974682022D2
:10079000473239205331222066697273742E0A0061
:1007A0004732380A47323920533200686173206E6D
:1007B0006F20646174612E0A004D65736820426584
:1007C00064204C6576656C696E67200053206F75F8
:1007D00074206F662072616E67652028302D352980
:1007E0002E0A004D65736820706F696E7420636116
:1007F0006E6E6F74206265207265736F6C766564CF
:100800000A004D302F3120427265616B2043616CCC
:100810006C656400436F6E74696E7565004D302FB2
:100820003120427265616B2043616C6C6564004EDF
:100830006F204D6F76652E00456E642066696C658D
:10084000206C6973740A00426567696E2066696C82
:1008500065206C6973740A00526573756D65205369
:100860004400286E6F2066696C65290043757272BA
:10087000656E742066696C653A20002E0A00446536
:100880006C6574696F6E206661696C65642C2046C6
:10089000696C653A200046696C652064656C657416
:1008A00065643A005072696E742074696D653A200F
:1008B000000A53746174733A2046696C616D656E09
:1008C0007420757365643A20002C204C6F6E676548
:1008D0007374206A6F623A2000546F74616C2074E4
:1008E000696D653A200053746174733A20002C20BE
:1008F0004661696C65643A20002C2046696E697314
:100900006865643A20005072696E74733A2000532F
:10091000746174733A20006F666600DB06D606CFFA
:1009200006C806BA0644454255473A004D313133B0
:1009300020530042656420436F6F6C696E672E2EF2
:100940002E004265642048656174696E672E2E2E04
:10095000006F6B004348414D4245525F54454D5036
:1009600045524154555245004D4F54494F4E5F4DED
:100970004F44455300544845524D414C5F50524FEF
:1009800054454354494F4E004155544F5245504FE2
:1009900052545F53445F5354415455530050524F87
:1009A0004D50545F535550504F525400454D455291
:1009B00047454E43595F50415253455200434153BE
:1009C000455F4C494748545F4252494748544E4559
:1009D000535300544F47474C455F4C494748545385
:1009E00000534F4654574152455F504F57455200B0
:1009F0004255494C445F50455243454E54004C4586
:100A000056454C494E475F44415441005A5F50524D
:100A10004F4245004155544F4C4556454C005052AD
:100A2000494E545F4A4F420050524F47524553532C
:100A3000004155544F5245504F52545F54454D500C
:100A400000564F4C554D4554524943004545505270
:100A50004F4D0042494E4152595F46494C455F5403
:100A600052414E534645520053455249414C5F58FE
:100A70004F4E5F584F4646004649524D57415245EA
:100A80005F4E414D453A4D61726C696E20322E3099
:100A90005F44573220544D33442053534D444E4EFF
:100AA00020534F555243455F434F44455F55524C89
:100AB0003A68747470733A2F2F6769746875622E80
:100AC000636F6D2F496E73616E6974794175746FD0
:100AD0006D6174696F6E2F4D61726C696E2F7472E7
:100AE00065652F437265616C6974795F4D61726CE5
:100AF000696E322E302E782050524F544F434F4C57
:100B00005F56455253494F4E3A312E30204D4143A6
:100B100048494E455F545950453A544D334420435B
:100B2000522D582045585452554445525F434F5515
:100B30004E543A3220555549443A636564653261F2
:100B400032662D343161322D343734382D396231EB
:100B5000322D6335356336326633363766660A00C2
:100B60002F2F2000205400205200416363656C65E4
:100B7000726174696F6E3A2050003F4A206F75743D
:100B8000206F662072616E67652028302E3031201C
:100B9000746F20302E33290A0020466C6F773A207C
:100BA0000050726F7465637465642050696E0A004A
:100BB000496E76616C6964206578747275646572DB
:100BC0000A0020643A0020693A0020703A0020644C
:100BD0003A0020693A0020703A0064697300656E3B
:100BE0000043290A0061626C656420286D696E20EB
:100BF00074656D702000436F6C6420657874727545
:100C00006465732061726520004F66667365747356
:100C1000204170706C696564004572723A20546FAF
:100C20006F206661722100546F6F206661722066CA
:100C3000726F6D207265666572656E636520706F98
:100C4000696E740A00454550524F4D204F4B0A00C3
:100C5000416476616E6365204B003F4B2076616C8A
:100C60007565206F7574206F662072616E676520F0
:100C700028302D3130292E0A003F542076616C75C2
:100C800065206F7574206F662072616E67652E0A2D
:100C9000004572726F722077726974696E67207492
:100CA0006F20454550524F4D210A00363726033CF0
:100CB0003D380E2E303E121A1C1824221E08440AFB
:100CC000FF430809070001627573793A2070617566
:100CD00073656420666F7220696E7075740A0062B5
:100CE0007573793A2070617573656420666F722040
:100CF000757365720A00627573793A2070726F635A
:100D0000657373696E670A004B494C4C20636175CB
:100D100073656420627920746F6F206D756368203D
:100D2000696E6163746976652074696D65202D2034
:100D300063757272656E7420636F6D6D616E643A77
:100D40002000706F7765726F6666004B494C4C45AA
:100D5000442E20005072696E7465722068616C7454
:100D600065642E206B696C6C28292063616C6C654E
:100D700064210A006563686F3A004572726F723AC7
:100D8000000A4D6561737572656420706F696E74D9
:100D9000733A0A002F2F616374696F6E3A006275AF
:100DA00074746F6E00656E640070726F6D70745F46
:100DB0000073686F77002020506C616E6E65724220
:100DC000756666657242797465733A2000204672D2
:100DD0006565204D656D6F72793A2000436F6D70C7
:100DE000696C65643A2053657020203720323031B9
:100DF000390A00207C20417574686F723A2054696A
:100E00006E794D616368696E657333440A003230F0
:100E100031392D30372D333000204C61737420551B
:100E20007064617465643A2000322E305F4457323A
:100E30000A004D61726C696E0020536F66747761B1
:100E400072652052657365740A0020576174636887
:100E5000646F672052657365740A002042726F7771
:100E60006E206F75742052657365740A0020457892
:100E70007465726E616C2052657365740A00506F00
:100E800077657255700A0073746172740A00617537
:100E9000746F25632E67006572726F7220777269B6
:100EA00074696E6720746F2066696C650A00446F10
:100EB0006E6520736176696E672066696C652E0ABF
:100EC000004D323900205A3A0020593A0020583A51
:100ED00000656E6473746F7073206869743A2000E3
:100EE00047323858590043616E6E6F74206F7065D9
:100EF0006E207375626469722000534420636172CE
:100F000064206F6B0A006F70656E526F6F7420669D
:100F100061696C65640A00766F6C756D652E696E2B
:100F20006974206661696C65640A00534420696EC7
:100F30006974206661696C0A004D3234004D3233A9
:100F40002025730057726974696E6720746F20667C
:100F5000696C653A20002E0A006F70656E2066612C
:100F6000696C65642C2046696C653A20002E0A0085
:100F70006F70656E206661696C65642C2046696CD3
:100F8000653A200046696C652073656C656374651D
:100F9000640A002053697A653A200046696C65202E
:100FA0006F70656E65643A200066726573680064F0
:100FB0006F696E67002066696C653A20004E6F7736
:100FC0002000454E4420535542524F5554494E45FA
:100FD0000A002220706F73002220706172656E74A7
:100FE0003A2200535542524F5554494E45204341F1
:100FF0004C4C207461726765743A2200747279698E
:101000006E6720746F2063616C6C207375622D674E
:10101000636F64652066696C657320776974682006
:10102000746F6F206D616E79206C6576656C732EC0
:10103000204D4158206C6576656C2069733A310A01
:10104000005344207072696E74696E67206279740F
:101050006520004E6F74205344207072696E74696D
:101060006E670A0000002100240027002A002D00DE
:101070003000330001010000040107010A010000F3
:101080002200250028002B002E0031003400020130
:101090000000050108010B010000200023002600CC
:1010A00029002C002F00320000010000030106017E
:1010B00009010505050507050808080802020202DE
:1010C0000A0A0808040404040101010101010101E4
:1010D0000303030303030303040707070C0C0C0CAF
:1010E0000C0C0C0C02020202060606060606060698
:1010F0000B0B0B0B0B0B0B0B010210202008081025
:101100002040102040800201020108040201010277
:101110000408102040808040201008040201800450
:1011200002018040201008040201080402010102AB
:1011300004081020408001020408102040800000B4
:101140000A0B02090C0D0E08070304010000000041
:10115000000000000000000000000000000000008F
:10116000000000000000000000001211100000004C
:10117000000000000000000000000000000000006F
:1011800000000000473238002046697273740A007C
:10119000486F6D652000486F6D65202573257325A8
:1011A0007320466972737400220A00556E6B6E6F6D
:1011B000776E20636F6D6D616E643A20220024F4B7
:1011C000D43050C38E20C2A24017828B7011127A85
:1011D000910D816CD90AA861E108C7586607615171
:1011E00043061E4B5D05C145A7041A411104093D84
:1011F0009803713931034036DB0265339102D430F4
:101200005402802E1D02632CEE01752AC501B02800
:10121000A001102781018F2564012B244B01E022BE
:101220003401AC211F018D200D01801FFC00841EA4
:10123000ED00971DDF00B81CD200E61BC600201B86
:10124000BC00641AB200B219A8000A19A0006A18FA
:101250009900D117910040178B00B5168400311604
:101260007E00B31579003A157300C7146F00581447
:101270006A00EE1366008813630025135E00C71230
:101280005B006C12570015125400C111510070110F
:101290004F0021114B00D61049008D104700461019
:1012A000440002104200C00F4000800F3E00420F79
:1012B0003C00060F3B00CB0E3800930E37005C0E4F
:1012C0003500270E3400F30D3200C10D3100900DB2
:1012D0003000600D2E00320D2D00050D2C00D90CB4
:1012E0002B00AE0C2900850C29005C0C2700350C66
:1012F00027000E0C2600E80B2400C40B2400A00BD2
:1013000023007D0B23005A0B2100390B2100180B01
:101310002000F80A1F00D90A1E00BB0A1E009D0A01
:101320001D00800A1D00630A1C00470A1B002C0ACE
:101330001B00110A1A00F7091A00DD091900C40977
:101340001900AB091900920917007B0918006309FD
:1013500017004C09160036091600200916000A0964
:101360001500F5081500E0081400CC081400B808B2
:101370001400A4081400900813007D0812006B08E4
:101380001300580812004608120034081100230800
:1013900011001208110001081100F0071000E00709
:1013A0001000D0071000C0071000B0070F00A10701
:1013B000100091070E0083070F0074070F006507E8
:1013C0000E0057070E0049070E003B070D002E07C1
:1013D0000E0020070D0013070D0006070D00F9068B
:1013E0000C00ED060D00E0060C00D4060C00C8064B
:1013F0000C00BC060C00B0060C00A4060B009906FD
:101400000C008D060B0082060B0077060B006C06A5
:101410000B0061060A0057060B004C060A00420644
:101420000A0038060A002E060A0024060A001A06D8
:101430000A001006090007060A00FD050900F40568
:101440000900EB050900E2050900D9050900D005EE
:101450000900C7050900BE050900B5050800AD056E
:101460000800A50509009C050800940508008C05E6
:101470000800840508007C050800740508006C0558
:101480000700650508005D050700560508004E05C4
:10149000070047050700400508003805070031052B
:1014A00007002A050700230507001C05060016058E
:1014B00007000F0507000805060002050700FB04EA
:1014C0000600F5040700EE040600E8040600E20446
:1014D0000700DB040600D5040600CF040600C9049B
:1014E0000600C3040600BD040600B7040600B104EC
:1014F0000500AC040600A6040600A00405009B0439
:10150000060095040500900406008A040500850481
:101510000500800406007A040500750405007004C7
:1015200005006B04050066040500610405005C0409
:10153000050057040500520405004D040500480449
:101540000500430405003E0404003A040500350488
:101550000500300404002C040500270404002304C3
:1015600005001E0404001A040400160405001104FA
:1015700004000D0404000904050004040400000430
:101580000400FC030400F8030400F4030400F00367
:101590000400EC030400E8030400E4030400E00397
:1015A0000400DC030400D8030400D4030400D003C7
:1015B0000400CC030400C8030300C503030024F4A3
:1015C00004D9201BC40C5C0E9804C4095F02650793
:1015D0007101F405F900FB04B30048048700C1035E
:1015E00069005803550003034500BE023A00840217
:1015F000310053022A002902250004022000E401E0
:101600001C00C8011900AF011700980114008401E3
:101610001300710110006101100051010E0043011F
:101620000D0036010B002B010B0020010B001501F2
:1016300009000C01090003010800FB000800F30089
:101640000800EB000700E4000600DE000600D800FA
:101650000600D2000600CC000500C7000500C2004D
:101660000500BD000400B9000400B5000400B1008D
:101670000400AD000400A9000400A5000300A200BE
:1016800003009F0004009B000300980003009500E6
:10169000020093000300900003008D0002008B0005
:1016A000030088000200860002008400030081001D
:1016B00002007F0002007D0002007B000200790032
:1016C0000200770001007600020074000200720040
:1016D0000100710002006F0002006D0001006C004B
:1016E00002006A0001006900020067000100660054
:1016F0000100650001006400020062000100610059
:101700000100600001005F0002005D0001005C005C
:1017100001005B0001005A0001005900010058005F
:10172000010057000100560001005500010054005F
:10173000010053000000530001005200010051005D
:101740000100500001004F0001004E0000004E005B
:1017500001004D0001004C0001004B0000004B0057
:1017600001004A0001004900010048000000480053
:10177000010047000100460000004600010045004E
:101780000000450001004400010043000000430048
:101790000100420000004200010041000000410041
:1017A0000100400001003F0000003F0001003E003A
:1017B00000003E0001003D0000003D0001003C0033
:1017C00000003C0000003C0001003B0000003B002A
:1017D00001003A0000003A00010039000000390021
:1017E0000100380000003800000038000100370018
:1017F000000037000100360000003600000036000F
:101800000100350000003500000035000100340003
:1018100000003400000034000100330000003300F9
:1018200000003300010032000000320000003200EE
:1018300001003100000031000000310001003000E3
:10184000000030000000300001002F0000002F00D9
:1018500000002F0000002F0001002E0000002E00CD
:1018600000002E0001002D0000002D0000002D00C2
:1018700000002D0001002C0000002C0000002C00B6
:1018800000002C0001002B0000002B0000002B00AA
:1018900000002B0001002A0000002A0000002A009E
:1018A00000002A0001002900000029000000290092
:1018B0000000290000002900010028000000280085
:1018C0000000280000002800000028000100270078
:1018D000000027000000270000002700000027006C
:1018E000010026000000260000002600000026005F
:1018F0000000260001002500000025000000250052
:101900000000250000002500000025000100240043
:101910000000240000002400000024000000240037
:10192000010023000000230000002300000023002A
:10193000000023000000230000002300010022001B
:10194000000022000000220000002200000022000F
:101950000000220001002100000021000000210001
:1019600000002100000021000000210000002100F3
:1019700001002000000020000000200000002000E6
:1019800000002000000020000000200000002000D7
:1019900001001F0000001F0000001F0000001F00CA
:1019A00000001F0000001F0000001F0001001E00BB
:1019B00000001E0000001E0000001E000000C231DA
:1019C00000001C260000F4190000D80F0000EB08EE
:1019D0000000C004000075020000400100002074F7
:1019E0006F6F206C6F6E6720657874727573696FA6
:1019F0006E2070726576656E7465640A0020636F90
:101A00006C6420657874727573696F6E207072658E
:101A100076656E7465640A00453120544845524D20
:101A2000414C2052554E41574159004245442054A3
:101A30004845524D414C2052554E41574159005452
:101A40006865726D616C2052756E617761790045D1
:101A500031204572723A204D415854454D50004551
:101A600072723A204D415854454D50204245440031
:101A70004D415854454D50207472696767657265D1
:101A800064004531204572723A204D494E54454D0F
:101A900050004572723A204D494E54454D502042F7
:101AA0004544004D494E54454D5020747269676756
:101AB00065726564000A0A0020205A5F4D494E3A5B
:101AC000002020595F4D494E3A002020585F4D4973
:101AD0004E3A004D383420582059205A20450020D5
:101AE0002F002042403A0020403A004520436F6FCB
:101AF0006C696E672E2E2E00452048656174696EF4
:101B0000672E2E2E0020573A0020573A00496E7655
:101B1000616C69642065787472756465720A00414D
:101B200063746976652045787472756465723A20CD
:101B300000486F74656E6420746F6F20636F6C640F
:101B40000A00220A00656E7175657565696E672009
:101B500022002042002050006F6B00526573656EBA
:101B6000643A200053544F505045442E2000507288
:101B7000696E7465722073746F707065642064752B
:101B80006520746F206572726F72732E20466978BB
:101B900020746865206572726F7220616E642075B2
:101BA0007365204D39393920746F20726573746103
:101BB00072742E202854656D70657261747572653B
:101BC0002069732072657365742E205365742069D3
:101BD00074206166746572207265737461727469D1
:101BE0006E67290A004E6F20436865636B73756DDD
:101BF0002077697468206C696E65206E756D62650A
:101C0000722C204C617374204C696E653A20004E32
:101C10006F20436865636B73756D20776974682006
:101C20006C696E65206E756D6265722C204C6173F7
:101C300074204C696E653A2000636865636B737548
:101C40006D206D69736D617463682C204C617374D1
:101C5000204C696E653A20004C696E65204E756DAA
:101C6000626572206973206E6F74204C61737420FA
:101C70004C696E65204E756D6265722B312C204C5F
:101C8000617374204C696E653A20004D313130002B
:101C9000776169740A004D313137004D333100539B
:101CA000442072656164206572726F720A00446F2D
:101CB0006E65207072696E74696E672066696C6506
:101CC0000A007C3C3E5E2B3D3F2F5B5D3B2C2A2275
:101CD0005C005A5F53544F505F50494E005A5F5357
:101CE0005445505F50494E005A5F4D494E5F504930
:101CF0004E005A5F454E41424C455F50494E005A96
:101D00005F4449525F50494E005A5F43535F504908
:101D10004E00595F53544F505F50494E00595F5326
:101D20005445505F50494E00595F4D494E5F5049F0
:101D30004E00595F454E41424C455F50494E005957
:101D40005F4449525F50494E00595F43535F5049C9
:101D50004E00585F53544F505F50494E00585F53E8
:101D60005445505F50494E00585F4D494E5F5049B1
:101D70004E00585F454E41424C455F50494E005819
:101D80005F4449525F50494E00585F43535F50498A
:101D90004E0053535F50494E00534552564F335FE8
:101DA00050494E00534552564F325F50494E0053F2
:101DB0004552564F315F50494E00534552564F30B1
:101DC0005F50494E00534453530053445F444554BD
:101DD0004543545F50494E0053434B5F50494E00BA
:101DE00052414D50535F44395F50494E0052414D6E
:101DF00050535F44385F50494E0052414D50535F3D
:101E00004431305F50494E004D4F53495F50494E69
:101E1000004D4F534645545F445F50494E004D4975
:101E2000534F5F50494E004D4158363637355F535A
:101E3000535F50494E004C45445F50494E00484561
:101E4000415445525F4245445F50494E0048454128
:101E50005445525F305F50494E0046494C5F5255E1
:101E60004E4F55545F50494E0046414E315F5049E8
:101E70004E0046414E5F50494E0045315F53544538
:101E8000505F50494E0045315F454E41424C455FE1
:101E900050494E0045315F4449525F50494E00451C
:101EA000315F43535F50494E0045305F53544550B6
:101EB0005F50494E0045305F454E41424C455F50B2
:101EC000494E0045305F4449525F50494E0045300D
:101ED0005F43535F50494E00455F4D5558325F5048
:101EE000494E00455F4D5558315F50494E00455FA2
:101EF0004D5558305F50494E004156525F53535F25
:101F000050494E004156525F53434B5F50494E007B
:101F10004156525F4D4F53495F50494E0041565212
:101F20005F4D49534F5F50494E0054454D505F42FD
:101F300045445F50494E0054454D505F315F504914
:101F40004E0054454D505F305F50494E0046494C5D
:101F500057494454485F50494E0054584400525821
:101F60004400546F6F6C6368616E67653A002020AF
:101F70004D32313700205A0020590020580020529D
:101F80000020500020450020530050574D3A20209B
:101F90002534640050574D3A2020253464005057B2
:101FA0004D3A20202534640050574D3A20202534E6
:101FB000640050574D3A20202534640050574D3A64
:101FC00020202534640050574D3A202025346400E9
:101FD00050574D3A20202534640050574D3A202068
:101FE0002534640050574D3A202025346400505762
:101FF0004D3A20202534640050574D3A2020253496
:10200000640050574D3A20202534640050574D3A13
:1020100020202534640050574D3A20202534640098
:1020200050574D3A202025346400433A2000423A6C
:102030002000413A200020202020434F4D00202046
:10204000206E6F6E2D7374616E64617264205057E0
:102050004D206D6F646500202020636F6D7061728C
:102060006520696E7465727275707420656E616248
:102070006C6564002020206F766572666C6F772037
:10208000696E7465727275707420656E61626C65DC
:1020900064003A20002020202054494D534B004238
:1020A0003A2000202020205443435200413A20008F
:1020B0002020202054434352002020202043533A24
:1020C00020002020202057474D3A200050574D3AFD
:1020D00020202534640050574D3A202025346400D8
:1020E00047004800000088008A008C00B300B4005C
:1020F000000098009A009C00A800AA00AC002801EB
:102100002A012C012020202054494D455200440032
:1021100045006E00800081006F00B000B1007000CB
:10212000900091007100A000A10072002001210127
:10213000730020697320616C736F2074696564207B
:10214000746F20746869732070696E0054494D453E
:10215000523143000A202E002020002020506F72B0
:10216000743A200020202000202020416E616C6FF6
:102170006720696E203D2025356C64003C756E75C6
:102180007365642F756E6B6E6F776E3E002028410D
:10219000253264292020002533642000257350490E
:1021A0004E3A20004F7574707574203D2000496EC2
:1021B00070757420203D2000416E616C6F6720694E
:1021C0006E203D2025356C640070726F74656374F9
:1021D0006564200020284125326429202000253311
:1021E000642000257350494E3A20005E1F00015ABA
:1021F0001F01014D1F3B00421F4300371F45002AAE
:102200001F44001D1F3201101F3301041F3401F948
:102210001E3501EE1E2801E31E2A01D81E2C01CE18
:102220001E2A01C31E1C01B51E1801A91E1A019FFA
:102230001E2C01941E2201861E1E017A1E2401728C
:102240001E0901691E07015A1E02014D1E0A013EA8
:102250001E0801361E0D01271E42011E1E320111ED
:102260001E0701081E3301FA1D0A01ED1D0801E0D9
:102270001D0901D81D3401CA1D3101C51D3501BA22
:102280001D0B01AF1D0601A41D0501991D0401923E
:102290001D3501891D35017F1D3701721D2601681D
:1022A0001D03015D1D3601521D0301491D31013F12
:1022B0001D3D01321D3801281D0E011D1D3C01125E
:1022C0001D0E01091D2801FF1C3001F21C3E01E812
:1022D0001C1201DD1C2E01D21C12015761697469A8
:1022E0006E6720666F72206865617475702E0A00D3
:1022F0004C656176696E6720473236003F537065E2
:1023000063696669656420582C5920636F6F726435
:10231000696E617465206F7574206F6620626F75D9
:102320006E64732E0A003F2852296570656174201F
:1023300076616C7565206E6F7420706C6175736961
:10234000626C653B206D757374206265206174203A
:102350006C6561737420312E0A003F285229657024
:10236000656174206D757374206265207370656398
:102370006966696564207768656E206E6F74207584
:1023800073696E6720616E204C43442E0A003F53F0
:102390007065636966696564206E6F7A7A6C652022
:1023A00074656D7065726174757265206E6F7420EE
:1023B000706C61757369626C652E0A003F537065BD
:1023C0006369666965642066696C616D656E742019
:1023D00073697A65206E6F7420706C6175736962C1
:1023E0006C652E0A003F53706563696669656420F9
:1023F0007072696D65206C656E677468206E6F74AD
:1024000020706C61757369626C652E0A003F5072B2
:10241000696D65206C656E677468206D75737420D6
:1024200062652073706563696669656420776865B5
:102430006E206E6F74207573696E6720616E204C1C
:1024400043442E0A003F53706563696669656420E2
:102450006E6F7A7A6C652073697A65206E6F74206E
:10246000706C61757369626C652E0A003F52657409
:1024700072616374696F6E204D756C7469706C69FC
:102480006572206D75737420626520737065636971
:10249000666965642E0A003F537065636966696505
:1024A000642052657472616374696F6E204D756C3F
:1024B0007469706C696572206E6F7420706C6175E0
:1024C0007369626C652E0A003F53706563696669C3
:1024D0006564206C6179657220686569676874203D
:1024E0006E6F7420706C61757369626C652E0A0082
:1024F00043292E0A003F537065636966696564204D
:102500006265642074656D706572617475726520B2
:102510006E6F7420706C61757369626C652028340D
:10252000302D00473236207374617274696E672EE5
:102530002E2E0A004F46460A004661646520486513
:10254000696768742000426564204C6576656C6933
:102550006E6720004661696C656420746F20656E4B
:1025600061626C6520426564204C6576656C696EBD
:10257000670A004D65736820426564204C65766586
:102580006C20646174613A0A00496E76616C69641A
:10259000206D6573682E0A00206E6F7420656E745E
:1025A000657265642E0A004D65736820706F696EF0
:1025B000742063616E6E6F74206265207265736F44
:1025C0006C7665640A004D34323120696E636F7237
:1025D0007265637420706172616D657465722075D7
:1025E000736167650A00446F6E652E0A0053455299
:1025F000564F206E6F74207365742075702E0A001C
:102600004D343320576169742043616C6C656400FC
:10261000436F6E74696E7565004D34332057616980
:10262000742043616C6C6564005761746368696E03
:10263000672070696E730A0064697300656E0061DB
:10264000626C65640A00656E6473746F70206D6FF0
:102650006E69746F722000204500205A00205900D6
:10266000204D3932205800205A00205900580020AF
:10267000204D61783A2000205A002059005800204F
:10268000204D696E3A2000536F667420656E647346
:10269000746F70733A20005761726E696E67203AEA
:1026A00020436C65616E20436972636C65207265BE
:1026B0007175697265732058590A0020496E7661F8
:1026C0006C6964206578747275646572200043617A
:1026D0006E6E6F74206F70656E20737562646972C0
:1026E00020002569730025696D202569730025691F
:1026F000682025696D202569730025696420256996
:10270000682025696D202569730025697920256970
:1027100064202569682025696D202569730023647C
:102720006566696E652044454641554C545F00001E
:10273000626564004B6420004B6920004B702000F0
:10274000504944204175746F74756E652066696EDA
:102750006973686564212050757420746865206C05
:10276000617374204B702C204B6920616E64204B88
:102770006420636F6E7374616E74732066726F6D24
:102780002062656C6F7720696E746F20436F6E6690
:10279000696775726174696F6E2E680A00504944EA
:1027A000204175746F74756E65206661696C65642F
:1027B000212074696D656F75740A00453120544895
:1027C00045524D414C2052554E41574159004245CA
:1027D0004420544845524D414C2052554E4157419A
:1027E0005900546865726D616C2052756E61776135
:1027F000790045312048656174696E6720466169DA
:102800006C6564004265642048656174696E672088
:102810004661696C65640048656174696E6720662D
:1028200061696C656400504944204175746F74752A
:102830006E65206661696C6564212054656D706504
:1028400072617475726520746F6F20686967680AB9
:1028500000204B643A2000204B693A2000204B7046
:102860003A20000A20436C61737369632050494425
:10287000200A00204B643A2000204B693A200020B7
:102880004B703A20000A204E6F206F766572736895
:102890006F6F740A002054753A2000204B753A205F
:1028A00000206D61783A2000206D696E3A2000208A
:1028B000643A200020626961733A20005049442044
:1028C0004175746F74756E652073746172740A005B
:1028D000504944204175746F74756E652066616956
:1028E0006C6564212054656D7065726174757265E4
:1028F00020746F6F20686967680A0050494420415E
:1029000075746F74756E65206661696C65642120ED
:10291000426164206578747275646572206E756DAD
:102920006265720A004D38373620526573706F6EDB
:1029300064696E672050524F4D50545F00554E4BA6
:102940004E4F574E2053544154450047434F444542
:102950005F494E464F004C43445F50415553455FDD
:10296000524553554D450046494C414D454E545FE7
:1029700052554E4F55545F434F4E54494E554500A6
:1029800046494C414D454E545F52554E4F555400AB
:102990004D323400436F6E74696E75650050757208
:1029A0006765204D6F7265005061757365640070D6
:1029B000617573656400486F74656E6420746F6F31
:1029C00020636F6C640A0050617573650050726516
:1029D000737320627574746F6E20286F72204D318E
:1029E00030382920746F20726573756D650A00494F
:1029F0006E736572742066696C616D656E742061BA
:102A00006E6420707265737320627574746F6E20CB
:102A1000286F72204D313038290A00436F6E746977
:102A20006E75650052656865617420446F6E65005F
:102A3000526568656174696E672E2E2E0052656856
:102A4000656174696E670048656174657254696D8B
:102A5000656F7574005265686561740048656174DE
:102A6000657254696D656F7574005072657373207B
:102A7000627574746F6E20286F72204D3130382962
:102A800020746F2068656174206E6F7A7A6C650AB5
:102A9000004E6F7A7A6C65205061726B65640043FA
:102AA0006F6E74696E7565004E6F7A7A6C65205032
:102AB00061726B656400486F74656E6420746F6F3B
:102AC00020636F6C640A00726573756D65640062E3
:102AD0006567696E00436F6E74696E756500507549
:102AE0007267654D6F726500506175736564004C67
:102AF0006F61642046696C616D656E7400436F6E32
:102B000074696E7565004C6F61642046696C616D17
:102B1000656E74205400496E736572742066696C2A
:102B2000616D656E7420616E6420707265737320D0
:102B3000627574746F6E20286F72204D31303829A1
:102B40000A00526573756D6500000000000000000A
:102B500000000000000000484200004842000080E1
:102B6000405761726E696E673A20486F6D696E6793
:102B70002042756D702044697669736F72203C2025
:102B8000310A000202040000A0400000A040000042
:102B9000004000009643000096430000C843FFFF3A
:102BA000FF544D33442043522D58205265616479BF
:102BB0002E005072696E74696E672E2E2E00507250
:102BC000696E74205061757365640063616E63653E
:102BD0006C005072696E742041626F72746564009B
:102BE00055492041626F727400726573756D65009E
:102BF0004D323400290A002062797465733B2063EA
:102C00007263200053657474696E67732053746F28
:102C10007265642028006F70656E00545249474702
:102C200045524544003A20007A5F6D696E00795F35
:102C30006D696E00785F6D696E005265706F7274B9
:102C4000696E6720656E6473746F7020737461744D
:102C500075730A00205A3A0020593A0020436F75D4
:102C60006E7420583A0020453A00205A3A00205904
:102C70003A00583A0000009643000096430000C80E
:102C80004300000000000000000000000020746FFE
:102C90006F206C6F6E6720657874727573696F6EE4
:102CA0002070726576656E7465640A0020636F6CCF
:102CB0006420657874727573696F6E2070726576C2
:102CC000656E7465640A00454550524F4D2064613D
:102CD000746173697A65206572726F722E0A0029B9
:102CE0000A002062797465733B20637263200020C0
:102CF00073746F7265642073657474696E67732092
:102D000072657472696576656420280020286361A5
:102D10006C63756C6174656429210A0020213D2073
:102D200000454550524F4D20435243206D69736D0D
:102D300061746368202D202873746F726564292084
:102D4000002053697A653A2000496E6465783A201C
:102D500000204D61726C696E3D563638290A004577
:102D60004550524F4D2076657273696F6E206D69C4
:102D7000736D617463682028454550524F4D3D0086
:102D80000A20696E6974207A70726F62655F7A6F6B
:102D90006666736574203D2000454550524F4D20B6
:102DA000496E697469616C697A65640A0048617288
:102DB00064636F6465642044656661756C74205358
:102DC000657474696E6773204C6F616465640A0092
:102DD000DC050000DC050000640000004B00000082
:102DE0000000FA430000FA43000020410000964230
:102DF0000000A0420000A0420000C8430000BE4204
:102E000020204D3630332000546F6F6C2D63686185
:102E10006E67696E673A0A002055005431204C00F5
:102E20002055005430204C0046696C616D656E740D
:102E3000206C6F61642F756E6C6F6164206C656EC1
:102E4000677468733A0A00204B0020204D393030F7
:102E50002054004C696E65617220416476616E6336
:102E6000653A0A0020440020490020204D333034C8
:102E700020500020440020490020204D33303120D4
:102E800050005049442073657474696E67733A0A40
:102E90000020590020204732392053332058002089
:102EA0005A0020204D3432302053004D6573682085
:102EB000426564204C6576656C696E673A0A00204D
:102EC0005A0020590020204D323036205800486FDB
:102ED0006D65206F66667365743A0A00204A0020AB
:102EE000540020530020204D323035204200204A2B
:102EF0003C6A756E635F6465763E00416476616E20
:102F00006365643A20423C6D696E5F7365676D6509
:102F10006E745F74696D655F75733E20533C6D69B7
:102F20006E5F66656564726174653E20543C6D69D0
:102F30006E5F74726176656C5F66656564726174FC
:102F4000653E0020540020520020204D32303420B5
:102F50005000416363656C65726174696F6E20280F
:102F6000756E6974732F7332293A20503C70726900
:102F70006E745F616363656C3E20523C726574726F
:102F80006163745F616363656C3E20543C7472617D
:102F900076656C5F616363656C3E0A0020450020C6
:102FA0005A0020590020204D3230312058004D6108
:102FB00078696D756D20416363656C6572617469D4
:102FC0006F6E2028756E6974732F7332293A0A0068
:102FD000204500205A0020590020204D3230332057
:102FE00058004D6178696D756D2066656564726124
:102FF0007465732028756E6974732F73293A0A00FB
:1030000053746570732070657220756E69743A0A26
:103010000020204D3230302044300A0020204D3234
:10302000303020543120440020204D3230302044B4
:10303000002044697361626C65640A0046696C61D2
:103040006D656E742073657474696E67733A0020E1
:10305000286D6D29002020473231202020203B2080
:10306000556E69747320696E206D6D00486F6D69CF
:103070006E67204661696C6564002E0A006F70659A
:103080006E206661696C65642C2046696C653A2027
:103090000070012C0190012701B0012201C0011D27
:1030A00001F00118011002130130020E0160020943
:1030B0000190020401C002FF000003FA004003F582
:1030C000008003F000D003EB002004E6007004E170
:1030D00000E004DC004005D700C005D2004006CD6A
:1030E00000D006C8008007C3003008BE00F008B951
:1030F00000C009B400B00AAF00B00BAA00D00CA504
:1031000000000EA000500F9B00C0109600501291BE
:103110000000148C00C0158700B0178200B0197D24
:1031200000D01B7800001E730040206E00902269C2
:1031300000F024640040275F0090295A00E02B55DE
:1031400000102E500020304B0010324600E033417A
:103150000090353C001037370070383200A0392D10
:1031600000B03A2800A03B2300603C1E00103D192F
:1031700000903D1400103E0F00703E0A00C03E0556
:1031800000003F0000403FFBFF803FF6FFC03FF1E3
:10319000FF626564002C2073797374656D2073740D
:1031A0006F7070656421204865617465725F494481
:1031B0003A20004265642048656174696E67204664
:1031C00061696C65640048656174696E6720666159
:1031D000696C65640042454420544845524D414C59
:1031E0002052554E4157415900546865726D616CCB
:1031F0002052756E617761790045312048656174B0
:10320000696E67204661696C656400486561746930
:103210006E67206661696C656400453120544845DD
:10322000524D414C2052554E41574159005468650A
:10323000726D616C2052756E6177617900202D206E
:10324000496E76616C696420657874727564657224
:10325000206E756D62657220210A001000C902108F
:10326000012C014001220170011801B0010E01F092
:103270000104015002FA00B002F0003003E600D071
:1032800003DC009004D2007005C800A006BE000058
:1032900008B400B009AA00D00BA000600E96006030
:1032A000118C000015820020197800C01D6E00A04E
:1032B000226400B0275A00902C500000314600E0F4
:1032C000343C0010383200903A2800603C1E00A0C8
:1032D0003D1400803E0A00203F0000446966666598
:1032E000723A200046726F6D5374703A00537465E1
:1032F000707065723A00556E4C6576656C3A004C9C
:103300006576656C65643A005261773A202020202A
:10331000000A4C6F676963616C3A004361703A0060
:103320007601440111241FBECFEFD1E2DEBFCDBF35
:1033300000E00CBF17E0A0E0B2E0ECE4F0E302E054
:103340000BBF02C007900D92A03DB107D9F72DE148
:10335000A0EDB7E001C01D92AB36B207E1F719E16D
:10336000C1E9D9E100E006C021970109802FFE01E3
:103370000F944314C039D10780E00807A9F70E94D1
:1033800009FC0D9414180C9400002F923F924F9258
:103390005F926F927F928F929F92AF92BF92CF92E5
:1033A000DF92EF92FF920F931F93CF93DF93CDB7EE
:1033B000DEB7E3970FB6F894DEBF0FBECDBF8091A6
:1033C0000901817091E098272091F607921781F109
:1033D0009093F607811116C00E9426588091C71C51
:1033E00083FF09C082EA93E00E94EE4F61E080E033
:1033F0000E94B15E1DC060E081E00E94B15E8BEB77
:1034000093E014C00091C71C03FB002700F90E9441
:10341000B5578091C71C877F8093C71C002341F05C
:1034200060E081E00E94B15E84ED93E00E94EE4F87
:103430008091D00781FF11C18091911A9091921AC9
:10344000891B8F70843008F008C18CE0E6E9FAE04F
:10345000DE01119601900D928A95E1F78091F80AAC
:103460009091F90AA091FA0AB091FB0A88A799A74E
:10347000AAA7BBA79C01AD016091960A7091970A1B
:103480008091980A9091990A0F9457146B017C01CE
:103490006093960A7093970A8093980A9093990A7A
:1034A0008091FC0A9091FD0AA091FE0AB091FF0A5A
:1034B0008CA79DA7AEA7BFA79C01AD0160919A0AFA
:1034C00070919B0A80919C0A90919D0A0F945714C9
:1034D00068A379A38AA39BA360939A0A70939B0A1B
:1034E00080939C0A90939D0A8091000B9091010B10
:1034F000A091020BB091030B88AB99ABAAABBBAB0D
:103500009C01AD0160919E0A70919F0A8091A00A72
:103510009091A10A0F9457144B015C0160939E0A8D
:1035200070939F0A8093A00A9093A10AA701960125
:10353000C701B6010F94BA0D2B013C0128A139A196
:103540004AA15BA1CA01B9010F94BA0D9B01AC015C
:10355000C301B2010F9458142B013C01A501940141
:10356000C501B4010F94BA0D9B01AC01C301B201B6
:103570000F9458140F9406179B01AC0160E070E0A3
:1035800080E89FE30F9452152091590230915A021E
:1035900040915B0250915C020F94BA0D2DEC3CEC13
:1035A0004CEC5DE30F94BA0D20E030E040E85EE3C0
:1035B0000F94BA0D2B013C0120E030E040E85FE3BE
:1035C0000F94540D87FFF3C3A3019201C701B60105
:1035D0000F94BA0D28A539A54AA55BA50F945814D8
:1035E0006093960A7093970A8093980A9093990A29
:1035F000A301920168A179A18AA19BA10F94BA0DA0
:103600002CA53DA54EA55FA50F94581460939A0A6A
:1036100070939B0A80939C0A90939D0AA301920148
:10362000C501B4010F94BA0D28A939A94AA95BA90B
:103630000F94581460939E0A70939F0A8093A00A77
:103640009093A10A0E94A1E08CE0FE013196A6E9C8
:10365000BAE001900D928A95E1F78091F50781110A
:103660000C94A5358091F3079091F4079C012F5F8E
:103670003F4F3093F4072093F307883E934010F4B4
:103680000C94A53581E08093F5071092F407109211
:10369000F3078091DA07882309F49AC30E9474BE65
:1036A000811196C38091F2078F5F8093F20780911A
:1036B000F207853620F01092F2071092DA07E091B7
:1036C000DA078E2FEE0F990BAA0BBB0BFC0131977B
:1036D000E730F10508F0A0C08827EE58FF4F8F4F64
:1036E0000D9443140E946CBE882309F495C081E0B8
:1036F0008093000287EE93E00E94EE4F80E190E01D
:103700009093241B8093231B85E08093171B02E872
:1037100000931A1B84E190E1A0E0B0E080931B1BB2
:1037200090931C1BA0931D1BB0931E1B0E94AEF117
:1037300081E09AE59093241B8093231B86E390E01D
:103740009093261B8093251B87E08093171B009383
:103750001A1B84E890E0A0E0B0E080931B1B9093DC
:103760001C1BA0931D1BB0931E1B0E94AEF152C0E8
:103770000E946CBE882309F44FC048C085EF93E0D7
:103780000E94EE4F81E09AE59093241B8093231BC7
:1037900080E490E09093261B8093251B07E0009324
:1037A000171B82E880931A1B84E890E0A0E0B0E049
:1037B00080931B1B90931C1BA0931D1BB0931E1B7F
:1037C0000E94AEF10093DA0727C08091F1078823A9
:1037D00019F10E946CBE8823F9F00E9474BE811119
:1037E0001BC0F9C20E946CBE8823B1F00E9474BE57
:1037F000811112C01EC30E9474BE81110DC042E02F
:1038000060E070E0CB010E94B3BE04C00E9474BEB1
:10381000811102C01092DA0780910002882309F416
:10382000AEC28091D8079091D907892B09F08FC13A
:103830008091EE079091EF07892B09F01EC184E07B
:1038400096E09093241B8093231B80EA90E890934A
:10385000261B8093251B17E01093171B02E800938B
:103860001A1B80EA90E0A0E0B0E080931B1B9093CD
:103870001C1BA0931D1BB0931E1B0E94AEF18091D8
:10388000090290910A02A0910B02B0910C020097DC
:10389000A105B10511F51092241B1092231B15E010
:1038A0001093171B00931A1B8AE890E1A0E0B0E088
:1038B00080931B1B90931C1BA0931D1BB0931E1B7E
:1038C0000E94AEF189E090E09093241B8093231B2B
:1038D0001093171B00931A1B40C00196A11DB11D28
:1038E000F5E0B695A79597958795FA95D1F7019745
:1038F000A109B109009731E0A307B10558F0B093D1
:10390000241BA093231B9093261B8093251B1093AD
:10391000171B07C09093241B8093231B85E0809383
:10392000171B12E810931A1B8AE890E1A0E0B0E0A0
:1039300080931B1B90931C1BA0931D1BB0931E1BFD
:103940000E94AEF188E090E09093241B8093231BAB
:1039500085E08093171B10931A1B8CE890E1A0E080
:10396000B0E080931B1B90931C1BA0931D1BB09376
:103970001E1B0E94AEF18091090290910A02A09153
:103980000B02B0910C020097E1E0AE07B10550F0D8
:10399000B093241BA093231B9093261B8093251B7D
:1039A00087E005C09093241B8093231B85E08093C0
:1039B000171B82E880931A1B88E890E1A0E0B0E032
:1039C00080931B1B90931C1BA0931D1BB0931E1B6D
:1039D0000E94AEF18091090290910A02A0910B021F
:1039E000B0910C02BA2FA92F982F88270097F1E0E9
:1039F000AF07B10550F0B093241BA093231B909305
:103A0000261B8093251B87E005C09093241B809381
:103A1000231B85E08093171B12E810931A1B81EA81
:103A200090E0A0E0B0E080931B1B90931C1BA09340
:103A30001D1BB0931E1B0E94AEF18091100B8823BA
:103A400019F082E090E002C083E090E09093241BA4
:103A50008093231B85E08093171B10931A1B85E42A
:103A600090E1A0E0B0E080931B1B90931C1BA093FF
:103A70001D1BB0931E1B0E94AEF10091EE0710912A
:103A8000EF07053611057CF41093241B0093231BCC
:103A900085E08093171B82E880931A1B80E090E1F9
:103AA000A0E0B0E011C0C801845691099093241B96
:103AB0008093231B85E08093171B82E880931A1B59
:103AC00081E090E1A0E0B0E080931B1B90931C1B71
:103AD000A0931D1BB0931E1B0E94AEF10F5F1F4FE2
:103AE0001093EF070093EE07093C110564F183E0A2
:103AF00094E00E94EE4F81E090E09093D90780938C
:103B0000D8078093000281E09AE59093241B80936C
:103B1000231B8DE290E09093261B8093251B87E06A
:103B20008093171B82E880931A1B84E890E0A0E042
:103B3000B0E080931B1B90931C1BA0931D1BB093A4
:103B40001E1B0E94AEF11092F5070C94A5358091D2
:103B5000911A9091921A891B8F7009F094C10E945A
:103B6000D6C8811190C18091C71C82FD8CC114C33D
:103B700084E690E09093241B8093231B1093171BE3
:103B800000931A1B8EE090E1A0E0B0E080931B1B35
:103B900090931C1BA0931D1BB0931E1B0E94AEF1A3
:103BA000C60182539048880F991F9093241B8093DD
:103BB000231B1093171B00931A1B8FE090E1A0E0CA
:103BC000B0E080931B1B90931C1BA0931D1BB09314
:103BD0001E1B0E94AEF10E94D2DE90E09093241B47
:103BE0008093231B85E08093171B82E880931A1B28
:103BF00086E190E1A0E0B0E080931B1B90931C1B3A
:103C0000A0931D1BB0931E1B0E94AEF160917C1906
:103C100070917D19072E000C880B990B0F945B0D8A
:103C200020E030E048EC52E40F94BA0D0F94C41534
:103C30007093241B6093231B15E01093171B02E85D
:103C400000931A1B86E290E1A0E0B0E080931B1B7A
:103C500090931C1BA0931D1BB0931E1B0E94AEF1E2
:103C600060913A0870913B0880913C0890913D0822
:103C70000F94C4157093241B6093231B1093171B80
:103C800000931A1B86E390E1A0E0B0E080931B1B39
:103C900090931C1BA0931D1BB0931E1B0E94AEF1A2
:103CA0006091510870915208809153089091540886
:103CB0000F94C4157093241B6093231B1093171B40
:103CC00000931A1B8CE390E1A0E0B0E080931B1BF3
:103CD00090931C1BA0931D1BB0931E1B0E94AEF162
:103CE00080913E0890913F089093241B8093231B62
:103CF0001093171B00931A1B84E390E1A0E0B0E03F
:103D000080931B1B90931C1BA0931D1BB0931E1B29
:103D10000E94AEF180915508909156089093241B13
:103D20008093231B1093171B00931A1B8AE390E1C7
:103D3000A0E0B0E080931B1B90931C1BA0931D1B65
:103D4000B0931E1B0E94AEF10091EA0701113CC125
:103D50008091EC07811138C18091F10781118BC1ED
:103D60008091CB1A9091CC1AA091CD1AB091CE1A15
:103D70008C3420E19207A105B10509F0A1C137E615
:103D8000C32E3BE1D32E0AE18DE799E10E94FE5557
:103D9000E090DF07F090E007181619060CF085C3D5
:103DA0008AE1E816F10414F40C94C9317EC38CE066
:103DB000FE013196A6E9BAE001900D928A95E1F7ED
:103DC0000E94A1E08091D0078D7F8093D00745CCE1
:103DD0001092F2076CCC8DEC95E00E94EE4F809132
:103DE000F00790E0A0E0B0E0895B9F4FAE4FB54A8E
:103DF00021E03AE53093241B2093231B9093261B4C
:103E00008093251B87E08093171B82E880931A1B01
:103E100084E890E0A0E0B0E080931B1B90931C1B13
:103E2000A0931D1BB0931E1B0E94AEF11092F107D0
:103E3000F1CC81E0809300021092DA078BED95E0DF
:103E40000E94EE4F81E09AE59093241B8093231B00
:103E50008EE490E09093261B8093251B87E080934F
:103E6000171B82E880931A1B84E890E0A0E0B0E082
:103E700080931B1B90931C1BA0931D1BB0931E1BB8
:103E80000E94AEF1C9CC8CE090E09093241B80930B
:103E9000231B05E00093171B82E880931A1B84E123
:103EA00090E1A0E0B0E080931B1B90931C1BA093BB
:103EB0001D1BB0931E1B0E94AEF10E94B4DD20E1D9
:103EC0003EE040E050E00F94AA132115310591E047
:103ED0004907510560F05093241B4093231B3093F6
:103EE000261B2093251B87E08093171B06C0309369
:103EF000241B2093231B0093171B02E800931A1B1B
:103F000080E190E1A0E0B0E080931B1B90931C1B2C
:103F1000A0931D1BB0931E1B0E94AEF10E94B4DD46
:103F200020E13EE040E050E00F94AA132CE330E0A3
:103F300040E050E00F94AA133093241B2093231BDE
:103F400015E01093171B00931A1B82E190E1A0E08B
:103F5000B0E080931B1B90931C1BA0931D1BB09380
:103F60001E1B0E94AEF10E94D2DE882391F00E94B7
:103F7000D2DE8F5F8093ED07C82ED12C833308F0FB
:103F8000F7CDC601880F991F9093241B8093231BA4
:103F900004C01092241B1092231B1093171B009334
:103FA0001A1B8EE090E1A0E0B0E080931B1B909381
:103FB0001C1BA0931D1BB0931E1B0E94AEF1109200
:103FC000241B1092231BF5CD20E030E048EC52E496
:103FD00060913A0870913B0880913C0890913D08AF
:103FE0000F94BA0D6B017C0160913E0870913F08FF
:103FF000072E000C880B990B0F945B0D9B01AC01F5
:10400000C701B6010F9452150F94CB156436710594
:1040100010F064E670E07093241B6093231B45E06E
:10402000A42EA092171B52E8B52EB0921A1B84E260
:1040300090E1A0E0B0E080931B1B90931C1BA09329
:104040001D1BB0931E1B0E94AEF1C0903A08D09089
:104050003B08E0903C08F0903D0820E030E040E272
:1040600053E4C701B6010F94B81618160CF03AC104
:10407000011188C137C18091E10701E0080F009369
:10408000E10790E09093241B8093231B85E08093AD
:10409000171B82E880931A1B82E490E1A0E0B0E055
:1040A00080931B1B90931C1BA0931D1BB0931E1B86
:1040B0000E94AEF10A3008F453CE1092E10750CEC0
:1040C0008A349041A105B10509F459CE80E00E94DF
:1040D00091BF20E030E040E251E40F94BA0D0F941C
:1040E000C4157093241B6093231B15E01093171BBA
:1040F00002E800931A1B88E490E1A0E0B0E080930E
:104100001B1B90931C1BA0931D1BB0931E1B0E9496
:10411000AEF181E00E9491BF20E030E040E251E446
:104120000F94BA0D0F94C4157093241B6093231B36
:104130001093171B00931A1B8AE490E1A0E0B0E0F3
:1041400080931B1B90931C1BA0931D1BB0931E1BE5
:104150000E94AEF182E00E9491BF20E030E040E298
:1041600051E40F94BA0D0F94C4157093241B6093FF
:10417000231B1093171B00931A1B8CE490E1A0E003
:10418000B0E080931B1B90931C1BA0931D1BB0934E
:104190001E1B0E94AEF1F3CD809151089091520800
:1041A000A0915308B091540888A399A3AAA3BBA3D4
:1041B0006091550870915608072E000C880B990BDA
:1041C0000F945B0D6B017C0120E030E040E050E497
:1041D0000F94571428A139A14AA15BA10F94B816D6
:1041E000181604F140903A0850903B0860903C0843
:1041F00070903D0860913E0870913F08072E000CBA
:10420000880B990B0F945B0D4B015C0120E030E0B3
:1042100040E251E40F945714A30192010F94B81691
:10422000181604F58DE090E09093241B8093231BD7
:1042300085E08093171B82E880931A1B84E190E14C
:10424000A0E0B0E080931B1B90931C1BA0931D1B50
:10425000B0931E1B0E94AEF18091D60781113FC022
:1042600081E03DC020E030E040E050E4C701B6010D
:104270000F94581428A139A14AA15BA10F94540DA1
:1042800087FD0EC020E030E040E251E4C501B401FA
:104290000F945814A30192010F94540D87FFB6CCCC
:1042A00084E190E09093241B8093231B85E080930E
:1042B000171B82E880931A1B84E190E1A0E0B0E034
:1042C00080931B1B90931C1BA0931D1BB0931E1B64
:1042D0000E94AEF18091D607811101C082E08093E7
:1042E000D60794CC60913E0870913F08072E000CD1
:1042F000880B990B0F945B0D9B01AC01C701B601B4
:104300000F94B8166091EC0787FDAEC0662309F4E0
:1043100023CD062E000C770B8FE996E00E94BB4E52
:104320001092EC071092EF071092EE0784E090E0F5
:104330009093241B8093231B85E08093171B02E836
:1043400000931A1B8EE890E1A0E0B0E080931B1B65
:1043500090931C1BA0931D1BB0931E1B0E94AEF1DB
:1043600081E09AE59093241B8093231B83E590E0E2
:104370009093261B8093251B87E08093171B009347
:104380001A1B63C01092EA0720E030E040E251E4DB
:104390006091E2077091E3078091E4079091E5074F
:1043A0000F94BA0D0F94C4157093241B6093231BB4
:1043B000A092171BB0921A1B84E590E1A0E0B0E038
:1043C00080931B1B90931C1BA0931D1BB0931E1B63
:1043D0000E94AEF120E030E040E251E46091E60757
:1043E0007091E7078091E8079091E9070F94BA0D63
:1043F0000F94C4157093241B6093231BA092171B6A
:10440000B0921A1B88E590E1A0E0B0E080931B1BFE
:1044100090931C1BA0931D1BB0931E1B0E94AEF11A
:1044200089EE95E00E94EE4F81E09AE59093241B7F
:104430008093231B81E490E09093261B8093251B9F
:1044400087E08093171BB0921A1B84E890E0A0E0ED
:10445000B0E080931B1B90931C1BA0931D1BB0937B
:104460001E1B0E94AEF178CC662309F475CC8091B6
:10447000EE079091EF079C012F5F3F4F3093EF07BE
:104480002093EE0765E070E00F942F149093241BA7
:104490008093231B85E08093171B82E880931A1B6F
:1044A0008EE890E1A0E0B0E0D4CF1E141F040CF021
:1044B0004ACB9091C81A8091671B981322C09091A3
:1044C000C91A8091681B98131CC023E0E216F104FE
:1044D000C4F09091691B9093C71A80916A1B8093D6
:1044E000CA1A9330D1F4982F9D7F9038B1F49091EF
:1044F0006B1B9F3409F059C090916C1B9B3409F0E1
:1045000054C08AE1E7E6FBE1DF011D928A95E9F7F5
:104510001092E0071092DF0716CB833809F045C0F0
:1045200080916B1B90916C1B982789279827A0E09E
:10453000B0E08093CB1A9093CC1AA093CD1AB0938D
:10454000CE1AC0906D1BD12CE12CF12CC092CF1A49
:10455000D092D01AE092D11AF092D21AAEE6BBE114
:1045600040E050E0BA014C155D056E057F0508F08E
:104570004AC04A015B01B694A79497948794F401CA
:104580003696EE0FFF1FE953F54E8C9190E0982F71
:10459000882711962C911197822B918380834E5FEF
:1045A0005F4F6F4F7F4F1296DECF813861F580915C
:1045B0006B1B90E0A0E0B0E08093CB1A9093CC1AF4
:1045C000A093CD1AB093CE1A80916C1B482F50E067
:1045D00060E070E04093CF1A5093D01A6093D11AE4
:1045E0007093D21AADE6BBE1E3EDFAE190E020E092
:1045F00030E02817390739F04D9150E0419351933D
:104600002F5F3F4FF6CF8AE1E7E6FBE1DF011D9226
:104610008A95E9F71092E0071092DF0784E194E0B1
:104620000E94EE4F6091DA07161664F4062E000C15
:10463000770B84E996E00E94BB4E8AE00E940D4D04
:104640000C94BA316091D31A7091D41A82E896E032
:104650000E94924E8AE00E940D4D4091CB1A5091DB
:10466000CC1A6091CD1A7091CE1A83E796E00E9421
:10467000814E8AE00E940D4D8091CB1A9091CC1A08
:10468000A091CD1AB091CE1AE3E7F2E000E010E07D
:1046900041915191619171914115510561057105EA
:1046A000D1F1481759076A077B0791F5AC01BD01A5
:1046B0004850504161097109453051056105710546
:1046C00068F1AC01BD01477F42335041610571057E
:1046D00041F18433F0E19F07A105B10511F1AC016F
:1046E000BD014654504161097109473051056105CA
:1046F0007105D0F0AC01BD0144555041610971090B
:10470000453051056105710588F402E110E00EC0E5
:104710000F5F1F4FBDCF0FEF1FEF08C003E010E08A
:1047200005C008E010E002C00FE010E08A5090429F
:10473000A109B109833D9105A105B10530F00F3FF5
:104740002FEF120721F40C94BA3109E110E0F5E3E0
:10475000CF2EF4E0DF2EF60181916F01882319F04E
:104760000E940D4DF8CFB801012E000C880B990B5B
:104770000E949F4E0E94E84F87E696E00E94EE4F0F
:104780000A31110510F00C94B631F8018827E7586A
:10479000FF4F8F4F0D9443148091D31A9091D41AE8
:1047A00081309105E1F4109200028FEF80936F0D3C
:1047B00060E080E00E94B15E03E414E0D8018D91D6
:1047C0008D01882319F00E940D4DF8CF81E09AE504
:1047D0009093241B8093231B8EE290E0AFC0823025
:1047E000910509F0B7C081E0809300020E9443DF89
:1047F00083E696E090938A08809389088BE090E0A6
:104800009093241B8093231B05E00093171B12E851
:1048100010931A1B80E092E1A0E0B0E080931B1B94
:1048200090931C1BA0931D1BB0931E1B0E94AEF106
:104830001092241B1092231B0093171B10931A1B1A
:104840008EE090E1A0E0B0E080931B1B90931C1BD6
:10485000A0931D1BB0931E1B0E94AEF11092241B4F
:104860001092231B0093171B10931A1B8FE090E1EB
:10487000A0E0B0E080931B1B90931C1BA0931D1B1A
:10488000B0931E1B0E94AEF11092241B1092231BAA
:104890000093171B10931A1B86E190E1A0E0B0E093
:1048A00080931B1B90931C1BA0931D1BB0931E1B7E
:1048B0000E94AEF162E070E080E090E00E94A5BF4F
:1048C0001092241B1092231B0093171B10931A1B8A
:1048D00080E190E1A0E0B0E080931B1B90931C1B53
:1048E000A0931D1BB0931E1B0E94AEF11092241BBF
:1048F0001092231B0093171B10931A1B82E190E167
:10490000A0E0B0E080931B1B90931C1BA0931D1B89
:10491000B0931E1B0E94AEF10DE614E0F8018191E8
:104920008F01882319F00E940D4DF8CF81E09AE5A0
:104930009093241B8093231B8DE290E09093261B81
:104940008093251B87E08093171B82E880931A1BB6
:104950000C94D7328330910549F581E080930002B1
:1049600007E914E0D8018D918D018823C9F00E94D8
:104970000D4DF8CF8091CB1A9091CC1AA091CD1A01
:10498000B091CE1A8233F0E19F07A105B10509F07D
:104990005CC48091D31A9091D41A009709F022C474
:1049A00080910802882309F40CC31CC3049711F0FA
:1049B0000C94BA31109200020C94BA318091D31A3F
:1049C0009091D41A81309105D9F41092000280910F
:1049D0000802882319F082E090E002C083E090E0B2
:1049E0009093241B8093231B85E08093171B82E800
:1049F00080931A1B8EE190E1A0E0B0E00C94DB32D2
:104A00008230910519F501EC14E0F80181918F01D4
:104A1000882319F00E940D4DF8CF81E080930002A9
:104A20008091D607843049F081E09AE59093241B69
:104A30008093231B85E390E081CF81E09AE59093FA
:104A4000241B8093231B86E390E078CF833091056D
:104A500009F04CC020910802222319F19093241BE5
:104A60008093231B85E08093171B82E880931A1B99
:104A70008EE190E1A0E0B0E080931B1B90931C1BA3
:104A8000A0931D1BB0931E1B0E94AEF140E060E09E
:104A900070E088EC92E40E94AADF109208020C9465
:104AA000BA3182E090E09093241B8093231B85E031
:104AB0008093171B82E880931A1B8EE190E1A0E09F
:104AC000B0E080931B1B90931C1BA0931D1BB09305
:104AD0001E1B0E94AEF140E060E070E0CB010E943E
:104AE000AADF81E0809308020C94BA31049711F098
:104AF0000C94BA31809164088823F1F082E090E050
:104B00009093241B8093231B85E08093171B82E8DE
:104B100080931A1B8FE190E1A0E0B0E080931B1B13
:104B200090931C1BA0931D1BB0931E1B0E94AEF103
:104B3000109264080C94BA3183E090E09093241BA7
:104B40008093231B85E08093171B82E880931A1BB8
:104B50008FE190E1A0E0B0E080931B1B90931C1BC1
:104B6000A0931D1BB0931E1B0E94AEF181E08093A9
:104B700064080C94BA316091D31A7091D41A80E011
:104B800090E00F94590D6B017C0120E030E04AEF7A
:104B900053E40F94540D87FF11C020E030E040E251
:104BA00051E4C701B6010F94B81618166CF0C12C69
:104BB000D12C70E2E72E71E4F72E06C0C12CD12C67
:104BC000EAEFEE2EE3E4FE2EC701B6010F94C41502
:104BD00070936D0260936C020C94BA318091CB1A81
:104BE0009091CC1AA091CD1AB091CE1A8830F0E1F4
:104BF0009F07A105B10509F050C081E09AE59093A7
:104C0000241B8093231B8DE290E09093261B8093BE
:104C1000251B87E08093171B12E810931A1B84E86A
:104C200090E0A0E0B0E080931B1B90931C1BA0932E
:104C30001D1BB0931E1B0E94AEF11092241B1092FC
:104C4000231B05E00093171B10931A1B80E190E1D2
:104C5000A0E0B0E080931B1B90931C1BA0931D1B36
:104C6000B0931E1B0E94AEF11092241B1092231BC6
:104C70000093171B10931A1B82E190E1A0E0B0E0B3
:104C800080931B1B90931C1BA0931D1BB0931E1B9A
:104C90000E94AEF10E9443DF8FC08A3020E192076C
:104CA000A105B105E1F58091D31A9091D41A813F05
:104CB000910511F00C94BA3181E09AE59093241B90
:104CC0008093231B86E390E09093261B8093251B03
:104CD00087E08093171B82E880931A1B84E890E09A
:104CE000A0E0B0E080931B1B90931C1BA0931D1BA6
:104CF000B0931E1B0E94AEF14CE355E063E475E0F7
:104D000084E00E948ACD60E08FE295E00E9404DF9B
:104D100085E295E090938A08809389084DC08C3095
:104D20009041A105B10509F047C08091D31A909137
:104D3000D41A019709F040C00F94FE051092D607CF
:104D400081E0809300028CE090E09093241B80939C
:104D5000231B85E08093171B12E810931A1B84E134
:104D600090E1A0E0B0E080931B1B90931C1BA093EC
:104D70001D1BB0931E1B0E94AEF181E09AE590933B
:104D8000241B8093231B85E390E09093261B809344
:104D9000251B87E08093171B10931A1B84E890E073
:104DA000A0E0B0E080931B1B90931C1BA0931D1BE5
:104DB000B0931E1B0E94AEF18091CB1A9091CC1A39
:104DC000A091CD1AB091CE1A8C309041A105B105B9
:104DD00011F00C94BA318091D31A9091D41A0297A1
:104DE00011F00C94BA310F94FE0581E08093EC072A
:104DF0001092D607809300021092EF071092EE07F0
:104E000081E09AE59093241B8093231B82E590E038
:104E100095CD2091D31A3091D41AB90180E090E059
:104E200037FF09C00F94590D20E030E040E857E407
:104E30000F94571402C00F94590D20E030E048EC55
:104E400052E40F9452156B017C0120E030E040EAFF
:104E500051EC0F94B81600917C1910917D1987FDC3
:104E60002BC020E030E040EA51E4C701B6010F94C6
:104E7000540D18160CF1B801110F880B990B0F94F3
:104E80005B0DA70196010F94571420E030E048EC29
:104E900053E40F94BA0D90580F94C415CB010E949F
:104EA000F2F3C701B6010E948ABE8EE596E09093A8
:104EB0008A088093890826C0B801110F880B990BC6
:104EC0000F945B0D20E030E048EC52E40F94BA0DF3
:104ED0000F94C4157093241B6093231B85E080936B
:104EE000171B82E880931A1B86E290E1A0E0B0E0F5
:104EF00080931B1B90931C1BA0931D1BB0931E1B28
:104F00000E94AEF160917C1970917D19072E000C02
:104F1000880B990B0F945B0D8E010B5E1F4F23E0E6
:104F200041E00F942C089F938F9380E596E09F9328
:104F30008F93045111091F930F930F94EC0CC80128
:104F40000E947FC00F900F900F900F900F900F90C6
:104F50000C94BA318091D31A9091D41A009729F405
:104F600081E0809300020C94BA3181309105B1F454
:104F700080910802882349F081E09AE59093241BF0
:104F80008093231B8CE390E0D9CC81E09AE5909349
:104F9000241B8093231B8BE390E0D0CC82309105BF
:104FA000F9F28330910539F58091080240E08823B9
:104FB00089F060E070E088EC92E40E94AADF109231
:104FC000080281E09AE59093241B8093231B89E3D8
:104FD00090E0B4CC60E070E0CB010E94AADF81E0F9
:104FE0008093080281E09AE59093241B8093231B11
:104FF0008AE390E0A3CC8530910559F540E060E06C
:1050000070E084E393E40E94FFBD46E060E070E05E
:105010008CE892E40E94FFBD84EB90E09093241B07
:105020008093231B05E00093171B12E810931A1BB3
:1050300084E390E1A0E0B0E080931B1B90931C1BE5
:10504000A0931D1BB0931E1B0E94AEF186E490E05E
:105050002DC08630910599F540E060E070E080E772
:1050600093E40E94FFBD46E060E070E08CED92E4C6
:105070000E94FFBD80EF90E09093241B8093231B40
:1050800005E00093171B12E810931A1B84E390E1CC
:10509000A0E0B0E080931B1B90931C1BA0931D1BF2
:1050A000B0931E1B0E94AEF18EE690E09093241BFD
:1050B0008093231B0093171B10931A1BC0C0813FC2
:1050C000910511F00C94BA3140E060E070E0CB0142
:1050D0000E94AADF41E060E070E0CB010E94AADFFD
:1050E0001092080240E060E070E0CB010E94FFBD3A
:1050F00046E060E070E0CB010E94FFBD1092241BEF
:105100001092231B05E00093171B12E810931A1B43
:1051100084E390E1A0E0B0E080931B1B90931C1B04
:10512000A0931D1BB0931E1B0E94AEF161E070E0C6
:1051300080E090E00E94A5BF1092241B1092231BD8
:105140000093171B10931A1B8AE390E1A0E0B0E0D4
:1051500080931B1B90931C1BA0931D1BB0931E1BC5
:105160000E94AEF161E070E080E090E00E94A5BF97
:1051700084E190E09093241B8093231B0093171BE2
:1051800010931A1B84E190E1A0E0B0E080931B1B18
:1051900090931C1BA0931D1BB0931E1B0E94AEF18D
:1051A00081E09AE59093241B8093231B89E390E090
:1051B0009093261B8093251B87E08093171B1093E9
:1051C0001A1B84E890E0A0E0B0E080931B1B909352
:1051D0001C1BA0931D1BB0931E1B0E94AEF182E00E
:1051E0000C94B33181309105B1F440E060E070E09F
:1051F000CB010E94FFBD1092241B1092231B85E05F
:105200008093171B82E880931A1B84E390E1A0E04F
:10521000B0E00C94DB32029711F00C94BA3146E006
:1052200060E070E0CB010E94FFBD1092241B109241
:10523000231B85E08093171B82E880931A1B8AE367
:1052400090E1A0E0B0E00C94DB32843320E19207DF
:10525000A105B10551F46091D31A7091D41A80E080
:1052600090E00F94590D40E010C08A339041A105A1
:10527000B10511F00C94BA316091D31A7091D41A1F
:1052800080E090E00F94590D46E00E94FFBD0C9421
:10529000BA318091D31A9091D41A009709F460CE54
:1052A0008130910509F04CC08091100B882319F0D2
:1052B00083E090E002C082E090E09093241B809312
:1052C000231B85E08093171B82E880931A1B85E4DB
:1052D00090E1A0E0B0E080931B1B90931C1BA09377
:1052E0001D1BB0931E1B0E94AEF18AE090E09093CC
:1052F000241B8093231B85E08093171B82E88093F7
:105300001A1B80E092E1A0E0B0E080931B1B909319
:105310001C1BA0931D1BB0931E1B0E94AEF10E948C
:105320006CBE811103C080E496E002C084E396E085
:1053300090938A088093890882E08093DA0772C18B
:105340008230910509F0A8C081E08093000288E0D6
:10535000E2EEF7E0DF011D928A95E9F780E090E048
:10536000A0E2B1E48093E2079093E307A093E407FF
:10537000B093E5078093E6079093E707A093E807CB
:10538000B093E90784E690E09093241B8093231B5D
:1053900005E00093171B12E810931A1B84E590E1B7
:1053A000A0E0B0E080931B1B90931C1BA0931D1BDF
:1053B000B0931E1B0E94AEF120E030E040E251E4C9
:1053C0006091E6077091E7078091E8079091E907FF
:1053D0000F94BA0D0F94C4157093241B6093231B74
:1053E0000093171B10931A1B88E590E1A0E0B0E032
:1053F00080931B1B90931C1BA0931D1BB0931E1B23
:105400000E94AEF160913A0870913B0880913C088F
:1054100090913D080F94C4157093241B6093231B37
:105420000093171B10931A1B86E390E1A0E0B0E0F5
:1054300080931B1B90931C1BA0931D1BB0931E1BE2
:105440000E94AEF180913E0890913F089093241BFA
:105450008093231B0093171B10931A1B84E390E186
:10546000A0E0B0E080931B1B90931C1BA0931D1B1E
:10547000B0931E1B0E94AEF162E070E080E090E00D
:105480000E94A5BF81E09AE59093241B8093231B83
:1054900081E490E00C94CE328330910509F077C01E
:1054A0001092F00780E00E9491BF20E030E040E2DF
:1054B00051E40F94BA0D0F94C4157093241B60939C
:1054C000231B05E00093171B12E810931A1B88E4B6
:1054D00090E1A0E0B0E080931B1B90931C1BA09375
:1054E0001D1BB0931E1B0E94AEF181E00E9491BF74
:1054F00020E030E040E251E40F94BA0D0F94C4155F
:105500007093241B6093231B0093171B10931A1B8B
:105510008AE490E1A0E0B0E080931B1B90931C1BF9
:10552000A0931D1BB0931E1B0E94AEF182E00E944F
:1055300091BF20E030E040E251E40F94BA0D0F94A7
:10554000C4157093241B6093231B0093171B1093A7
:105550001A1B8CE490E1A0E0B0E080931B1B9093B9
:105560001C1BA0931D1BB0931E1B0E94AEF162E09A
:1055700070E080E090E00E94A5BF81E09AE5909302
:10558000241B8093231B87E490E00C94CE3284305C
:10559000910509F4EFC68530910549F44EE750E1D5
:1055A00060E070E088EE94E00E945DF1E3C606974B
:1055B00009F0E0C680E396E090938A08809389081A
:1055C0008BE090E053C28091D31A9091D41A019746
:1055D00011F51092000281E09AE59093241B8093CC
:1055E000231B8FE390E09093261B8093251B87E07D
:1055F0008093171B82E880931A1B84E890E0A0E058
:10560000B0E080931B1B90931C1BA0931D1BB093B9
:105610001E1B0E94AEF18091D31A9091D41A02976A
:1056200009F0A8C681E09AE59093241B8093231B80
:1056300080E490E083C98091D31A9091D41A8E357A
:10564000910509F4A5C168F58330910509F45FC19E
:10565000A0F48130910509F46EC1029709F000C2EF
:1056600042E060E070E080E890E40E94B3BE40E079
:1056700060E070E082E893E46AC18430910509F447
:1056800073C1059709F0ECC142E060E070E080E88A
:1056900090E40E94B3BE40E060E070E082E893E4F2
:1056A0006FC18136910509F469C098F58F35910570
:1056B00009F48AC08036910509F0D2C183E0809355
:1056C000DA0783E090E09093241B8093231B85E00E
:1056D0008093171B82E880931A1B8DE890E1A0E06D
:1056E000B0E080931B1B90931C1BA0931D1BB093D9
:1056F0001E1B0E94AEF1E12CF12C00E0DD24D394BE
:10570000AA24A39445E0942E55E0852E62E8762ED7
:1057100085C08236910561F08336910509F0A0C1FC
:1057200080917C1980FF60C6869580FD60C65CC64E
:1057300060917C1970917D19072E000C880B990BD4
:105740000F945B0D2DEC3CEC4CEC5DE30F94581486
:105750006B017C0120E030E040EA51EC0F94B81678
:1057600087FD82C120E030E040EA51E4C701B60184
:105770000F94540D18160CF041C676C160917C1937
:1057800070917D19072E000C880B990B0F945B0DFF
:105790002DEC3CEC4CEC5DE30F9457146B017C0159
:1057A00020E030E040EA51EC0F94B81687FD5CC170
:1057B00020E030E040EA51E4C701B6010F94540DF7
:1057C00018160CF07EC650C180E00E94224C0E9448
:1057D0006CBE811103C087ED95E002C089EC95E0B5
:1057E00090938A088093890882E08093DA0781E0A9
:1057F0009AE59093241B8093231B84E590E090937B
:10580000261B8093251B87E08093171B82E88093DB
:105810001A1B84E890E0A0E0B0E017C1DD2031F071
:10582000CC24C39435E0B32E10E005C0CC24CA9438
:10583000BB24BA9414E0DA24B116D1F1802F90E0A1
:105840004897A4F50F5FF701919EE00DF11D11241B
:10585000EE0FFF1FEE0FFF1FE253F74E20E030E088
:105860004AE754E460817181828193810F94BA0D7B
:105870000F94C4157093241B6093231B8092171BF5
:1058800070921A1B802F90E08158974F880F991FB4
:10589000092E000CAA0BBB0B80931B1B90931C1BA7
:1058A000A0931D1BB0931E1B0E94AEF11C0DC4CF14
:1058B000BFEFEB1AFB0AE5E0EE16F10409F0AECFFC
:1058C00081E09AE59093241B8093231B85E590E06B
:1058D0009093261B8093251B87E08093171B82E8FB
:1058E00080931A1B84E890E0A0E0B0E080931B1B3B
:1058F00090931C1BA0931D1BB0931E1B0E94AEF126
:1059000085EC95E090938A0880938908ADC042E0C9
:1059100060E070E080E890E40E94B3BE40E060E0A8
:1059200070E086E193E40E94B3BE41E060E070E085
:1059300086E193E413C042E060E070E080E890E428
:105940000E94B3BE40E060E070E080E292E40E941A
:10595000B3BE41E060E070E080E292E40E94B3BE3A
:1059600086E08093DA0780C042E060E070E080E883
:1059700090E40E94B3BE40E060E070E080E292E418
:105980000E94B3BE41E060E070E082E893E4E6CFBD
:105990008091100B81111CC083E090E09093241B38
:1059A0008093231B85E08093171B82E880931A1B4A
:1059B00085E490E1A0E0B0E080931B1B90931C1B5A
:1059C000A0931D1BB0931E1B0E94AEF181E01BC073
:1059D00082E090E09093241B8093231B85E08093CA
:1059E000171B82E880931A1B85E490E1A0E0B0E0E9
:1059F00080931B1B90931C1BA0931D1BB0931E1B1D
:105A00000E94AEF180E00E94224C60917C1970915E
:105A10007D19072E000C880B990B0F945B0D20E06D
:105A200030E048EC52E40F94BA0D0F94C415709313
:105A3000241B6093231B85E08093171B82E88093CF
:105A40001A1B86E290E1A0E0B0E080931B1B9093CC
:105A50001C1BA0931D1BB0931E1B0E94AEF104C023
:105A600089EA95E00E94EE4F8AE090E09093241B33
:105A70008093231B85E08093171B82E880931A1B79
:105A80004BC184E08093DA078091CB1A9091CC1AB5
:105A9000A091CD1AB091CE1A6091D31A7091D41AF8
:105AA0008834F0E19F07A105B10509F453C08A3499
:105AB00020E19207A105B10509F456C08C3430E10C
:105AC0009307A105B10509F45AC086349041A10598
:105AD000B10509F05EC063307105B9F588E995E05C
:105AE00090938A088093890881E08093F1078093DE
:105AF00000021092E10781E09AE59093241B8093C5
:105B0000231B8AE490E09093261B8093251B87E05B
:105B10008093171B12E810931A1B84E890E0A0E012
:105B2000B0E080931B1B90931C1BA0931D1BB09394
:105B30001E1B0E94AEF18AE090E09093241B80939C
:105B4000231B85E08093171BE5C06093F00710923C
:105B5000DA0710C480E090E0A6E9B3E48CA39DA32B
:105B6000AEA3BFA3312C15C080E090E0A6E9B3E45A
:105B70008CA39DA3AEA3BFA3332433940AC080E0BB
:105B800090E0A8ECB3E48CA39DA3AEA3BFA382E0F6
:105B9000382E80E090E00F94590D20E030E040E294
:105BA00051E40F9452156B017C0120E030E0A90113
:105BB0000F94540D87FF09C01092DB071092DC0789
:105BC0001092DD071092DE071FC02CA13DA14EA14F
:105BD0005FA1C701B6010F94B81618164CF0C09219
:105BE000DB07D092DC07E092DD07F092DE070CC005
:105BF0008CA19DA1AEA1BFA18093DB079093DC0790
:105C0000A093DD07B093DE076091DB077091DC079E
:105C10008091DD079091DE07432D0E94B3BE61E0C5
:105C200070E080E090E00E94A5BF80E00E9491BFFC
:105C300020E030E040E251E40F94BA0D0F94C41517
:105C40007093241B6093231B05E00093171B12E83D
:105C500010931A1B88E490E1A0E0B0E080931B1B36
:105C600090931C1BA0931D1BB0931E1B0E94AEF1B2
:105C700081E00E9491BF20E030E040E251E40F94C7
:105C8000BA0D0F94C4157093241B6093231B0093CB
:105C9000171B10931A1B8AE490E1A0E0B0E08093F8
:105CA0001B1B90931C1BA0931D1BB0931E1B0E94DB
:105CB000AEF182E00E9491BF20E030E040E251E48A
:105CC0000F94BA0D0F94C4157093241B6093231B7B
:105CD0000093171B10931A1B8CE490E1A0E0B0E036
:105CE00080931B1B90931C1BA0931D1BB0931E1B2A
:105CF0000E94AEF161E070E080E090E00E94A5BFFC
:105D00001092DA078AE090E09093241B8093231B83
:105D10000093171B10931A1B80E092E1A0E0B0E003
:105D20004AC48091CB1A9091CC1AA091CD1AB0910F
:105D3000CE1A8635E0E19E07A105B10509F041C004
:105D400020E030E040E253E460913A0870913B0873
:105D500080913C0890913D080F94540D2091D31AE6
:105D60003091D41A87FF32C42530310508F02EC493
:105D700080EA90E09093241B8093231B85E080931E
:105D8000171B12E810931A1B80E290E1A0E0B0E02C
:105D900080931B1B90931C1BA0931D1BB0931E1B79
:105DA0000E94AEF165E070E080E090E00E94A5BF47
:105DB00081E09AE59093241B8093231B82E490E07A
:105DC000EDC38435F0E19F07A105B105B9F46091F9
:105DD000D31A7091D41A80E090E00F94590D20E00E
:105DE00030E040E251E40F9452156093E207709363
:105DF000E3078093E4079093E507BCC288359041A0
:105E0000A105B10509F0B6C26091D31A7091D41AF8
:105E100080E090E00F94590D20E030E040E251E442
:105E20000F9452156093E6077093E7078093E80795
:105E30009093E9079FC26091D31A7091D41A82E8B7
:105E400095E00E94924E8091D31A9091D41A82309C
:105E50009105A1F038F4009771F00197E1F481E128
:105E600095E086C28430910599F058F0059799F431
:105E700087E595E008C08BEF94E07AC284E795E06F
:105E800002C08AE695E090938A088093890872C2DE
:105E900085E695E0F8CF85E295E06AC284E395E077
:105EA0000E94EE4F8091D31A9091D41A81309105BF
:105EB00009F046C082E495E00E94EE4F81E00E9426
:105EC0006ED08DE090E09093241B8093231B85E09F
:105ED0008093171B12E810931A1B84E190E1A0E055
:105EE000B0E080931B1B90931C1BA0931D1BB093D1
:105EF0001E1B0E94AEF183E08093D60781E09AE5F5
:105F00009093241B8093231B85E390E09093261BA2
:105F10008093251B87E08093171B10931A1B84E83E
:105F200090E0A0E0B0E080931B1B90931C1BA0931B
:105F30001D1BB0931E1B0E94AEF11092D1071AC216
:105F4000892B09F017C28AE595E00E94EE4F8091F7
:105F5000D107813039F580E795E00E94EE4F81E06E
:105F60009AE59093241B8093231B8EE290E09093FC
:105F7000261B8093251B87E08093171B82E8809364
:105F80001A1B84E890E0A0E0B0E080931B1B909384
:105F90001C1BA0931D1BB0931E1B0E94AEF1109200
:105FA000D50735C0823069F484E895E00E94EE4F51
:105FB00081E09AE59093241B8093231B86E390E075
:105FC0000EC0833031F588E995E00E94EE4F81E004
:105FD0009AE59093241B8093231B81E490E0909397
:105FE000261B8093251B87E08093171B82E88093F4
:105FF0001A1B84E890E0A0E0B0E080931B1B909314
:106000001C1BA0931D1BB0931E1B0E94AEF110928F
:1060100043191092D1070E9443DFACC18091D31A7B
:106020009091D41A8F3F910531F028F08FEF90E0D6
:10603000A0E0B0E002C0A0E0B0E08093090290933D
:106040000A02A0930B02B0930C0280910902909176
:106050000A02A0910B02B0910C020097A105B105B4
:1060600009F51092241B1092231B05E00093171BC7
:1060700012E810931A1B8AE890E1A0E0B0E0809348
:106080001B1B90931C1BA0931D1BB0931E1B0E94F7
:10609000AEF189E090E09093241B8093231B009342
:1060A000171B3DC00196A11DB11D05E0B695A79532
:1060B000979587950A95D1F70197A109B10900979E
:1060C00031E0A307B10550F0B093241BA093231B2C
:1060D0009093261B8093251B87E005C09093241B7B
:1060E0008093231B85E08093171B12E810931A1BE3
:1060F0008AE890E1A0E0B0E080931B1B90931C1B0A
:10610000A0931D1BB0931E1B0E94AEF188E090E08F
:106110009093241B8093231B85E08093171B10937F
:106120001A1B8CE890E1A0E0B0E080931B1B9093D9
:106130001C1BA0931D1BB0931E1B0E94AEF18091EF
:10614000090290910A02A0910B02B0910C02BA2FA1
:10615000A92F982F88270097E1E0AE07B10550F0EE
:10616000B093241BA093231B9093261B8093251B85
:1061700087E005C09093241B8093231B85E08093C8
:10618000171B82E880931A1B81EA90E0A0E0B0E040
:1061900012C28CEA95E00E94EE4F0E94F3BD40913E
:1061A000CB1A5091CC1A6091CD1A7091CE1A8823D7
:1061B00039F0433DF0E25F076105710509F465C3FD
:1061C000423D50426105710509F0D4C08091D31A57
:1061D0009091D41A019709F0AFC40E94F3BD8823AF
:1061E00009F4AAC480916F0D87FDC4C0A2E18A02A0
:1061F000C0011124865D904F0E94CE57C12C90E2C1
:10620000D92EE12CF12C05E012E81092241B1092FB
:10621000231B0093171B10931A1BC0921B1BD092B9
:106220001C1BE0921D1BF0921E1B0E94AEF1BFEFE3
:10623000CB1ADB0AEB0AFB0AEAE0CE16E0E2DE0646
:10624000E104F10411F700916F0DF2E10F028001FA
:1062500011240E53124FF80101900020E9F7C801F4
:106260008E1B9F0B439697FD01967C01F594E79456
:106270001E141F040CF05AC49E012F5F3F4F69018A
:1062800084E1D9011D928A95E9F7A7016DEB75E0CC
:10629000C9010F94CB17B801C6018E0D9F1D0F9435
:1062A000B61740E050E260E070E0C6010E945DF188
:1062B00062E070E080E090E00E94A5BF40E060E016
:1062C00070E08FE793E40E94AADF41E060E070E0B5
:1062D0008FE793E40E94AADF109208028DE090E01D
:1062E0009093241B8093231B85E08093171B12E857
:1062F00010931A1B84E190E1A0E0B0E080931B1B97
:1063000090931C1BA0931D1BB0931E1B0E94AEF10B
:1063100062E070E080E090E00E94A5BF81E09AE535
:106320009093241B8093231B85E390E09093261B7E
:106330008093251B87E08093171B10931A1B84E81A
:1063400090E0A0E0B0E080931B1B90931C1BA093F7
:106350001D1BB0931E1B0E94AEF181E080930002D2
:106360008093D50783E08093D60704C08CE495E042
:106370000E94EE4F80E5E7ECFAE1DF011D928A957D
:10638000E9F78AE58093C81A85EA8093C91A0C94C4
:10639000A31D8DE799E10E94DC55F701E959F44E00
:1063A00080838091671B8A3581F01E141F0414F0CE
:1063B0000C94C41ED601E02F1D92EA95E9F71092C5
:1063C000E0071092DF070C94C41E62E070E080E0EA
:1063D00090E00E94A5BFFFEFEF1AFF0AF092E007DE
:1063E000E092DF070C94C41E80E296E002C08FE0CA
:1063F00096E090938A088093890807CB88E290E022
:106400000E94F2F360917C1970917D19072E000CA7
:10641000880B990B0F945B0D2DEC3CEC4CEC5DE381
:106420000F9458140E948ABE60917C1970917D1956
:10643000072E000C880B990B0F945B0D20E030E0C9
:1064400048EC52E40F94BA0D0F94C4157093241BBA
:106450006093231B85E08093171B82E880931A1BAF
:1064600086E290E1A0E0B0E080931B1B90931C1BA0
:10647000A0931D1BB0931E1B0E94AEF160917C196E
:1064800070917D19072E000C880B990B0F945B0DF2
:106490008E010B5E1F4F23E041E00F942C089F9369
:1064A0008F9381E096E09F938F93045111091F937E
:1064B0000F930F94EC0CC8010E947FC08CEF95E005
:1064C00062C088ED9FEF0E94F2F360917C19709199
:1064D0007D19072E000C880B990B0F945B0D2DEC8A
:1064E0003CEC4CEC5DE30F9457140E948ABE609123
:1064F0007C1970917D19072E000C880B990B0F9455
:106500005B0D20E030E048EC52E40F94BA0D0F949C
:10651000C4157093241B6093231B85E08093171B85
:1065200082E880931A1B86E290E1A0E0B0E08093BD
:106530001B1B90931C1BA0931D1BB0931E1B0E9442
:10654000AEF160917C1970917D19072E000C880BBB
:10655000990B0F945B0D8E010B5E1F4F23E041E002
:106560000F942C089F938F938EEE95E09F938F93BB
:10657000045111091F930F930F94EC0CC8010E9452
:106580007FC089EE95E090938A08809389080F90E8
:106590000F900F900F900F900F9066CA9093261B4C
:1065A0008093251B87E08093171B10931A1B84E8A8
:1065B00090E0A0E0B0E080931B1B90931C1BA09385
:1065C0001D1BB0931E1B0E94AEF1D4CE24303105AA
:1065D00089F481E00F94F7042091E6073091E707F2
:1065E0004091E8075091E9070F94581441E00F9447
:1065F000CB04B2C02530310508F4F3C02630310594
:1066000009F430C108F022C181E08093EA0740E03C
:1066100060E070E08EE393E40E94FFBD20E030E094
:1066200048EC52E460913A0870913B0880913C0834
:1066300090913D080F94BA0D6B017C0160913E086A
:1066400070913F08072E000C880B990B0F945B0D7F
:106650009B01AC01C701B6010F9452150F94CB15E5
:106660006436710510F064E670E07093241B60934B
:10667000231B05E00093171B12E810931A1B84E2FA
:1066800090E1A0E0B0E080931B1B90931C1BA093B3
:106690001D1BB0931E1B0E94AEF160913A087091D1
:1066A0003B0880913C0890913D080F94C41570936D
:1066B000241B6093231B0093171B10931A1B86E364
:1066C00090E1A0E0B0E080931B1B90931C1BA09373
:1066D0001D1BB0931E1B0E94AEF180913E0890914D
:1066E0003F089093241B8093231B0093171B109348
:1066F0001A1B84E390E1A0E0B0E080931B1B909311
:106700001C1BA0931D1BB0931E1B0E94AEF165E0E5
:1067100070E080E090E00E94A5BF81E09AE5909350
:10672000241B8093231B84E490E09093261B80938A
:10673000251B87E08093171B10931A1B84E890E0B9
:10674000A0E0B0E080931B1B90931C1BA0931D1B2B
:10675000B0931E1B0E94AEF120E030E040E251E415
:106760006091E2077091E3078091E4079091E5075B
:106770000F94BA0D0F94C4157093241B6093231BC0
:1067800005E00093171B12E810931A1B84E590E1B3
:10679000A0E0B0E080931B1B90931C1BA0931D1BDB
:1067A000B0931E1B0E94AEF120E030E040E251E4C5
:1067B0006091E6077091E7078091E8079091E907FB
:1067C0000F94BA0D0F94C4157093241B6093231B70
:1067D0000093171B10931A1B88E590E1A0E0B0E02E
:1067E000EACE2230310579F480E00F94F70420914D
:1067F000E2073091E3074091E4075091E5070F94D9
:10680000581440E0F4CE2330310570F081E00F944D
:10681000F7042091E6073091E7074091E80750918F
:10682000E9070F945714E2CE2130310509F094CFD7
:1068300080E00F94F7042091E2073091E307409144
:10684000E4075091E5070F945714DBCF213F310542
:1068500009F082CF1092EA0761E070E080E090E0FA
:106860000E94A5BF81E09AE59093241B8093231B8F
:1068700081E490E09093261B8093251B87E0809312
:10688000171B82E880931A1B59CF8AE096E00E947A
:10689000EE4F8091700D9091710D99272091D31A30
:1068A0003091D41A8217930708F464CD85EB95E0F4
:1068B0000E94EE4F8091D31A815080936F0DA4ED0A
:1068C0008A2EA0E29A2EA12CB12C05E012E810929B
:1068D000241B1092231B0093171B10931A1B8092EA
:1068E0001B1B90921C1BA0921D1BB0921E1B0E9492
:1068F000AEF12FEF821A920AA20AB20A3EED831677
:1069000030E29306A104B10411F780916F0DA2E16A
:106910008A02C0011124FC01EE53F24F7F01019065
:106920000020E9F7C7018E1B9F0B439697FD019648
:106930008C011595079510161106FCF49E012F5F2A
:106940003F4F690184E1D9011D928A95E9F7A801B9
:106950006DEB75E0C9010F94CB17B701C601800F2D
:10696000911F0F94B61744ED50E260E070E0C6014D
:106970000E945DF105E012E806C044ED50E260E0DF
:1069800070E0C701F5CF1092241B1092231B0093D7
:10699000171B10931A1B80921B1B90921C1BA0921A
:1069A0001D1BB0921E1B0E94AEF1BFEF8B1A9B0AFB
:1069B000AB0ABB0AE6EE8E16E0E29E06A104B10425
:1069C00011F78E010F5F1F4F84E1D8011D928A9548
:1069D000E9F78091710D8F938091700D8F93809165
:1069E000D41A8F938091D31A8F9387EC95E09F935D
:1069F0008F931F930F930F94E5174EED50E260E0D5
:106A000070E0C8010E945DF162E070E080E090E01B
:106A10000E94A5BF0FB6F894DEBF0FBECDBF31E216
:106A2000C32E32E1D32EE12CF12C43E1442E40E67B
:106A3000542E612C712C88248394912CAA24AA941E
:106A4000BA2C75E0272EE2E83E2E0AE010E0809195
:106A5000700D9091710D8815990594F1B092241BD9
:106A6000A092231B2092171B30921A1B40921B1BD3
:106A700050921C1B60921D1B70921E1B0E94AEF157
:106A80001093241B0093231B2092171B30921A1B78
:106A9000C0921B1BD0921C1BE0921D1BF0921E1B70
:106AA0000E94AEF1FFEF8F1A9F0A20E1420E511CA7
:106AB000611C711C3FEFC31AD30AE30AF30AC7CF64
:106AC0008091D31A9091D41A24E0880F991F2A95A7
:106AD000E1F78D5F9F49A0E0B0E020EF37E8309309
:106AE000241B2093231B05E00093171B12E810932F
:106AF0001A1B80931B1B90931C1BA0931D1BB09310
:106B00001E1B0E94AEF18091D31A9091D41A805E20
:106B10009D4EA0E0B0E026E030E03093241B2093AF
:106B2000231B0093171B10931A1B45CD40E050E226
:106B300060E070E0C801BACB8091D31A9091D41A6A
:106B4000892B11F40C94B02715CCE3960FB6F8946A
:106B5000DEBF0FBECDBFDF91CF911F910F91FF9090
:106B6000EF90DF90CF90BF90AF909F908F907F90ED
:106B70006F905F904F903F902F9008952F923F928B
:106B80004F925F926F927F928F929F92AF92BF923D
:106B9000CF92DF92EF92FF920F931F93CF93DF93E9
:106BA000CDB7DEB7C154D1090FB6F894DEBF0FBE22
:106BB000CDBF22968FAF229720910A082CAF21E0FB
:106BC00020930A08809131178D3409F40FC584355C
:106BD00011F40C941A48873411F00C942B488091CE
:106BE0002F17909130178A31910509F421C2B4F41E
:106BF0008430910534F482309105DCF597FF2DC087
:106C0000F1C48C30910509F40FC28531910511F45E
:106C10000C942D48049709F0E5C4C7C18A32910548
:106C200009F465C454F48C31910509F42AC20CF4BA
:106C300003C24D9709F435C2D5C48B35910509F4CB
:106C4000D6C38C35910509F4D6C38A35910509F070
:106C5000C9C4109209080C942D48809140028823E1
:106C600011F40C942D480E9448B50E94A1E00C94A8
:106C70002D4820914002222311F40C942D4811E05C
:106C8000029709F010E00E9448B519821A821B820F
:106C90001C821D821E821F82188682E50E948ACC79
:106CA000882309F43AC10E940ACC4B015C0120E020
:106CB00030E0A9010F94540D882309F444C1409198
:106CC000F80A5091F90A6091FA0A7091FB0A4CA3F4
:106CD0005DA36EA37FA36091FC0A7091FD0A809171
:106CE000FE0A9091FF0A68A779A78AA79BA78091BF
:106CF000960A9091970AA091980AB091990A8CA748
:106D00009DA7AEA7BFA720919A0A30919B0A4091F8
:106D10009C0A50919D0A28AB39AB4AAB5BAB9C01F6
:106D2000AD016CA17DA18EA19FA10F94540D811185
:106D30000DC028A939A94AA95BA968A579A58AA582
:106D40009BA50F94540D882309F4FDC020E030E08A
:106D5000A901C501B4010F94540D881F8827881F0D
:106D6000181749F040E050E060E87FEB48AF59AFBA
:106D70006AAF7BAF08C060E070E080E89FE368AF77
:106D800079AF8AAF9BAF2CA13DA14EA15FA16CA5AD
:106D90007DA58EA59FA50F9457146CAB7DAB8EABD4
:106DA0009FAB28A539A54AA55BA568A979A98AA999
:106DB0009BA90F9457146B017C012CA93DA94EA9E6
:106DC0005FA9CA01B9010F94BA0D2B013C01A701BB
:106DD0009601C701B6010F94BA0D9B01AC01C30126
:106DE000B2010F9458140F9406172B013C019B011C
:106DF000AC0160E070E080E89FE30F9452152196AB
:106E00006CAF7DAF8EAF9FAF219720E030E040E0C8
:106E10005FE3C301B2010F94BA0D2B013C01A50140
:106E20009401C501B4010F94BA0D4B015C01A3019B
:106E30009201C301B2010F94BA0D9B01AC01C501CF
:106E4000B4010F9457140F94061728AD39AD4AAD0D
:106E50005BAD0F94BA0D4B015C01C701B6019058B0
:106E600021962CAD3DAD4EAD5FAD21970F94BA0D7F
:106E7000A50194010F94BA0D6B017C012CA53DA5D1
:106E80004EA55FA56CA17DA18EA19FA10F94581462
:106E900020E030E040E05FE30F94BA0D9B01AC01CD
:106EA000C701B6010F9458142CA13DA14EA15FA1BA
:106EB0000F94571469837A838B839C8328A939A9FB
:106EC0004AA95BA968A579A58AA59BA50F94581422
:106ED00020E030E040E05FE30F94BA0D6B017C01ED
:106EE00021962CAD3DAD4EAD5FAD21976CA97DA92E
:106EF0008EA99FA90F94BA0DA50194010F94BA0D04
:106F00009B01AC01C701B6010F94581428A539A5FF
:106F10004AA55BA50F94571412C089E40E948ACC3D
:106F2000882331F00E940ACC69837A838B839C8307
:106F30008AE40E948ACC882331F00E940ACC6D83B7
:106F40007E838F83988720E030E0A90169817A8170
:106F50008B819C810F94540D81110BC020E030E097
:106F6000A9016D817E818F8198850F94540D8823AE
:106F7000A1F0412FBE016F5F7F4F86E99AE00E942A
:106F80003C950E94336860937419709375198093CF
:106F90007619909377190C942D480E94B84D80EE85
:106FA00096E00E941F4D0C942D4880E50E948ACCEB
:106FB000882329F00E944CA96B017C0103C0C12CDD
:106FC000D12C760183E50E948ACC882361F00E944F
:106FD0000ACC20E030E04AE754E40F94BA0D0F9455
:106FE000CB156B017C010E9469D38091A70A8111A6
:106FF00005C060E086EF96E00E9404DF0E943368DF
:10700000C60ED71EE81EF91E0E943368DC01CB01B4
:107010008C199D09AE09BF09B7FD02C00C942D481B
:1070200080E00E94AA50F0CF0E9428B80C942D480E
:107030000E9436AC0C942D480E94626381110C941E
:107040002D4880E090E0A8E4B2E489839A83AB8382
:10705000BC8380E090E0A0E2B1E48D839E83AF83A7
:10706000B88789879A87AB87BC8760E070E080E546
:107070000E9415B8BE016F5F7F4F0E943CDE0C94EA
:107080002D488091A60A8770873011F00C943848FB
:1070900060E08FE40E9497CC81110C942D480C94F1
:1070A000384860E083E50E947FAA182F863030F0D0
:1070B0008CEC97E00E941F4D0C942D48833009F40E
:1070C0000EC128F4813039F1823099F106C0843044
:1070D00009F45BC1853009F468C189EB97E00E942F
:1070E0001F4D0E94414C882389F08091100B88230A
:1070F00019F080E297E002C08CE197E00E941F4DFA
:107100008AE00E940D4D0E943D4F55C18BEA97E0E9
:107110000E941F4D50C10E94FF4B1092020210921C
:10712000010280EA97E090938A08809389080C9482
:107130002D48809101029091020297FF06C087E7D7
:1071400097E00E941F4D0C942D480097A1F4809168
:107150006B028093110819821A821B821C821C8E7A
:107160001D8E1E8E1F8EBE016F5F7F4FCE014C960F
:107170000E949CE427C0815065E00F940D1480FFAD
:1071800003C024E0291B922F25E09202F001112474
:10719000E80FF11D87FDFA95EE0FFF1FEE0FFF1FA1
:1071A000E253F74E8091000B9091010BA091020BDE
:1071B000B091030B80839183A283B38380911108E4
:1071C00080936B02809101029091020289319105B6
:1071D0000CF063C010926B029C012F5F3F4F309305
:1071E00002022093010265E00F940D1480FF03C09A
:1071F00024E0291B922F19821A821B821C8244E0F0
:10720000840290011124B9016A57744E4B01DB01CD
:107210002D913D914D915C91B4E09B02C0011124F0
:10722000FC01E656F44E5F01608171818281938199
:10723000DE0111966D01E12CF12C00EA10E40E94B0
:10724000BDE319821A821B821C828DEC9CECACE49B
:10725000BEE38C8F9D8FAE8FBF8FB601CE014C9653
:107260000E949CE4F50180819181A281B381809389
:10727000F80A9093F90AA093FA0AB093FB0AF40172
:1072800080819181A281B3818093FC0A9093FD0A51
:10729000A093FE0AB093FF0A90C080E090E0A0EABD
:1072A000B0E48093000B9093010BA093020BB0937A
:1072B000030B89E592E00E949EE30E9469D38FEF61
:1072C0009FEF909302028093010283E697E00E9471
:1072D0001F4D0E94076681E00E94224C6EC089E427
:1072E0000E948ACC8823B1F00E9406CC182F8530EA
:1072F00060F064E070E080E597E00E94BB4E8DE4B2
:1073000097E00E941F4D0C942D488AE40E948ACC7D
:10731000811105C08AE40F94C5040C942D480E9485
:1073200006CC082F853060F064E070E08AE397E0D7
:107330000E94BB4E87E397E00E941F4D0C942D489E
:107340008AE50E948ACC8823D9F00E940ACC9B014E
:10735000AC0165E01602F0011124E00FF11D07FDFC
:10736000FA95EE0FFF1FEE0FFF1FE253F74E20833B
:10737000318342835383602F812F0E94C0BF33C06B
:107380008AE50F94C5040C942D488AE50E948ACCA6
:107390008823B1F30E940ACC6093CA187093CB186B
:1073A0008093CC189093CD181EC080E00E94224C90
:1073B0000E94FF4B18C01230B1F46091010270912D
:1073C00002026931710514F069E170E088E297E02A
:1073D0000E94BB4E69E170E083E297E00E94BB4EE1
:1073E0008AE00E940D4D0E94D9E40C942D48209310
:1073F00009080C942D485BED252E52E0352E6EEBDE
:10740000E62E68E1F62E88EF9AE09DA38CA372EB3E
:10741000C72E78E1D72E00E010E0D1018D911D013B
:107420000E948ACC882309F44BC00E940ACC2B010D
:107430003C01133049F0F6012081318142815381B2
:107440000F9457142B013C01ACA1BDA12D913D918E
:107450004D915C91C301B2010F9457144B015C0133
:107460002DEB37E346E855EB0F94B81687FD0AC0BD
:107470002DEB37E346E855E3C501B4010F94540DF5
:107480001816F4F4133051F44092040B5092050B8B
:107490006092060B7092070B01E012C0A5019401E7
:1074A000F70160817181828193810F945814D70113
:1074B0006D937D938D939C931397812F0E94ACD8ED
:1074C0001F5FB4E0EB0EF11CECA1FDA13496FDA30F
:1074D000ECA3F4E0CF0ED11C143009F09ECF0023B2
:1074E00009F481CF84E09BE00E947AD37CCF809125
:1074F0004002882311F40C942D4889E40E948ACC20
:10750000E82E882321F00E9406CC082F01C000E05D
:107510008AE40E948ACCF82E882321F00E9406CCAF
:10752000182F01C010E0EE2011F0053020F4FF20EC
:1075300041F0153030F083EE97E00E941F4D0C941F
:107540002D480E94B4CAEE2091F024E00202F0011E
:107550001124E656F44E80819181A281B3818093FB
:10756000960A9093970AA093980AB093990AFF20DD
:1075700091F034E01302F0011124EA57F44E8081B7
:107580009181A281B38180939A0A90939B0AA093E0
:107590009C0AB0939D0A60E080E50E9497CC40E091
:1075A00050E0BA0186E40E948DC16B017C0120E0AD
:1075B00030E0A9010F94B816181684F420E030E0EA
:1075C00040E752E4C701B6010F9452156093590287
:1075D00070935A0280935B0290935C020E94A1E038
:1075E0000C942D480E9454630C942D4880912F17C1
:1075F000909130178337910509F4ABC70CF0D4C0D4
:107600008934910509F477C40CF05CC08931910587
:1076100009F4F8C21CF58431910509F46FC27CF4B9
:107620008131910509F456C22CF4029708F4CBC1BC
:107630000C941748429709F4BCC60C94174886313D
:10764000910509F485C20CF47FC28731910509F4D4
:1076500088C2489709F49DC20C9417488E31910551
:1076600009F45DC3ACF48B31910509F4E4C20CF468
:10767000D4C28C31910509F448C34D9711F00C9494
:1076800017488091C71C8E7F8093C71C0C942D488F
:107690008132910509F4D8C34CF48F31910509F476
:1076A000E7C3809709F49AC30C9417488A3291056E
:1076B00009F4FEC38B9711F00C9417480E946CBC20
:1076C0000C942D488836910509F4BEC4D4F5813553
:1076D000910509F45CC6C4F48C34910509F41AC40C
:1076E0004CF48B34910511F00C9417480E9465718D
:1076F0000C942D488D34910509F410C48E349105F5
:1077000009F410C40C9417488435910509F451C646
:1077100074F48235910509F449C68335910511F059
:107720000C94174881E0809304080C942D4885350B
:10773000910509F46BC68C35910509F480C60C944B
:1077400017488D36910509F4B6C48CF48A36910534
:1077500009F4EDC50CF4B1C58B36910509F40DC6DD
:107760008C36910511F40C942D480C9417488037F1
:10777000910511F40C942D4854F48E36910509F4BA
:1077800000C58F36910509F40DC50C941748813753
:10779000910509F44CC58237910511F00C941748F6
:1077A0000E9432FA0C942D48823241E0940711F481
:1077B0000C9421450CF07BC0883C910509F47FC7EF
:1077C000D4F58937910509F473C7ECF48637910530
:1077D00009F439C734F48537910509F423C70C94AB
:1077E00017488737910509F460C78837910511F06C
:1077F0000C94174881E080937908809378080E9460
:1078000006E60C942D488C38910509F432C54CF4E9
:107810008D37910511F00C9417480E9447B70C94CE
:107820002D488B39910509F45CC58E3B910509F40F
:1078300032C50C9417488E3C910511F40C944C44BD
:10784000B4F48B3C910509F4C7C734F4893C910525
:1078500009F49EC70C9417488C3C910509F4DDC7C8
:107860008D3C910511F40C943E440C9417488C3DCA
:10787000910511F40C94724474F4833D910511F454
:107880000C946F44893D910511F00C9417480E94A7
:1078900076A80C942D488D3D910511F40C947F44ED
:1078A000823E910511F40C94D5440C941748853F01
:1078B00061E0960711F40C94FD460CF047C0803946
:1078C000A1E09A0711F40C946646DCF48E32E1E0F4
:1078D0009E0711F40C941F463CF48D32914011F434
:1078E0000C942C450C9417488F3231E0930711F417
:1078F0000C9463468033914011F40C94AC450C9485
:107900001748853A51E0950711F40C9469467CF4C8
:107910008A3971E0970711F40C942D48843A91400C
:1079200011F00C9417480E948BAA0C942D488C3AA5
:10793000B1E09B0711F40C946C46843F914011F028
:107940000C9417480E94CCD80C942D488835F2E04E
:107950009F0711F40C942347B4F4873F31E0930759
:1079600011F40C94034714F40C940047883F51E041
:10797000950711F40C940A478C30924011F40C9442
:107980001B470C941748843873E0970711F40C9444
:10799000A1476CF48B35B2E09B0711F40C94264799
:1079A0008C36934011F40C942D480C941748803A6F
:1079B000F3E09F0709F44CC2873E934011F40C9406
:1079C00009480C94174800919C1810919D1880E567
:1079D0000E948ACC882361F00E944CA96B017C0133
:1079E000BB24B394672B682B692B31F4B12C04C0F2
:1079F000B12CC12CD12C760183E50E948ACC88233E
:107A000011F40C94074A0E940ACC20E030E04AE7C7
:107A100054E40F94BA0D0F94CB156B017C01B11097
:107A20000BC0672B682B692B39F40115110521F068
:107A3000D8018C91811102C0B12C02C0BB24B39437
:107A40000E9469D3B11003C089E196E001C0C8016A
:107A50000E94C4C010910A0883E080930A0881E064
:107A60008093431944E158E06DE178E082E00E94A0
:107A70008A4D82E098E00E94C4C0C114D104E104A0
:107A8000F104B1F00E943368C60ED71EE81EF91E3D
:107A90000E943368DC01CB018C199D09AE09BF0936
:107AA000B7FF0EC08091431981110C940C4A08C095
:107AB00080914319882321F080E00E94AA50F8CFDA
:107AC00080E090E00E94C4C01092431910930A080D
:107AD0000C942D4880912B1784FF02C00C94114AFE
:107AE00080912D1787FF02C00C94114A80912E17A8
:107AF000837011F00C94114A0C942E4A87E498E09C
:107B00000E941F4D10927D0A83E79AE10E94419BDB
:107B10008BE1E3E7FAE1DE01119601900D928A957F
:107B2000E1F740E050E0BE016F5F7F4F80E090E002
:107B30000E943B59CE0101960E94779C88E398E011
:107B40000E941F4D0C942D480E9426580C942D48DD
:107B50000E94B5578091C71C877F8093C71C0C94E7
:107B60002D48E0919C18F0919D188081882329F080
:107B7000803209F410823196F8CF40E061E08091C4
:107B80009C1890919D180E94115B109244190C94BE
:107B90002D4880910F0A8823E9F080E090E0A0EA68
:107BA000B1E488A399A3AAA3BBA31C8E1D8E1E8E2D
:107BB0001F8E19821A821B821C8220E0AE01405E59
:107BC0005F4FBE01645E7F4FCE0101960E9491CD52
:107BD0000C942D480E94D6C8882321F00E94C657D5
:107BE0000E94657140E050E068E578E085E00E9421
:107BF0008ACD61E089EE9BE20E942E4D0E9488DFD3
:107C00000C942D488091C71C82FF03C08B7F80930A
:107C1000C71C0E9447B70C942D488091C71C83FD58
:107C200002C00C942D4883E50E948ACC81110C94EB
:107C30003D4A0C942D4883E40E9441CC8823D9F11D
:107C40008CE698E00E941F4D80911D1A882351F107
:107C5000BE016F5F7F4F8AE19AE10E94089A8E0110
:107C60000F5F1F4FF80181918F01882319F00E9447
:107C70000D4DF8CFBE016F5F7F4F80E090E00E9416
:107C8000D95A8091200D882389F080E20E940D4D01
:107C900000E21DE0D8018D918D01882339F00E940A
:107CA0000D4DF8CF82E698E00E941F4D8AE00E94B9
:107CB0000D4D0C942D4883E50E948ACC882309F150
:107CC0000E94E2CB182F90E0CD970CF01CE31093AC
:107CD000FB070E9433686B017C01212F30E0A8EE86
:107CE000B3E00F94FE13C60ED71EE81EF91EC09215
:107CF000F707D092F807E092F907F092FA070C9490
:107D00002D480E948E570C942D4840E060E08091F1
:107D10009C1890919D180E94115B0C942D488091A5
:107D2000C71C83FD02C00C942D480E943A638091C9
:107D3000C71C83FD02C00C942D4860919C18709163
:107D40009D18CE014C960E940AF38C01009711F405
:107D50000C942D486C8D7D8D19821C8222E0AC0123
:107D6000CE0101960E945AA0811102C0F12C14C0CC
:107D7000CE0101960E9478F28823C1F361E0CE0122
:107D800001960E94EC99009789F325EEFC0120836F
:107D90001C820E94FB9BF82ECE0101960E94779CCC
:107DA000B801FF2089F086E998E00E94A54D8AE09D
:107DB0000E940D4D1092C31C1092C41C1092C51C41
:107DC0001092C61C0C942D488EE798E00E94A54D99
:107DD0008BE798E00E941F4D0C942D488091C71CA2
:107DE00082FD0E9469D38091C71C83FD02C00C9460
:107DF0002D4860E080E50E9497CC182F482F61E065
:107E000080919C1890919D180E94115B83E50E94BF
:107E10008ACC882381F00E94D2CBAB01BC01409375
:107E2000C31C5093C41C6093C51C7093C61C8AE18C
:107E30009AE10E9402990E94C65711110C942D4894
:107E40000E9465710C942D480E94F9C70C942D482E
:107E500020919C1830919D189091C71C926090932E
:107E6000C71C40E060E0C9010E94115B0C942D48E2
:107E70000E94B4DD6C8F7D8F8E8F9F8FBE016F5FF0
:107E80007F4FCE014C960E941DC760E0CE01019647
:107E90000E945FDF0E94BC4DBE016F5F7F4F84EA8E
:107EA00098E00E94A54D8AE00E940D4D0C942D484B
:107EB00083E50E948ACC882311F40C942D480E94FB
:107EC000E2CBF82E6DE070E080E50E94FFA78C0108
:107ED00097FF02C00C942D48E82E60E089E40E94D0
:107EE00097CC81110C944E4A802F0E94954C8111A1
:107EF00079C50C944E4A80E50E9441CC882311F448
:107F00000C942D488091C71C82FF02C00C942D4810
:107F10000C94674A0E9403DE0C942D480E94C9719C
:107F20000C942D4860E070E083E50E94FFA78E343A
:107F3000910531F40E943E720E9488DF0C942D4816
:107F40008FE099E00E941F4D609168087091690868
:107F500086E099E00E94924E60916A0870916B08E9
:107F600089EF98E00E94924E6091680870916908CC
:107F700080916A0890916B08681B790B80919F1023
:107F8000815021E030E0823010F020E030E0621BD0
:107F9000730B8EEE98E00E94924E8AE00E940D4D87
:107FA00086EE98E00E941F4D80916C0890916D08BC
:107FB000A0916E08B0916F088C8F9D8FAE8FBF8F90
:107FC000BE016F5F7F4FCE014C960E941DC7BE0160
:107FD0006F5F7F4F89ED98E00E94A54D80917008FA
:107FE00090917108A0917208B09173088C8F9D8F49
:107FF000AE8FBF8FBE016F5F7F4FCE014C960E9448
:108000001DC7BE016F5F7F4F89EC98E00E94A54DB0
:1080100020E030E04AE754E46091740870917508FC
:1080200080917608909177080F945215AB01BC01AE
:1080300081EB98E00E94D74F8DE60E940D4D8AE0BB
:108040000E940D4D0C942D488091E91683FF02C0CB
:108050000C942D480E94F7B5182F87FF02C00C948E
:108060002D4883E50E948ACC882311F10E940ACC16
:108070000F94C4157B01212F110F330BF901EE0F63
:10808000FF1FE052F94E718360834091F70A50E080
:108090002417350711F00C942D48CB010E944BA1F9
:1080A000F1E5EF16F10424F40E94C9710E9488DF03
:1080B0000F949504D2C78091E91683FDCEC70E9424
:1080C000F7B5082F87FDC9C783E50E948ACCF82E33
:1080D000811107C082E50E948ACC182F882309F4F9
:1080E00046C00E940ACC0F94C415402F002E000CED
:1080F000550BFA01EE0FFF1FE052F94E71836083BA
:108100002091F70A30E04217530709F0A6C7CB01C8
:108110000E944BA10E940ACC20E030E040EA52E4E9
:108120000F94540D181614F40C94724A0E94C971DD
:108130000E9488DF60913E0870913F08072E000C76
:10814000880B990B0F945B0D20913A0830913B08F6
:1081500040913C0850913D080F94B816181614F43D
:108160000C94764AFF2011F40C94764A11E00F9497
:108170009504112309F471C76F2D802F0E944B873E
:108180006CC78EE40E948ACC882309F466C70E94DB
:10819000D2CB6093B4177093B5178093B6179093B2
:1081A000B7175BC783E50E9441CC882331F060E0BC
:1081B00083E50E947FAA8093E9160E94BC4D85E268
:1081C00099E00E941F4D8091E916882369F19BE197
:1081D000E92E99E0F92E00E010E020E08091E91608
:1081E00090E0A0E0B0E0002E04C0B695A79597956A
:1081F00087950A94D2F780FF0EC0DD24D394D20E67
:10820000222319F08CE20E940D4DF7018591949183
:108210000E941F4D2D2D0F5F1F4F32E0E30EF11C0A
:1082200005301105D9F642CD87E199E03DCD83E5D2
:108230000E948ACC882371F00E94E2CB282F30E084
:108240002D3331051CF48093030207C78CE3809320
:10825000030203C70E94BC4D4091030250E060E05E
:1082600070E08CE299E00E94814E8AE00E940D4D00
:10827000F4C68091E91683FDF0C683E50E948ACC9E
:10828000882309F4EAC60E940ACC0F94C415CB01D6
:108290000E94A6CAE2C68091E91683FDDEC683E588
:1082A0000E948ACC182F81110C947B4A82E50E948F
:1082B0008ACC81110C947B4AD0C60E94F7B5182F46
:1082C00087FD0AC081E599E00E941F4D812F0E9421
:1082D0005A858AE00E940D4D4CAD40930A080C94DB
:1082E000E54B83E50E948ACC882309F4B6C60E9438
:1082F000E2CB182F90E0CD970CF01CE31093000810
:108300000E9433686B017C01212F30E0A8EEB3E0BE
:108310000F94FE13C60ED71EE81EF91EC092FC076E
:10832000D092FD07E092FE07F092FF0796C660919B
:10833000F70A80E50E947FAA182F823008F08DC6C8
:1083400081E40E9441CC882341F0E091F70AF0E0FB
:10835000EA51F94E608170E002C06FEF70E083E592
:108360000E9415B88F3F910519F010F08FEF90E043
:10837000BC01812F0E94A7F970C66091F70A80E5C1
:108380000E947FAA60E070E00E94A7F966C60E9482
:10839000378F0E94C9710E94FDD40E94C64C68EEBE
:1083A00073E080E090E00E946E4C57C61092040883
:1083B00054C683E50E948ACC882399F00E940ACC97
:1083C00020E030E04AE754E40F94BA0D0F94CB1547
:1083D0006093040270930502809306029093070253
:1083E0003CC680912B1784FF02C00C94B04A809148
:1083F0002D1787FF02C00C94B04A80912E1783700E
:1084000011F00C94B04A0E94FDD427C683E50E9467
:1084100041CC882309F421C60E940ACC20E030E038
:108420004AE754E40F94BA0D0F94CB1560930508F6
:108430007093060880930708909308080EC60E9460
:10844000F7B587FD0AC690912B1794FD04C0909153
:108450002D1797FF0AC00BEDC02E02E0D02E88E941
:10846000E82E86E1F82E10E009C090912E17937047
:1084700091F7682F81E00E9431BCEFC5D6018D9144
:108480006D010E948ACC882309F459C0133009F089
:108490004FC00E940ACC4B015C0120E030E040EA72
:1084A00051E40F94540D87FF3AC0A50194016091E7
:1084B000B8167091B9168091BA169091BB160F94A8
:1084C00052152B013C019B01AC016091C8167091C3
:1084D000C9168091CA169091CB160F94BA0D60936D
:1084E000C8167093C9168093CA169093CB166091E4
:1084F0004716709148168091491690914A160F942C
:10850000590DA30192010F94BA0D0F94CB156093EE
:108510004716709348168093491690934A16809296
:10852000B8169092B916A092BA16B092BB1607C0B0
:108530000E940ACCF701648B758B868B978B1F5F2B
:10854000F4E0EF0EF11C143009F098CF0E94E7849C
:1085500084C588E79AE00E941F4D60E088E69AE0B3
:108560000E9418FA60E083E59AE00E9418FA61E040
:108570008CE49AE00E9418FA61E081E49AE00E949B
:1085800018FA61E081E39AE00E9418FA60E088E25C
:108590009AE00E9418FA61E08EE19AE00E9418FACF
:1085A00060E084E19AE00E9418FA60E08CE09AE0D2
:1085B0000E9418FA61E08EEF99E00E9418FA61E0DB
:1085C00080EF99E00E9418FA60E081EE99E00E9445
:1085D00018FA60E083ED99E00E9418FA60E08DEBF4
:1085E00099E00E9418FA61E08CEA99E00E9418FA7A
:1085F00061E08DE999E00E9418FA61E088E899E06D
:108600000E9418FA61E085E799E00E9418FA60E09C
:1086100088E699E00E9418FA60E084E599E00E94FB
:1086200018FA1BC580919C1890919D18009741F0F5
:10863000DC012C91222321F060E00E945FDF0DC558
:108640000E9488DF0AC500919C1810919D1883E054
:10865000F12C40E08150E1F0F8019081292F2B7F2F
:108660002134C1F721812133A9F7913421F09534C8
:1086700021F441E002C0FF24F39498012E5F3F4FA4
:1086800089012F5F3F4FD8019C919032C9F3E2CF0F
:1086900041110E94BC4DFF2021F080E69BE00E942A
:1086A0001F4DC8010E94EE4FD8C40E94EAE5D5C410
:1086B00010927908109278080E9406E6CEC40E94B3
:1086C000F7B5182F87FDC9C484E40E9441CC8823E4
:1086D00009F45BC00E940ACC6B017C0101E020E040
:1086E00030E0A9010F94540D811101C000E0009306
:1086F000321920E030E0A901C701B6010F94540DF2
:10870000882309F442C00E940ACCB4E01B02F001A5
:108710001124E55CF64E608371838283938320E0AD
:1087200030E0A90160913B1970913C1980913D198D
:1087300090913E190F94540D81110CC080E090E08F
:10874000A0EEBFE380933B1990933C19A0933D1991
:10875000B0933E1920E030E0A90160913F1970917B
:10876000401980914119909142190F94540D811133
:108770000CC080E090E0A0EEBFE380933F1990939F
:108780004019A0934119B09342190E9454D665C470
:108790000E94F7B587FD61C41BEDE12E12E0F12EBA
:1087A00008E916E1F70181917F010E9441CC8823FD
:1087B00051F00E940ACC0F94CB15D8016D937D9394
:1087C0008D939C9313970C5F1F4FB6E1083A1B07DC
:1087D00049F70E94F2D241C40E94F7B587FD3DC41B
:1087E000BBEDEB2EB2E0FB2E08E916E1F70181911B
:1087F0007F010E9441CC882349F00E940ACCD80115
:1088000094966D937D938D939C9397970C5F1F4FD8
:10881000B6E1083A1B0751F720C480912C1787FD59
:10882000D0C680912D178E7009F0CBC64091CC1622
:108830005091CD166091CE167091CF168AE69BE0CE
:108840000E94D74F4091D0165091D1166091D21608
:108850007091D31687E69BE00E94D74F4091D416C3
:108860005091D5166091D6167091D71684E69BE08C
:108870000E94D74F8AE00E940D4DEFC380912B17C5
:1088800081FDE5C680912C1781FDE1C680912D17F1
:108890008C7009F0DCC6E1C3FBEDCF2EF2E0DF2ED9
:1088A000ACE7EA2EA8E0FA2E10E0F60181916F0104
:1088B0000E9441CC882359F00E940ACCD7016D93C5
:1088C0007D938D939C931397812F0E94ACD81F5F4B
:1088D000B4E0EB0EF11C133041F70C94F3390E9415
:1088E0007CBBBBC383E50E948ACC882309F4B5C353
:1088F0000E9406CC90936D0280936C02AEC30E94DE
:10890000F7B5F82E87FDA9C383E50E948ACC0F2D09
:108910000F2C000C110B882369F10E9406CCF80182
:10892000EE0FFF1FE959FD4F91838083000F111F48
:10893000000F111FF801EF5CFD4F7F01BC01990F83
:10894000880B990B0F945B0D2AE037ED43E25CE353
:108950000F94BA0DF801ED5CF64E20813181428111
:1089600053810F94BA0DD7016D937D938D939C9392
:10897000139773C30E94BC4D85E40E940D4D80E3A4
:108980008F0D0E940D4DF801EE0FFF1FE959FD4FAD
:108990006081718189E99BE00E94BB4E85E20E9463
:1089A0000D4D8AE00E940D4D58C380E50E9441CCD8
:1089B000882309F452C360E070E080E50E94FFA7BD
:1089C000F82E6FEF7FEF83E50E94FFA78C010196E1
:1089D000039708F042C3F7FC40C38F2D0E94954CCB
:1089E000882339F00E94B84D81EA9BE00E941F4D18
:1089F00034C30E9469D360E08F2D0E94D5660F3F7B
:108A0000BFEF1B0731F00130110571F000E010E0FD
:108A10000DC08F2D0E947D6631E020E0892B09F08A
:108A200030E0032F122F02C001E010E08F2D0E94D2
:108A30007D668017910709F410C380E00E94AA5058
:108A4000F5CF8AE50E948ACC811184C683E50E9415
:108A50008ACC81117FC601C360E085E40E947FAAB1
:108A6000811173C080E50E9441CC882351F00E949F
:108A70000ACC609341087093420880934308909316
:108A8000440889E40E9441CC882381F00E940ACCEA
:108A90002CEA35EC47E25EE30F94BA0D609345088B
:108AA00070934608809347089093480884E40E9496
:108AB00041CC882381F00E940ACC2CEA35EC47E2B5
:108AC0005EE30F9452156093490870934A088093AF
:108AD0004B0890934C080E94BC4D40914108509126
:108AE000420860914308709144088AEC9BE00E9420
:108AF000D74F2CEA35EC47E25EE360914508709170
:108B0000460880914708909148080F945215AB0190
:108B1000BC0186EC9BE00E94D74F2CEA35EC47E283
:108B20005EE36091490870914A0880914B089091EA
:108B30004C080F94BA0DAB01BC0182EC9BE00E9483
:108B4000D74F8AE00E940D4D88C20E94B84D80EB3D
:108B50009BE00E941F4D81C280E50E9441CC88238A
:108B600051F00E940ACC6093580870935908809382
:108B70005A0890935B0889E40E9441CC882381F0D5
:108B80000E940ACC2CEA35EC47E25EE30F94BA0D62
:108B900060935C0870935D0880935E0890935F0813
:108BA00084E40E9441CC882381F00E940ACC2CEA04
:108BB00035EC47E25EE30F945215609360087093C2
:108BC000610880936208909363080E94BC4D4091B5
:108BD00058085091590860915A0870915B0886EDC9
:108BE0009BE00E94D74F2CEA35EC47E25EE36091B0
:108BF0005C0870915D0880915E0890915F080F9409
:108C00005215AB01BC0182ED9BE00E94D74F2CEACC
:108C100035EC47E25EE360916008709161088091F5
:108C20006208909163080F94BA0DAB01BC018EEC01
:108C30009BE00E94D74F8AE00E940D4D0EC283E553
:108C40000E9441CC182F882371F00E940ACC0F9407
:108C5000C41570935E0260935D0221E0672B09F0FA
:108C600020E02093E81680E50E9441CC882359F04B
:108C700020915D0230915E02232B11F00E94F6CB11
:108C80008093E816EAC11111E8C10E94BC4D86EF3D
:108C90009BE00E941F4D8091E816882319F08EED0D
:108CA0009BE002C08AED9BE00E941F4D60915D0237
:108CB00070915E0285EE9BE00E94BB4E81EE9BE0D0
:108CC0000E941F4DCAC10E94A4C1C7C10E9469D39E
:108CD000C4C10E949BA9C1C10E9462638111BDC130
:108CE00009E41BE2E8EFFAE0FDA3ECA39E012F5F8D
:108CF0003F4F59015EE9852E5BE2952E1901F8017F
:108D00006591759185919491ACA1BDA1CD90DD90B7
:108D1000ED90FD90BDA3ACA3A70196010F9457144D
:108D20002B013C01F101608371838283938320E0F6
:108D300030E040EA51EC0F94B81687FD0AC020E0FD
:108D400030E040EA51E4C301B2010F94540D18160B
:108D50002CF4F401849118160CF42CC5D101CD909B
:108D6000DD90ED90FD901D0120E030E040EA51ECF7
:108D7000C701B6010F94B81687FD0AC020E030E0A5
:108D800040EA51E4C701B6010F94540D181664F47B
:108D90000E94B84D87E29CE00E941F4D61E089E18E
:108DA0009CE00E9404DF59C10C5F1F4FBFEF8B1A7C
:108DB0009B0AEBE205351E0709F0A1CF4CE7E42E34
:108DC00048E0F42E10E0F50181919191A191B191CB
:108DD0005F01F70181939193A193B1937F01812F5B
:108DE0000E94ACD81F5F133071F70E94D9E460E095
:108DF00089E09CE00E9404DF30C10E94E2F02DC1B6
:108E00000E945BEC2AC161E083E50E9497CC0E943E
:108E1000CFED23C181E080935F190E9411E610928B
:108E20005F19882309F419C10E94BC4D85E49CE0B8
:108E30000E941F4D12C18091C71C82FF0EC180622B
:108E40008093C71C0AC10E9421B607C10E94F7B5D2
:108E5000082F87FD02C185E50E9441CC8823B1F12E
:108E6000A02E002E000CBB080E940ACC6B017C01D6
:108E700020E030E0A9010F94B81687FF04C0F7FA8C
:108E8000F094F7F8F094C50133E0880F991F3A95F4
:108E9000E1F79C012C59364E5901D901CD92DD9252
:108EA000ED92FC92139720E030E04AEF53E4C701C3
:108EB000B6010F94B81618164CF480E090E0AAEFB3
:108EC000B3E4F50180839183A283B3838CE40E9491
:108ED00041CC882309F4C1C0002E000C110B0E9464
:108EE0000ACC6B017C0120E030E0A9010F94B81698
:108EF00087FF04C0F7FAF094F7F8F09423E0000F2E
:108F0000111F2A95E1F70C59164ED8011496CD92EF
:108F1000DD92ED92FC92179720E030E04AEF53E4A7
:108F2000C701B6010F94B81618160CF096C080E071
:108F300090E0AAEFB3E4F80184839583A683B78316
:108F40008CC06091F70A70E084E50E94FFA78C0155
:108F5000823028F089E79CE00E941F4D7EC08BE4A0
:108F60000E948ACC882349F10E940ACC6B017C01C3
:108F700020E030E0A9010F94B81687FD19C020E069
:108F800030E040E251E4C701B6010F94540D1816C9
:108F90007CF00E9469D3F801FF27EE0FFF1FEE0F50
:108FA000FF1FED5AF94EC082D182E282F38255C092
:108FB0008AE59CE00E941F4D50C00E94BC4D80E598
:108FC0009CE00E941F4D03E516E1C12CD12C7601D7
:108FD00080E20E940D4DC701B6010E949F4E8DE3B5
:108FE0000E940D4DD8016D917D918D919D918D01C6
:108FF00042E00E94C84EBFEFCB1ADB0AEB0AFB0A25
:10900000E2E0CE16D104E104F10411F40C94563ED2
:10901000DFCF81E0809340021092E70A60E083E5B1
:109020000E9497CC811119C00E942D9016C00E94F9
:10903000546313C010912F178091F70A181729F065
:1090400060E083E50E9497CC01C081E0682F812F0A
:109050000E94CA8802C00E9454632296FFAD2297E4
:10906000F11102C00E94D88F2CAD20930A08ADC325
:109070000E9469D33091100B3CAB80E00E94224CDF
:109080008091590290915A02A0915B02B0915C02CA
:1090900080930D0890930E08A0930F08B0931008CA
:1090A00080916C0290916D0290930C0880930B0854
:1090B00084E690E090936D0280936C0281E080934F
:1090C00079080E9406E688E50E9441CC182F89E5C0
:1090D0000E9441CC082F8AE50E9441CC101395C113
:1090E000181711F0012F91C101E011E071E07CA788
:1090F0000E94B4CA82E50E948ACC882361F00E9453
:109100000ACC6B017C0120E030E0A9010F94540DE2
:10911000882369F106C0C12CD12C80E8E82E80E4B8
:10912000F82E111103C0002309F4FCC0C0929E0A5E
:10913000D0929F0AE092A00AF092A10AA70196019C
:109140006091000B7091010B8091020B9091030BC9
:109150000F94540D87FF0BC019821A821B821C8248
:10916000BE016F5F7F4F8EE99AE00E949CE411235D
:1091700009F4D3C0002309F4CDC01092FC0A109268
:10918000FD0A1092FE0A1092FF0A1092F80A10923D
:10919000F90A1092FA0A1092FB0A0E94D7E4EEE94B
:1091A000FBE2849188AFE2E9FBE2C590D590E590BF
:1091B000F490E6E9FBE285909590A590B490A50126
:1091C0009401C701B6010F94B81618162CF4A70124
:1091D0009601C501B40104C0A5019401C701B601FF
:1091E0000F9452152B013C01E9E5FBE225913591E5
:1091F000459154912CA33DA34EA35FA3E5E5FBE26B
:10920000459155916591749148A759A76AA77BA785
:109210009A01AB016CA17DA18EA19FA10F94B816FC
:10922000181634F428A439A45AA558AB1BA505C0B8
:109230002CA03DA06EA168AB1FA1A3019201C301A8
:10924000B2010F94BA0D20E030E040E85FE30F94E4
:1092500058140F940617910148A9512F0F94BA0D75
:1092600068A379A38AA39BA3EFE9FBE2149120E012
:1092700030E040EC5FE3C501B4010F94BA0D4B013F
:109280005C01612F110F770B880B990B0F945B0D0D
:109290009B01AC01C501B4010F94BA0D69837A83B7
:1092A0008B839C8320E030E040EC5FE3C701B60194
:1092B0000F94BA0D6B017C01A8AD6A2FAA0F770B32
:1092C000880B990B0F945B0D9B01AC01C701B60194
:1092D0000F94BA0D6C8F7D8F8E8F9F8FAE01405E85
:1092E0005F4FBE016F5F7F4FCE014C960E947AE4C4
:1092F0000F94E2061092FC0A1092FD0A1092FE0AE8
:109300001092FF0A1092F80A1092F90A1092FA0AC3
:109310001092FB0A80E00F942905002319F081E0E8
:109320000F942905BCA5BB2309F44BC080917C197F
:109330008370833061F060E08EE097E00E9404DF8C
:109340000E94BC4D8FEF96E00E941F4D3AC00E94D4
:10935000D7E480E090E0A8E4B2E48093960A90938A
:10936000970AA093980AB093990A80E090E0ACE83D
:10937000B2E480939A0A90939B0AA0939C0AB093BC
:109380009D0A8091000B9091010BA091020BB0916E
:10939000030B80939E0A90939F0AA093A00AB09318
:1093A000A10A19821A821B821C82AE014F5F5F4F95
:1093B0006AE97AE086E99AE00E947AE482E00F9412
:1093C00029050E94D7E480917808809379088CA9B8
:1093D0000E94224C80910D0890910E08A0910F08D8
:1093E000B09110088093590290935A02A0935B02A7
:1093F000B0935C0280910B0890910C0890936D02E1
:1094000080936C020E94D9E428CE8CA771CEB11053
:109410000C941C3D0C94153D80E00E94AA500C94C5
:10942000483D88E50E9441CC81115F9889E50E9402
:1094300041CC81118A988AE50E9441CC882329F089
:109440008091080181708093060185E40E9441CCDF
:10945000882309F402CE12984798FFCD60E08FE28E
:1094600098E00E9404DF5F988A98809108018170DB
:109470008093060112984798F0CD0E94D2CBAB01A1
:10948000BC014093C31C5093C41C6093C51C7093D3
:10949000C61C8AE19AE10E940299DFCD61E0802F2B
:1094A0000E94D5666F2D802F0E94A6666F2D70E0FA
:1094B000802F0E94116747E0E41203C0F092E71684
:1094C000CCCD59E0E512C9CDF092E616C6CD0E948A
:1094D000E2CB90E08536910514F084E690E080932D
:1094E0004419BBCD0E9465710C949A40802F0E9454
:1094F0003C850C94B6400E940ACC0F94C415CB0155
:109500000E94A6CA0E940ACC20E030E040EA50E463
:109510000F94B816181614F40E94657160915508DE
:1095200070915608072E000C880B990B0F945B0D59
:10953000209151083091520840915308509154089D
:109540000F94B81618161CF482E499E002C083E365
:1095500099E060E00E9404DF812F0E94CC857DCDE0
:109560000E9469D388E50E9441CC882331F05F9A3C
:1095700080917C198E7F80937C1989E50E9441CC73
:10958000882331F08A9A80917C198D7F80937C1991
:109590008AE50E9441CC882359F08091080180958A
:1095A00081708093060180917C198B7F80937C1958
:1095B00085E40E9441CC882309F44FCD0E94924C4F
:1095C0004CCD83E50E948ACC882391F00E940ACC7E
:1095D0006093CC167093CD168093CE169093CF16D1
:1095E0006093D4167093D5168093D6169093D716A1
:1095F00080E50E948ACC882351F00E940ACC6093B7
:10960000CC167093CD168093CE169093CF1682E52C
:109610000E948ACC882351F00E940ACC6093D01615
:109620007093D1168093D2169093D31684E50E943E
:109630008ACC882309F411CD0E940ACC6093D416F9
:109640007093D5168093D6169093D71606CD82E4E4
:109650000E9441CC882351F00E944CA96093A81627
:109660007093A9168093AA169093AB1683E50E9477
:1096700041CC882351F00E940ACC6093D816709395
:10968000D9168093DA169093DB1684E50E9441CCBC
:10969000882351F00E940ACC6093DC167093DD168B
:1096A0008093DE169093DF168AE40E9441CC8823D3
:1096B00009F4D3CC0E940ACC6B017C012AE037ED7F
:1096C00043E25CE30F94B81687FD3DC02AE939E90F
:1096D00049E95EE3C701B6010F94540D18169CF1D9
:1096E000C0923716D0923816E0923916F0923A1698
:1096F0006091A4167091A5168091A6169091A71658
:109700000F94590D4B015C0123EF34E045E35FE317
:10971000C701B6010F94BA0D9B01AC01C501B4019C
:109720000F94BA0D29E732E84AE550E40F94BA0DD8
:109730000F94061760934F1670935016809351162E
:10974000909352168ACC0E94B84D8AE79BE00E9403
:109750001F4D83CC0E940ACC20E030E040E050EC6A
:109760000F94540D87FD12C00E940ACC20E030E017
:1097700040E050E40F94B81618161CF00E940ACC72
:1097800009C060E070E080E090E404C060E070E058
:1097900080E090EC2091B4163091B5164091B61649
:1097A0005091B7160F94BA0D0F94C415CB010E94B7
:1097B000F2F353CCF7FAF094F7F8F094D101CD928C
:1097C000DD92ED92FC921397C9CACF5BDF4F0FB6C3
:1097D000F894DEBF0FBECDBFDF91CF911F910F91E7
:1097E000FF90EF90DF90CF90BF90AF909F908F90C1
:1097F0007F906F905F904F903F902F900895CF9300
:10980000DF931092CA181092CB181092CC181092B5
:10981000CD1884E6EEECF8E1DF011D928A95E9F7B8
:10982000C0E0D0E020E030E0A9016D2F8C2F0E9435
:10983000C0BFDF5FD530B1F7CF5FC53091F7DF91A3
:10984000CF9108959091100B9817D1F00E9469D391
:109850008091100B882359F040E05BE06CEF7AE0D8
:1098600088EF9AE00E94AED51092100B07C081E0FD
:109870008093100B88EF9AE00E947AD50C94D7E47D
:109880000895EF92FF921F93CF93DF938EECE82E13
:1098900088E1F82E15E0C0E0D0E020E030E0A9013A
:1098A000F701EC0FFD1F60817181828193810F941C
:1098B000540D81110CC02496C431D10571F711509B
:1098C00084E1E80EF11C1111E6CF80E001C081E0D7
:1098D000DF91CF911F91FF90EF900895CF92DF928B
:1098E000EF92FF926B017C0183E3C816D104E1047F
:1098F000F10470F082E3C81AD108E108F10862E3CC
:1099000070E080E090E00E94F9670E94A5F5ECCF3E
:10991000C701B6010E94F967FF90EF90DF90CF90EA
:109920000C94A5F5129A479A0895FF920F931F93EE
:10993000CF93DF931F92CDB7DEB7F82E0BEA1CE072
:1099400041E050E0B801CE0101960F948E0C898160
:109950008F1102C081E007C00F5F1F4F8CE0073CF2
:10996000180771F780E00F90DF91CF911F910F9151
:10997000FF90089580911708811107C00E94E2F0BE
:10998000882319F081E080931708089560E070E063
:1099900080E00E94A7F960E070E081E00C94A7F9F4
:1099A0008F929F92AF92BF92CF92DF92EF92FF92EF
:1099B0000F93CF93DF931F92CDB7DEB75C016B019E
:1099C0007A014901F501808191810F948413898383
:1099D000002311F0F6018083BE016F5F7F4FC40149
:1099E0000E9445F1F50180819181019691838083E8
:1099F000FFEFCF1ADF0A81E0E81AF10819F780E0DB
:109A00000F90DF91CF910F91FF90EF90DF90CF906B
:109A1000BF90AF909F908F9008959091C00095FF58
:109A2000FCCF8093C6000895CF93C82FCC2329F094
:109A300080E20E940D4DC150F9CFCF910895CF9390
:109A4000DF93FC018491EF012196882321F00E948D
:109A50000D4DFE01F7CFDF91CF9108950F931F9326
:109A6000CF938C01C62F84E99DE00E941F4DC80151
:109A70000E941F4DCC2331F08AE0CF911F910F91AE
:109A80000C940D4DCF911F910F91089560E089EADC
:109A90009DE00E942E4D85EA9DE00E941F4D8AE0C8
:109AA0000C940D4D60E089EA9DE00E942E4D81EB03
:109AB0009DE00E941F4D8AE00C940D4DEF92FF92A5
:109AC0000F931F93CF937C018B01C42F60E089EA31
:109AD0009DE00E942E4DC7010E941F4D80E20E9412
:109AE0000D4DC8010E941F4DCC2341F08AE0CF915B
:109AF0001F910F91FF90EF900C940D4DCF911F91FE
:109B00000F91FF90EF90089541E0BC018EE99DE038
:109B10000C945E4D0F931F93CF93DF938B01EA015B
:109B200080939E180E94464D41E0B8018FEC9AE266
:109B30000E945E4D209719F0CE010E94844DDF9166
:109B4000CF911F910F910C94524D0F931F93CF9370
:109B5000DF938B010E941F4DE8018991882319F042
:109B60000E940D4DFACFDF91CF911F910F91089573
:109B70008AE79DE00C941F4D84E79DE00C941F4DF7
:109B80007F928F929F92AF92BF92CF92DF92EF928D
:109B9000FF920F931F93CF93DF931F92CDB7DEB742
:109BA0007C0159018B016B01C40ED51E0C151D05DE
:109BB00059F1F70180809180F80171908F017982CD
:109BC000C4010F948413781691F0672DC4010F948B
:109BD0008C13C4010F9484139981891741F00E945A
:109BE000BC4D81E99CE00E941F4D81E00EC0BE018A
:109BF0006F5F7F4FC5010E9445F1F7018081918120
:109C0000019691838083D2CF80E00F90DF91CF9136
:109C10001F910F91FF90EF90DF90CF90BF90AF908A
:109C20009F908F907F9008958F929F92AF92BF9256
:109C3000EF92FF920F931F93CF93DF93CDB7DEB7D1
:109C4000A0970FB6F894DEBF0FBECDBF61157105AA
:109C50008105910591F100E0842E912CA12CB12C6D
:109C6000102FEE24E394F12CEC0EFD1EE00EF11CFF
:109C700007FDFA94A50194010F94AA13F7016083DC
:109C8000B901CA010F5F611571058105910541F7A1
:109C90001F3F31F1E1E0F0E0EC0FFD1FE10FF11D9E
:109CA00017FDFA9580818A3010F097E301C090E3A8
:109CB000890F0E940D4D1150EBCF80E3A0960FB697
:109CC000F894DEBF0FBECDBFDF91CF911F910F91F2
:109CD000FF90EF90BF90AF909F908F900C940D4DA0
:109CE000A0960FB6F894DEBF0FBECDBFDF91CF9127
:109CF0001F910F91FF90EF90BF90AF909F908F902A
:109D00000895CF92DF92EF92FF926A017B010E9449
:109D10001F4D4AE0C701B601FF90EF90DF90CF9052
:109D20000C94144ECF93DF93EB010E941F4DBE01A4
:109D300080E090E04AE0DF91CF910C94144ECF92F6
:109D4000DF92EF92FF926B017C0197FF0BC08DE2D7
:109D50000E940D4DF094E094D094C094C11CD11C8D
:109D6000E11CF11C4AE0C701B601FF90EF90DF90C3
:109D7000CF900C94144ECF93DF93EB010E941F4DB4
:109D8000BE01DD0F880B990BDF91CF910C949F4E94
:109D90008F929F92AF92BF92CF92DF92EF92FF92FB
:109DA000CF936B017C01B42E20E030E0A9010F9429
:109DB000540D87FF07C08DE20E940D4DF7FAF09415
:109DC000F7F8F094C0E060E070E080E09FE3CB152E
:109DD00041F02DEC3CEC4CEC5DE30F94BA0DCF5F01
:109DE000F6CF9B01AC01C701B6010F9458146B016B
:109DF0007C010F94CB154B015C014AE00E94144E8C
:109E0000CC2389F1C501B4010F94590D9B01AC011C
:109E1000C701B6010F9457146B017C018EE20E94BA
:109E20000D4D20E030E040E251E4C701B6010F944F
:109E3000BA0D4B015C010F94C4156B01770FEE084E
:109E4000FF08C701B6010E949F4EC701B6010F94DB
:109E50005B0D9B01AC01C501B4010F9457146B015C
:109E60007C01C150F1F6CF91FF90EF90DF90CF9041
:109E7000BF90AF909F908F9008958F929F92AF92D6
:109E8000BF92CF92DF92EF92FF920F931F93CF93E7
:109E9000DF93CCE2D6E08991882319F00E940D4D22
:109EA000FACF6091CA187091CB188091CC1890911C
:109EB000CD1845E00E94C84E81E89DE00E941F4DEC
:109EC000C12CD12C760188E00E94144DC701B60147
:109ED0000E949F4E8FEFC81AD80AE80AF80A95E048
:109EE000C916D104E104F10471F78AE00E940D4D16
:109EF0000EEC18E1C12CD12C760180E20E940D4DB0
:109F0000C701B6010E949F4EC0E0D0E080E20E94EF
:109F10000D4DF801EC0FFD1F80809180A280B38071
:109F2000A5019401C501B4010F944A17811112C013
:109F300020E030E0A901C501B4010F94B81687FDF7
:109F400003C08BE20E940D4D45E0C501B4010E94A3
:109F5000C84E09C0B12C80E20E940D4DB3948DE330
:109F600098E0B912F9CF6496C436D10579F68AE043
:109F70000E940D4D8FEFC81AD80AE80AF80A0C5F44
:109F80001F4F95E0C916D104E104F10409F0B5CFE3
:109F90008AE0DF91CF911F910F91FF90EF90DF90BA
:109FA000CF90BF90AF909F908F900C940D4DCF921B
:109FB000DF92EF92FF926A017B010E941F4D42E007
:109FC000C701B601FF90EF90DF90CF900C94C84E80
:109FD0008DE00E940D4D8AE00C940D4DCF93DF93E0
:109FE000EC018991882319F00E940D4DFACFDF9181
:109FF000CF910C94E84FCF93DF93CDB7DEB7A897FE
:10A000000FB6F894DEBF0FBECDBF8C010E94378F14
:10A010000E94B84D84E59DE00E941F4D0115110579
:10A0200011F40BE41DE08091D00780FD75C08160C4
:10A030008093D00781E496E00E94EE4F88248394B9
:10A040008AE5982E9092241B8092231B8FE090E04B
:10A050009093261B8093251B97E0A92EA092171B97
:10A0600022E8B22EB0921A1B34E8C32ED12CE12C78
:10A07000F12CC0921B1BD0921C1BE0921D1BF09276
:10A080001E1B0E94AEF19092241B8092231B88E538
:10A0900090E09093261B8093251BA092171BB092F3
:10A0A0001A1BC0921B1BD0921C1BE0921D1BF0922E
:10A0B0001E1B0E94AEF163E070E080E090E00E9421
:10A0C000A5BF8AE289838A838B838C83DE01159600
:10A0D000F801CE0101969D01281B390B4491319660
:10A0E000442311F04D93F7CFFC01E20FF31F2AE256
:10A0F000AF01481B590B4832510511F02193F8CF9D
:10A1000040E650E160E070E00E945DF16AE070E0DE
:10A1100080E090E00E94A5BF61E082E49DE00E94A3
:10A120002E4D89EE93E030E6019729F0232F2A95F2
:10A130000000E9F7F9CFF89489EE93E038EE019743
:10A1400029F0232F2A950000E9F7F9CF0E94378FD5
:10A15000A895FECF2F923F924F925F926F927F927F
:10A160008F929F92AF92BF92CF92DF92EF92FF9227
:10A170000F931F93CF93DF93CDB7DEB727970FB61B
:10A18000F894DEBF0FBECDBF89830E94C5190E941F
:10A1900033686B017C0180910302882359F180911F
:10A1A0000A08882339F140911808509119086091E4
:10A1B0001A0870911B0897018601041B150B260BCA
:10A1C000370B37FD2AC0833079F03CF4813094F0AE
:10A1D0000E94BC4D86EF9CE00BC0843059F40E9475
:10A1E000BC4D87EC9CE004C00E94BC4D8FED9CE010
:10A1F0000E941F4D2091030230E0A8EEB3E00F94BF
:10A20000FE13C60ED71EE81EF91EC0921808D09283
:10A210001908E0921A08F0921B0880910D0A843008
:10A2200020F40E9472900E9493920E9433686B0106
:10A230007C014091050850910608609107087091D3
:10A240000808411551056105710529F180917419BE
:10A2500090917519A0917619B0917719840F951F77
:10A26000A61FB71FA7019601281B390B4A0B5B0BD2
:10A2700057FD11C00E94B84D6091E90A7091EA0A39
:10A2800088E09DE00E94A54D8AE00E940D4D80E08F
:10A2900090E00E94FB4F40910402509105026091B2
:10A2A000060270910702411551056105710509F417
:10A2B0004FC09091911A8091921A981759F00E946C
:10A2C000336860937419709375198093761990931D
:10A2D00077193EC080910F0A811138C009810111A0
:10A2E00035C08091741990917519A0917619B0912B
:10A2F0007719840F951FA61FB71FA7019601281B6A
:10A30000390B4A0B5B0B57FD21C080912C08811142
:10A310001FC081E080932C085F9A80917C198E7F0A
:10A3200080937C198A9A80917C198D7F80937C1907
:10A3300080910801809581708093060180917C193D
:10A340008B7F80937C190E94924C02C010922C0843
:10A350008091280890912908A0912A08B0912B0893
:10A36000B701A601481B590B6A0B7B0B77FDCDC1CA
:10A370009091911A8091921A6091390250913A020B
:10A380005983981317C08091E616869FB001112457
:10A39000660F672F661F770B71956A838091E716AA
:10A3A000859FB0011124660F672F661F770B71958B
:10A3B00069832AC08091921A74E5879FC001112495
:10A3C0008C559F4EFC01EE5AFF4F2081269FB00115
:10A3D0001124660F672F661F770B71956A8331967C
:10A3E00080819981899FB0011124660F672F661FB4
:10A3F000770B719569838091921A9091911A9817B1
:10A4000019F08F5F8F70F9CF0A81002349F10E9404
:10A410003368009120081091210820912208309182
:10A420002308DC01CB01011511052105310579F463
:10A430008C599F4FAF4FBF4F8093200890932108B6
:10A44000A0932208B09323081FEF1A8311C0801B2A
:10A45000910BA20BB30BB7FF0BC00FEF0A8308C021
:10A4600010922008109221081092220810922308BE
:10A470001A81612F70E089E00E9411670981002331
:10A4800049F10E9433680091240810912508209119
:10A49000260830912708DC01CB01011511052105A3
:10A4A000310579F48C599F4FAF4FBF4F80932408EB
:10A4B00090932508A0932608B09327081FEF1983CF
:10A4C00011C0801B910BA20BB30BB7FF0BC00FEF9A
:10A4D000098308C0109224081092250810922608BB
:10A4E000109227081981612F70E087E00E941167A0
:10A4F00080919316882309F4FBC0209029023090A4
:10A500002A0200912B020F8310912C021E8360916E
:10A510003E0870913F086E5F7F4F072E000C880B3E
:10A52000990B0F945B0D9101A8010F94540D87FDB9
:10A53000DFC00091921A09831A821B821C821D823D
:10A540008091911A1981811709F460C0812F90E0E0
:10A5500024E5289FF001299FF00D1124EC55FF4EB2
:10A56000458956896789708D452B462B472B81F489
:10A57000418D528D638D748D452B462B472B41F4B5
:10A58000458D568D678D70A1452B462B472BC9F104
:10A5900034E5389F8001399F100D11240C551F4E52
:10A5A000F80161817281838194810F9406174B01B8
:10A5B0005C01F80161A172A183A194A10F94590DCE
:10A5C0002B013C01F80165A176A187A190A50F940C
:10A5D000590D9B01AC01C301B2010F945215A501A5
:10A5E00094010F94BA0D5B018C012A813B814C814F
:10A5F0005D810F94B816181624F4AA82BB820C83CE
:10A600001D8389818F5F8F7089839ACF20912D025E
:10A6100030912E0240912F02509130026A817B814D
:10A620008C819D810F94BA0D91014F815E810F94B1
:10A6300058145B018C016090250270902602809076
:10A640002702909028029B01AC01B1018F819E816D
:10A650000F94B81618167CF09301A401B501C80137
:10A660000F94B816181624F413018F829E8203C02B
:10A6700015010F831E8380901C0890901D08A090E8
:10A680001E08B0901F0891014F815E81C501B40181
:10A690000F94B8161816D4F420E037ED43EA5CE3C3
:10A6A000B1018F819E810F94BA0D2B013C0128E4EA
:10A6B00031EE4AE75FE3C501B4010F94BA0DA3017F
:10A6C00092010F9458141B018F839E83C101AF81A7
:10A6D000BE8180931C0890931D08A0931E08B09320
:10A6E0001F08B101CD010F94C415CB010E944BA1ED
:10A6F000F4E6CF0ED11CE11CF11CC0922808D092C8
:10A700002908E0922A08F0922B080E94A5F5809172
:10A710009F10813009F06EC00E9433686B017C018C
:10A720008091310890913208A0913308B09134089B
:10A7300097018601081B190B2A0B3B0B37FD3AC00A
:10A740008090A0109090A110A090A210B090A310A3
:10A750000E94B4DD6093A0107093A1108093A210AA
:10A760009093A31000916C0810916D0820916E08D1
:10A7700030916F08081919092A093B09DC01CB013E
:10A78000800F911FA21FB31F80936C0890936D08D8
:10A79000A0936E08B0936F08D701C601805F984DF3
:10A7A000AF4FBF4F8093310890933208A093330886
:10A7B000B093340880912D0890912E08A0912F0815
:10A7C000B0913008A7019601281B390B4A0B5B0B8F
:10A7D00057FD10C030E8C30E3EEED31EE11CF11C45
:10A7E000C0922D08D0922E08E0922F08F0923008E7
:10A7F0000E94A37180910008882391F00E94336821
:10A800000091FC071091FD072091FE073091FF0792
:10A81000DC01CB01801B910BA20BB30BB7FF44C033
:10A820000E9433686B017C012091FB07222309F40D
:10A830005AC08091F7079091F807A091F907B0915D
:10A84000FA07B701A601481B590B6A0B7B0B77FD72
:10A850004AC030E0A8EEB3E00F94FE13C60ED71E38
:10A86000E81EF91EC092F707D092F807E092F907A8
:10A87000F092FA0727960FB6F894DEBF0FBECDBF51
:10A88000DF91CF911F910F91FF90EF90DF90CF90CC
:10A89000BF90AF909F908F907F906F905F904F9000
:10A8A0003F902F900C948E570E9433686B017C016F
:10A8B0002091000830E0A8EEB3E00F94FE13C60E1E
:10A8C000D71EE81EF91EC092FC07D092FD07E09249
:10A8D000FE07F092FF078091F70A0E945A858AE0EE
:10A8E0000E940D4D9DCF27960FB6F894DEBF0FBE88
:10A8F000CDBFDF91CF911F910F91FF90EF90DF902F
:10A90000CF90BF90AF909F908F907F906F905F900F
:10A910004F903F902F900895809132179091331768
:10A92000981759F0E92FF0E0EE5CF84E82819F5FB6
:10A930009F779093331790E008958FEF9FEF0895DE
:10A940001F920F920FB60F9211240F900FBE0F900F
:10A950001F9018951F920F920FB60F9211240BB6ED
:10A960000F920F931F932F933F934F935F936F9388
:10A970007F938F939F93AF93BF93CF93DF93EF9387
:10A98000FF9300913317D091321711E01D0F1F77FD
:10A99000C091C60090911608492F092E000C550B46
:10A9A000660B770B4131510508F064C0FA01882726
:10A9B000ED56FF4F8F4F0D944314CD3449F0CE34F4
:10A9C000B9F481E006C0CA3338F0CD3409F043C091
:10A9D00082E08093160875C0C03308F072C0C032A0
:10A9E00009F46FC0CD32B9F56CC0C13351F018F421
:10A9F000C03289F566C0C43331F0C83361F58BE0ED
:10AA0000E8CF83E0E6CF88E0E4CFC03321F0C13364
:10AA100011F586E0DECF84E0DCCFC833E1F485E0D9
:10AA2000D8CFC233C1F487E0D4CFC133A1F489E0D9
:10AA3000D0CFC03381F48AE0CCCFC73361F48CE04F
:10AA4000C8CFC63341F48DE0C4CFC032D1F1C33595
:10AA500011F48EE0BECF80E1BCCF80ED8C0F8A3048
:10AA600080F59FE090931608809315082AC0CA309D
:10AA700041F525C0CA3029F58091851B8823F9F05E
:10AA8000973089F03CF49530D1F41092170210926F
:10AA9000431915C09A3059F09F3089F480911508F8
:10AAA0000E946ED00CC081E080932F1D08C00E94D0
:10AAB00053D50E9469D30E94F2620E94D7E410929B
:10AAC0001608011731F0ED2FF0E0EE5CF84EC2836E
:10AAD000D12FD0933217FF91EF91DF91CF91BF919A
:10AAE000AF919F918F917F916F915F914F913F9126
:10AAF0002F911F910F910F900BBE0F900FBE0F90D3
:10AB00001F9018958EBD0DB407FEFDCF08958FEFF1
:10AB10008EBD0DB407FEFDCF8EB5089590916400F3
:10AB20009B7F90936400982F906A96959CBD80FDC2
:10AB300003C091E0863009F490E09DBD0895CF9266
:10AB4000DF92EF92FF920F931F93CF93DF936C01ED
:10AB50007A018B01C0E0D0E0CE15DF0581F0D8018D
:10AB60006D918D01D601ED91FC910190F081E02D68
:10AB7000C6011995892B11F02196EECF7E01C701F0
:10AB8000DF91CF911F910F91FF90EF90DF90CF90C9
:10AB90000895089580E090E00895FC01538D448D60
:10ABA000252F30E0842F90E0821B930B541710F078
:10ABB000CF96089501970895FC01918D828D981785
:10ABC00061F0828DDF01A80FB11D5D968C91928D91
:10ABD0009F5F9F73928F90E008958FEF9FEF08958E
:10ABE000FC01918D828D981731F0828DE80FF11D57
:10ABF000858D90E008958FEF9FEF0895FC01918D72
:10AC0000228D892F90E0805C9F4F821B91098F736A
:10AC1000992708958DE799E10E94FE5521E0892B3F
:10AC200009F420E0822F0895FC01848DDF01A80F34
:10AC3000B11DA35ABF4F2C91848D90E001968F7364
:10AC40009927848FA689B7892C93A089B1898C9183
:10AC5000837080648C93938D848D981306C00288D2
:10AC6000F389E02D80818F7D80830895EF92FF929C
:10AC70000F931F93CF93DF93EC0181E0888F9B8D1F
:10AC80008C8D981305C0E889F989808185FD26C0DF
:10AC9000F62E0B8D10E00F5F1F4F0F731127E02E64
:10ACA0008C8DE8120CC00FB607FCFACFE889F98941
:10ACB000808185FFF5CFCE010E941456F1CF8B8D98
:10ACC000FE01E80FF11DE35AFF4FF0829FB7F894A1
:10ACD0000B8FEA89FB89808180620AC09FB7F89454
:10ACE000EE89FF896083E889F989808183708064B7
:10ACF00080839FBF81E090E0DF91CF911F910F9102
:10AD0000FF90EF900895CF93DF93EC01888D882317
:10AD1000C9F0EA89FB89808185FD05C0A889B989C8
:10AD20008C9186FD0FC00FB607FCF5CF808185FFA3
:10AD3000F2CFA889B9898C9185FFEDCFCE010E9411
:10AD40001456E7CFDF91CF91089580E090E0892BF2
:10AD500041F080E090E0892B21F00E9400008111F9
:10AD600021C080E090E0892B41F080E090E0892BC9
:10AD700021F00E940000811118C080E090E0892B32
:10AD800021F00E940A56811113C080E090E0892BC7
:10AD9000A1F080E090E0892B81F00E9400008111F9
:10ADA0000AC008950E940000DCCF0E940000E5CF99
:10ADB0000E940000EACF0C9400000895FC0120E0FE
:10ADC0003EE2DB014C91403241F0283011F43083F7
:10ADD0003196DB014C91408331962F5F6F5F7F4F3F
:10ADE0002B3079F7108208950F946A170F931F93F1
:10ADF000CF93DF938B01EA01DB016D917C910E947F
:10AE0000089AD801ED91FC9111979081888199233E
:10AE100049F0893638F43196ED93FC9388818F5F41
:10AE20008883EFCF893658F48FE28083F8018081E0
:10AE3000918101969183808388818F5F8883DF91E0
:10AE4000CF911F910F9108951F920F920FB60F92FD
:10AE500011240BB60F922F933F934F935F936F93F1
:10AE60007F938F939F93AF93BF93EF93FF938DE760
:10AE700099E10E941456FF91EF91BF91AF919F917C
:10AE80008F917F916F915F914F913F912F910F9093
:10AE90000BBE0F900FBE0F901F9018951F920F9230
:10AEA0000FB60F9211240BB60F922F938F939F938F
:10AEB000EF93FF93E0918D19F0918E198081E091CD
:10AEC0009319F091941982FD12C090818091961986
:10AED0008F5F8F7320919719821751F0E091961927
:10AEE000F0E0E358F64E958F8093961901C080816B
:10AEF000FF91EF919F918F912F910F900BBE0F902B
:10AF00000FBE0F901F9018958BE1E3E7FAE1A8E5DB
:10AF1000BAE101900D928A95E1F708958091C71CDE
:10AF200082FF1FC081E490E10E941F4D6091C31C0D
:10AF30007091C41C8091C51C9091C61C4AE00E946F
:10AF4000144E8FE20E940D4D6091BF1C7091C01C89
:10AF50008091C11C9091C21C4AE00E94144E0C9436
:10AF6000E84F83E590E10C941F4D10920F0A8091F9
:10AF7000C71C8F7D8B7F8093C71C0E94D6C88823F7
:10AF800021F08AE19AE10C946E9C08958091C71C8F
:10AF900083FF03C084608093C71C0895CF92DF9223
:10AFA000EF92FF920F931F93CF93DF93CDB7DEB74E
:10AFB000EDB6FEB6DC010D900020E9F79D01281BDF
:10AFC000390B2C5F3F4F4DB75EB7421B530B0FB68B
:10AFD000F8945EBF0FBE4DBF0DB71EB70F5F1F4F7A
:10AFE0009F938F938DE39FE09F938F931F930F9376
:10AFF0000F94EC0C680154E0C50ED11C0F900F901B
:10B000000F900F900F900F90F6018081882349F0E8
:10B01000082E000C990B0F946F17F60181936F01A6
:10B02000F3CFC8010E94069289E39FE00E94389204
:10B030000FB6F894FEBE0FBEEDBEDF91CF911F910B
:10B040000F91FF90EF90DF90CF9008958F929F9295
:10B05000AF92BF92CF92DF92EF92FF92CF93809107
:10B06000C71C877F8093C71C8091761A882321F0A4
:10B0700083E79AE10E946E9C1092571A1092541A1C
:10B0800085E38093531A0E9433686B017C0120EDA5
:10B09000C20E27E0D21EE11CF11CA89561E0809150
:10B0A000531A0E94A66661E08091531A0E94D566E9
:10B0B000209A289A219A2398229A81E00E948E55FC
:10B0C00085E08093551A0E948E55CAE08FEF0E944A
:10B0D0008255C150D9F7A89520E030E0A90160E081
:10B0E00083E59AE10E944E9B8093561A813061F06D
:10B0F0000E943368DC01CB018C199D09AE09BF09A0
:10B10000B7FDEACF81E062C0A8952AEA31E040E0CD
:10B1100050E068E083E59AE10E944E9B853011F48F
:10B1200081E00AC0C4E00E9487558093561AC1503E
:10B13000D1F78A3A61F482E08093571AA8958091FA
:10B14000571A823081F0812C912C540111C00E9439
:10B150003368DC01CB018C199D09AE09BF09B7FD2D
:10B16000D4CF82E033C0812C912CA12C80E4B82E66
:10B1700020E030E0A90167E383E59AE10E944E9B5D
:10B18000A501940169E283E59AE10E944E9B8093B8
:10B19000561A882361F00E943368DC01CB018C19B8
:10B1A0009D09AE09BF09B7FDE3CF8AE00FC08091CA
:10B1B000571A823021F520E030E0A9016AE383E5E7
:10B1C0009AE10E944E9B882361F088E08093541A94
:10B1D00083E59AE10E94469B0E94BC4D8BE29FE072
:10B1E00022C00E948755807C803C19F483E08093C4
:10B1F000571A0E9487550E9487550E94875583E5FC
:10B200009AE10E94469B1092551A81E00E94BD600F
:10B2100081110CC080E00E94BD60811107C00E94B6
:10B22000B84D87E19FE00E941F4D1AC065E37AE1A7
:10B2300083E79AE10E949999811105C00E94B84D57
:10B2400086E09FE0F0CF8091C71C88608093C71C88
:10B250000E94BC4D8AEF9EE00E941F4D0E94BA4C96
:10B26000CF91FF90EF90DF90CF90BF90AF909F90E5
:10B270008F900C9484572F923F925F926F927F929F
:10B280008F929F92AF92BF92CF92DF92EF92FF92F6
:10B290000F931F93CF93DF93CDB7DEB7C356D1097A
:10B2A0000FB6F894DEBF0FBECDBF8C016B014A0113
:10B2B0002DB63EB6512C7E0187E5E80EF11CF60155
:10B2C0008381823008F41FC180859185A285B38572
:10B2D0008F719927AA27BB27892B8A2B8B2B09F0E3
:10B2E00012C11092200D40E25DE0BE016F5F7F4F02
:10B2F000C6010E94039E18160CF005C18C85982F7C
:10B300009871903129F420917D0A2150223078F4EF
:10B310002981222309F4F7C0253E89F22E3279F2E1
:10B320002091200D2E3259F28A7049F67CC06DB6FC
:10B330007EB6BE016F5F7F4FC7010E94DE560115CA
:10B34000110521F0F8018081811163C021E081E0C5
:10B3500090E0F70101900020E9F73197EE19FF091D
:10B36000E80FF91F32968DB79EB78E1B9F0B0FB655
:10B37000F8949EBF0FBE8DBFEDB7FEB731965F014B
:10B38000211102C0B80102C06EE876E0C5010F9439
:10B39000B617B701C5010F94A0176EE876E0C50196
:10B3A0000F94A01719A21CA221E0A701B601CE019B
:10B3B00081960E945AA081110DC080917D0A811151
:10B3C00009C00E94BC4D86EE9EE00E941F4DC70141
:10B3D0000E94EE4F8BE1FE01B196DE01DC960190FA
:10B3E0000D928A95E1F740E050E0BE01645C7F4F2A
:10B3F000C5010E943B59CE01CC960E94779CCE019C
:10B4000081960E94779C0FB6F8947EBE0FBE6DBEEB
:10B4100056CFF80101900020E9F73197CF01801B4A
:10B42000910B20E096CF21E0903109F020E080914F
:10B43000C71C20FB84F98093C71C903141F089859B
:10B44000873409F03CCF8A858E3709F438CF809154
:10B450007D0A813021F068F08230C1F130CF8091D7
:10B46000800A9091810A01969093810A8093800AC4
:10B4700026CFBE016F5F7F4F82E69DE00E94DE56C1
:10B480000115110529F482E6A82E8DE0B82E09C019
:10B490005801F50181915F018823A9F30E940D4DA8
:10B4A000F8CFF50181915F01882319F00E940D4DBD
:10B4B000F8CF80E20E940D4D6D8D7E8D8F8D98A10D
:10B4C0004AE00E94144E0E94E84FF9CEBE016F5F21
:10B4D0007F4F82E69DE00E94DE568114910441F088
:10B4E00062E67DE0C4010F948D17892B51F40BC0E7
:10B4F000852D90E020917E0A30917F0A8217930774
:10B5000011F05394DCCE0FB6F8943EBE0FBE2DBEA4
:10B51000CD59DF4F0FB6F894DEBF0FBECDBFDF9120
:10B52000CF911F910F91FF90EF90DF90CF90BF9040
:10B53000AF909F908F907F906F905F903F902F90F3
:10B540000895CF93DF93CDB7DEB76B970FB6F8941E
:10B55000DEBF0FBECDBF81E080937D0A1092810ACD
:10B560001092800A88E59AE10E94419B8BE1E8E510
:10B57000FAE1DE01119601900D928A95E1F740E023
:10B5800050E0BE016F5F7F4F80E090E00E943B592A
:10B59000CE0101960E94779C8091800A9091810A49
:10B5A0006B960FB6F894DEBF0FBECDBFDF91CF9183
:10B5B00008950F931F93CF93DF93CDB7DEB76B97AB
:10B5C0000FB6F894DEBF0FBECDBF8B0122E02093F3
:10B5D0007D0A90937F0A80937E0A88E59AE10E9413
:10B5E000419B8BE1E8E5FAE1DE01119601900D92B5
:10B5F0008A95E1F7A801BE016F5F7F4F80E090E080
:10B600000E943B59CE0101960E94779C6B960FB623
:10B61000F894DEBF0FBECDBFDF91CF911F910F9188
:10B620000895DF92EF92FF920F931F93CF93DF93D2
:10B6300000D01F92CDB7DEB72091C71C23FF3DC1BC
:10B64000F42EE62E8C010E94D6C8882309F481C00E
:10B65000FF2009F48CC08091BE1C882351F00E9409
:10B66000B84D8CEF9FE00E941F4D80E090E00E945B
:10B67000FB4F85E19AE09A8389838FE28093140AD5
:10B6800081E08B83F12C9BE1D92E8091BD1CF816B3
:10B6900078F4DF9CC0011124AE014D5F5F4FBE0105
:10B6A0006F5F7F4F8155944E0E94F656F394EDCF15
:10B6B0008B818B3578F4AE014D5F5F4FBE016F5FBC
:10B6C0007F4F8AE19AE10E94F65689819A8101971B
:10B6D0009A838983E981FA811082E091BE1C84E01B
:10B6E000E89FF0011124E05FF54F8091C31C909119
:10B6F000C41CA091C51CB091C61C80839183A283F9
:10B70000B3830E94BC4DB80183EE9FE00E94A54D1B
:10B710006091BE1C89E6689FB00111246C5E754F74
:10B7200088ED9FE00E94A54D4091C31C5091C41C20
:10B730006091C51C7091C61C82ED9FE00E94814EF5
:10B740008AE00E940D4D8091BE1C8F5F8093BE1CCD
:10B7500026C0FF2039F00E94BC4D82EC9FE00E9481
:10B760001F4D1DC01092BE1C82E0F82E02C0FF24A7
:10B77000F3940E94BC4D8DEB9FE00E941F4D81E031
:10B78000F81609F497C089EA9FE00E941F4DB8019E
:10B7900085EB9FE00E94A54D8AE00E940D4D0E941E
:10B7A000B557B801CE0103960E940AF38C010097A9
:10B7B00009F483C06B817C81EE2009F450C021E044
:10B7C000AC018AE19AE10E945AA0882309F43FC0A3
:10B7D00080912B1A90912C1AA0912D1AB0912E1AAB
:10B7E0008093BF1C9093C01CA093C11CB093C21C3B
:10B7F0001092C31C1092C41C1092C51C1092C61C3F
:10B80000B8018BE99FE00E94A54D4091BF1C50916B
:10B81000C01C6091C11C7091C21C83E99FE00E9412
:10B82000814E8AE00E940D4D84E89FE00E941F4DEA
:10B83000B80180E090E00E94D95A8091200D8111DA
:10B8400002C0C80102C080E29DE060E030C0B801E3
:10B8500080E79FE00E94A54D8DE69FE00FC026E5A2
:10B86000AC018AE19AE10E945AA081110AC0B80194
:10B8700089E59FE00E94A54D86E59FE00E941F4D4F
:10B880001CC08091C71C81608093C71CB80180E0F8
:10B8900090E00E94D95A1092851BB80184E49FE081
:10B8A0000E94A54D8AE00E940D4D60E0C8010E94F3
:10B8B0005FDF03C08FEA9FE068CF0F900F900F907B
:10B8C0000F90DF91CF911F910F91FF90EF90DF903C
:10B8D0000895CF92DF92EF92FF92CF936B017C019C
:10B8E000C42F8091150D9091160DA091170DB09158
:10B8F000180D8C159D05AE05BF05D1F00E94FB9B70
:10B90000811102C080E018C025E13BE0B701A6012B
:10B9100080911E0D90911F0D0E947D9C882391F3B4
:10B92000C092150DD092160DE092170DF092180DE1
:10B9300081E0C11180931D0DCF91FF90EF90DF90BA
:10B94000CF9008954F925F926F927F928F929F92C5
:10B95000AF92BF92CF92DF92EF92FF920F931F931D
:10B96000CF93DF93EC01423051056105710510F46E
:10B9700080E069C089859A85AB85BC850196A11D4B
:10B98000B11D84179507A607B70790F38F898031FB
:10B9900049F4852E962EA72EBB248B899C89AD89D0
:10B9A000BE890FC0803221F78B889C88AD88BE8805
:10B9B000DB01CA01E7E0B695A79597958795EA95CB
:10B9C000D1F7880E991EAA1EBB1E280139016A01F3
:10B9D0007B0141E0C501B4010E94695C882341F20A
:10B9E0009F89903161F4DD24EE24FF249601220F1B
:10B9F000331FF901EB5EF44F5182408211C0E8948D
:10BA0000C7F8DD24EE24FF249601220F331F220FF6
:10BA1000331FF901EB5EF44F4082518262827382E0
:10BA20009A89923080F04D815E816F817885840E95
:10BA3000951EA61EB71E8092190D90921A0DA09207
:10BA40001B0DB0921C0DDF91CF911F910F91FF90B4
:10BA5000EF90DF90CF90BF90AF909F908F907F90AE
:10BA60006F905F904F900895CF92DF92EF92FF9288
:10BA70000F931F93CF93DF93FC0181859285A3855C
:10BA8000B4850196A11DB11D84179507A607B707B8
:10BA900010F480E061C08789803149F4BB27A72F6B
:10BAA000962F852FC388D488E588F6880FC080320A
:10BAB00081F783899489A589B6896A017B01C7E0EA
:10BAC000F694E794D794C794CA95D1F78C0D9D1D31
:10BAD000AE1DBF1DE9016A017B018F014091150D6B
:10BAE0005091160D6091170D7091180D84179507E0
:10BAF000A607B70739F040E0BC01CD010E94695CA0
:10BB0000882339F2F8018789803179F4B701A601D9
:10BB1000552766277727440F551FFA01EB5EF44F30
:10BB200080819181A0E0B0E012C0B701A6014F77FB
:10BB3000552766277727440F551F440F551FFA01D5
:10BB4000EB5EF44F80819181A281B381BF708883C5
:10BB50009983AA83BB8381E0DF91CF911F910F91DD
:10BB6000FF90EF90DF90CF9008954F925F926F9289
:10BB70007F92AF92BF92CF92DF92EF92FF920F939C
:10BB80001F93CF93DF9300D01F92CDB7DEB78C0108
:10BB900049835A836B837C835901C12CD12C760154
:10BBA000412C82E0582E612C712C49815A816B8185
:10BBB0007C819E012F5F3F4FC8010E94345D882326
:10BBC00041F1D301C201F801058404C0880F991F17
:10BBD000AA1FBB1F0A94D2F7C80ED91EEA1EFB1E6D
:10BBE00049815A816B817C818789803139F481E078
:10BBF000483F5F4F6105710538F4D7CF81E0483F7A
:10BC00005F4F6F4F7F4088F2F501C082D182E282A0
:10BC1000F3820F900F900F900F90DF91CF911F91B3
:10BC20000F91FF90EF90DF90CF90BF90AF907F90FB
:10BC30006F905F904F90089590E0FC013197E23152
:10BC4000F10508F04EC08827EC55FF4F8F4F0D943B
:10BC50004314809180008F7703C0809180008F7D96
:10BC600080938000089580918000877FF9CF84B50C
:10BC70008F7702C084B58F7D84BD08958091B00018
:10BC80008F7703C08091B0008F7D8093B0000895BE
:10BC9000809190008F7707C0809190008F7D03C0C6
:10BCA00080919000877F8093900008958091A000FC
:10BCB0008F7707C08091A0008F7D03C08091A00086
:10BCC000877F8093A0000895809120018F7707C01F
:10BCD000809120018F7D03C080912001877F809318
:10BCE000200108953FB7F8948091860A9091870AC1
:10BCF000A091880AB091890A26B5A89B05C02F3F5C
:10BD000019F00196A11DB11D3FBFBA2FA92F982F81
:10BD10008827820F911DA11DB11DBC01CD0142E0FC
:10BD2000660F771F881F991F4A95D1F70895CF9303
:10BD3000DF93CDB7DEB78091E70A81110FC09E0176
:10BD4000275F3F4F46E951E16FE370E087EA9AE0F1
:10BD50000F941B0D87EA9AE00E947FC0DF91CF917C
:10BD600008952F923F924F925F926F927F928F929F
:10BD70009F92AF92BF92CF92DF92EF92FF920F937A
:10BD80001F93CF93DF93D82FC62F80E996E00E94B0
:10BD9000EE4FD1115AC0CC2389F00E94A15A8C01D8
:10BDA000C12CD12CC0E0D0E0A12CB12C80E2282EF7
:10BDB0008DE0382E44244394512C3FC00E94F3BDA3
:10BDC0008111EBCF44C0C016D10608F037C1C501C0
:10BDD0004496C816D90608F031C12FEFC21AD20A0C
:10BDE0000F3F3FEF130709F0C3C10E94A15A8C0116
:10BDF0008C159D0508F04EC1F10101900020E9F776
:10BE00003197CF0180529D403C01EE24E394F12C08
:10BE10009701205E324F490146E050E069E976E043
:10BE2000C9010F94BD17892B09F0F4C0E614F7047B
:10BE30000CF43FC18FEFA81AB80A0F3F2FEF12077B
:10BE400011F60E94A15A8C01BECFC111A6CF3AE0D3
:10BE5000C32E30E2D32EE12CF12CC5E0D2E8812CA8
:10BE6000912C54011092241B1092231BC093171B7A
:10BE7000D0931A1BD701C601880D991DAA1DBB1DA1
:10BE800080931B1B90931C1BA0931D1BB0931E1B28
:10BE90000E94AEF18FEF881A980AA80AB80A9AE0B1
:10BEA00089169104A104B104E9F62AE0C20ED11C5E
:10BEB000E11CF11C32EDC31630E2D306E104F104BB
:10BEC00071F6C12C20E2D22EE12CF12CD5E0C2E893
:10BED0001092241B1092231BD093171BC0931A1B84
:10BEE000C0921B1BD0921C1BE0921D1BF0921E1BCC
:10BEF0000E94AEF11092241B1092231BD093171BAB
:10BF0000C0931A1BD701C6018C529F4FAF4FBF4F32
:10BF100080931B1B90931C1BA0931D1BB0931E1B97
:10BF20000E94AEF18FEFC81AD80AE80AF80A9AE020
:10BF3000C91690E2D906E104F10451F69EEDC92E2E
:10BF400090E2D92EE12CF12CD5E0C2E81092241B0E
:10BF50001092231BD093171BC0931A1BC0921B1B5C
:10BF6000D0921C1BE0921D1BF0921E1B0E94AEF192
:10BF70002FEFC21AD20AE20AF20A36EEC31630E2F4
:10BF8000D306E104F10411F7CC24C39482E1D82E46
:10BF9000E12CF12C0AE010E0D5E0C2E81093241B5C
:10BFA0000093231BD093171BC0931A1BC0921B1B1B
:10BFB000D0921C1BE0921D1BF0921E1B0E94AEF142
:10BFC0001093241B0093231BD093171BC0931A1BA1
:10BFD000D701C6018096A11DB11D80931B1B9093B4
:10BFE0001C1BA0931D1BB0931E1B0E94AEF18FEF74
:10BFF000C81AD80AE80AF80A95E1C91692E1D906E2
:10C00000E104F10459F684ED93E00E94EE4F82E1E1
:10C0100090E016C046E050E060EA76E0C4010F947C
:10C02000BD17892B09F402CF3FEFE31AF30AC701CA
:10C030000197861597050CF4EBCEF8CE81E190E0E0
:10C040009093241B8093231B85E08093171B82E829
:10C0500080931A1B84E190E1A0E0B0E080931B1B69
:10C0600090931C1BA0931D1BB0931E1BDF91CF91BF
:10C070001F910F91FF90EF90DF90CF90BF90AF9006
:10C080009F908F907F906F905F904F903F902F90F8
:10C090000C94AEF10F3F8FEF180719F40E94A15ACC
:10C0A0008C0160E070E0C8018C199D090E94D95A8A
:10C0B000A3CE22E12C9FC0012D9F900D11249C0145
:10C0C0002E53324F4901A7014231510514F041E18D
:10C0D00050E060E27DE0C4010F94CB1732E13C9F59
:10C0E000C0013D9F900D112462E67DE0865D904F7A
:10C0F0000F94B6178AE08C9FA0018D9F500D1124DC
:10C10000465F5F4D052E000C660B770BFE01EE0FB0
:10C11000FF1FEE0FFF1FE159F24F438354836583E6
:10C120007683C4010E945DF17E019FEFE91AF90A4E
:10C13000F092710DE092700D5092241B4092231BDF
:10C1400025E02093171B32E830931A1BCF5FDD4E9A
:10C15000CE01DD0FAA0BBB0B80931B1B90931C1B06
:10C16000A0931D1BB0931E1B0E94AEF1E70165CE8C
:10C170000C151D0508F440CE94CF4F925F926F923C
:10C180007F928F929F92AF92BF92CF92DF92EF9267
:10C19000FF921F93CF93DF93C82F83E59AE190938B
:10C1A0001F0D80931E0D10924C1A82E090E0A0E0CB
:10C1B000B0E08093351A9093361AA093371AB09353
:10C1C000381A10921D0D1092190D10921A0D10921E
:10C1D0001B0D10921C0D8FEF9FEFDC018093150D4E
:10C1E0009093160DA093170DB093180DCC2379F1F1
:10C1F000C53008F001C140E060E070E0CB010E9472
:10C20000695C882309F4F8C020E1C29FC0011124B1
:10C210008B5F944FFC01E254FE4F20812F7709F091
:10C22000EBC03C9640815181628173814436510557
:10C230006105710508F4E0C03497C080D180E280C8
:10C24000F380C114D104E104F10421F4D5C0C12C60
:10C25000D12C760140E0C701B6010E94695C182F1D
:10C26000882309F4C9C08091200B9091210B81157E
:10C27000924009F0C1C0A091250BAA2309F4BCC0CB
:10C280006091230B7091240B6115710509F4B4C002
:10C290008090220B882009F4AFC0A093471A8092A7
:10C2A000391A80E0912CA12CB12C412C512C320157
:10C2B0004394C82FA3019201082E04C0220F331FFC
:10C2C000441F551F0A94D2F782169306A406B5069A
:10C2D00039F08F5FC83069F789E08093421A8CC0CB
:10C2E0008093421A20912B0B30912C0B2115310594
:10C2F00019F040E050E008C02091390B30913A0B22
:10C3000040913B0B50913C0B20933A1A30933B1ACF
:10C3100040933C1A50933D1A46015701860E971ED2
:10C32000A11CB11C8092481A9092491AA0924A1AF4
:10C33000B0924B1AE091260BF091270BF0934E1A16
:10C34000E0934D1AB0E00F94EB13860E971EA81ED3
:10C35000B91E80924F1A9092501AA092511AB09220
:10C36000521A85E0EE0FFF1F8A95E1F7E150FE4F6C
:10C37000EF2FFF27E6958E0E9F1EA11CB11C809209
:10C38000431A9092441AA092451AB092461A2091EC
:10C39000280B3091290B2115310521F0A90160E00E
:10C3A00070E008C04091350B5091360B6091370B0F
:10C3B0007091380BD701C60188199909AA09BB09E0
:10C3C000840F951FA61FB71F04C0B695A795979514
:10C3D0008795CA95D2F780933E1A90933F1AA093FF
:10C3E000401AB093411A853F2FE09207A105B1058D
:10C3F00028F48CE080934C1A10E01AC0853F9F4FC0
:10C40000A105B10510F480E111C08091410B90911C
:10C41000420BA091430BB091440B80934F1A909321
:10C42000501AA093511AB093521A80E280934C1A7A
:10C43000812FDF91CF911F91FF90EF90DF90CF90F0
:10C44000BF90AF909F908F907F906F905F904F9034
:10C450000895FF920F931F93CF93DF938B01D82FF3
:10C46000C92F9B01482F592F6091110B7091120B0E
:10C470008091130B9091140B0F94540D882309F4A1
:10C480005FC0F090100B80E00E94224C20E030E072
:10C49000A901B8018D2F9C2F0F94B816181624F0FF
:10C4A00000E010E0D0E0C0E0C801AD2FBC2F8093C9
:10C4B000110B9093120BA093130BB093140B2DEB55
:10C4C00037E346E855EBB8018D2F9C2F0F94B81633
:10C4D00087FD0BC02DEB37E346E855E3B8018D2F00
:10C4E0009C2F0F94540D181654F498014D2F5C2F67
:10C4F00060E070E080E89FE30F94521503C060E0B5
:10C5000070E0CB0160930C0B70930D0B80930E0BBE
:10C5100090930F0B80EF9FEFA9E7B4EC8093080B8B
:10C520009093090BA0930A0BB0930B0BFF2041F0E3
:10C5300081E0DF91CF911F910F91FF900C94224CDD
:10C54000DF91CF911F910F91FF900895CF93DF93CB
:10C55000CDB7DEB760970FB6F894DEBF0FBECDBF84
:10C56000E8EFFAE080819181A281B38189839A8387
:10C57000AB83BC8384819581A681B7818D839E83A3
:10C58000AF83B88780859185A285B38589879A878F
:10C59000AB87BC8784859585A685B7858D879E8763
:10C5A000AF87B88BAE01475F5F4FBE016B5F7F4FB8
:10C5B000CE0101960E94AED59E01235F3F4FAE0192
:10C5C000475F5F4FBE016B5F7F4FCE0101960E94B8
:10C5D000D6D360960FB6F894DEBF0FBECDBFDF9105
:10C5E000CF910895CF93DF93CDB7DEB760970FB6A5
:10C5F000F894DEBF0FBECDBF0E94BBE4EBEEFAE0C5
:10C6000080819181A281B38189839A83AB83BC832A
:10C6100084819581A681B7818D839E83AF83B887FE
:10C6200080859185A285B38589879A87AB87BC87EA
:10C630008091040B9091050BA091060BB091070B14
:10C640008D879E87AF87B88BCE0101960E947AD5E1
:10C6500080E1FE013196A8EFBAE001900D928A9533
:10C66000E1F760960FB6F894DEBF0FBECDBFDF9145
:10C67000CF9108958AE19AE10E943B9C8AE19AE178
:10C680000E946E9C8091C71C8D7F8E7F8093C71CFB
:10C690001092C31C1092C41C1092C51C1092C61C90
:10C6A00081E08093851B08950E94BC4D6091E90A4A
:10C6B0007091EA0A8BEA91E10E94A54D88EA91E126
:10C6C0000C941F4D1F93CF93DF938091A60AC82F20
:10C6D000C270D82FD470182F117080FF04C0CC23E3
:10C6E00011F0D11145C00E94BC4D80E991E10E943A
:10C6F0001F4D111103C088E50E940D4DC11103C0EB
:10C7000089E50E940D4DD11103C08AE50E940D4DAF
:10C7100088E891E10E941F4DDD2319F046EC55E0B9
:10C7200002C040EB57E0CC2319F026EC35E002C004
:10C7300027EA36E0112319F086EC95E002C081E685
:10C7400096E05F934F933F932F939F938F9386E948
:10C7500091E19F938F931F920E94975E8DB79EB732
:10C7600009960FB6F8949EBF0FBE8DBF81E001C041
:10C7700080E0DF91CF911F910895AF92BF92CF9249
:10C78000DF92EF92FF920F931F93CF93DF93CDB77A
:10C79000DEB72C970FB6F894DEBF0FBECDBF2BEDE2
:10C7A000C22E22E0D22E5C0170E0CB0185529D4F5B
:10C7B0007C01CE14DF0409F180E20E940D4DF601E8
:10C7C00081916F010E940D4D8AE30E940D4DF5018C
:10C7D00061917191819191915F018E010F5F1F4F66
:10C7E00023E041E00F942C088C01F80181918F0126
:10C7F0008823F9F20E940D4DF8CF8AE00E940D4D7A
:10C800002C960FB6F894DEBF0FBECDBFDF91CF914F
:10C810001F910F91FF90EF90DF90CF90BF90AF905E
:10C820000895CF93DF9300D01F92CDB7DEB78091EC
:10C83000921081111BC081E0809392108091920A26
:10C840009091930AA091940AB091950AB058898367
:10C850009A83AB83BC839E012F5F3F4F4EE95AE022
:10C860006AE97AE086E99AE00E94BECA0F900F90CA
:10C870000F900F90DF91CF910895CF93DF9300D069
:10C880001F92CDB7DEB7809192108823F9F02AE984
:10C8900039E949E95FE36091920A7091930A8091C6
:10C8A000940A9091950A0F94BA0D69837A838B83C9
:10C8B0009C839E012F5F3F4F4EE95AE06AE97AE080
:10C8C00086E99AE00E94BECA109292100F900F90D3
:10C8D0000F900F90DF91CF9108952F923F924F923A
:10C8E0005F926F927F928F929F92AF92BF92CF9200
:10C8F000DF92EF92FF920F931F93CF93DF93CDB709
:10C90000DEB7A0970FB6F894DEBF0FBECDBF1C01F7
:10C910008B015A8749873C872B87C090F80AD090B3
:10C92000F90AE090FA0AF090FB0ADC018D919D91E2
:10C930000D90BC91A02D8D879E87AF87B88B9C01F1
:10C94000AD01C701B6010F9457142B013C01809132
:10C95000FC0A9091FD0AA091FE0AB091FF0A898B12
:10C960009A8BAB8BBC8BD8018D919D910D90BC9116
:10C97000A02D8D8B9E8BAF8BB88F9C01AD016989EB
:10C980007A898B899C890F9457144B015C01A30110
:10C990009201C301B2010F94BA0D2B013C01A50114
:10C9A0009401C501B4010F94BA0D9B01AC01C30100
:10C9B000B2010F945814698F7A8F8B8F9C8FE98501
:10C9C000FA854080518062807380A3019201C70183
:10C9D000B6010F9457146D8F7E8F8F8F98A3AB8500
:10C9E000BC858D909D90AD90BC90A5019401698906
:10C9F0007A898B899C890F9457146B017C012D8552
:10CA00003E854F855889C301B2010F9457142B01FD
:10CA10003C012D893E894F89588DC501B4010F9481
:10CA200057144B015C01A3019201C301B2010F94A1
:10CA3000BA0D2B013C01A5019401C501B4010F946D
:10CA4000BA0D9B01AC01C301B2010F9458140F94AD
:10CA500006174B015C012D8D3E8D4F8D58A1CA01EB
:10CA6000B9010F94BA0D2B013C01A7019601C70132
:10CA7000B6010F94BA0D9B01AC01C301B2010F9432
:10CA800058149B01AC01698D7A8D8B8D9C8D0F9410
:10CA9000B816181604F520E030E0A901C501B4016C
:10CAA0000F94B81687FF04C0C501B401905802C0A6
:10CAB000C501B40120E030E040EA50E40F94B8161C
:10CAC00018164CF49801A1016B857C8589859A859F
:10CAD0000E946D6483C020E030E040E050E4698D46
:10CAE0007A8D8B8D9C8D0F94B81618160CF044C05F
:10CAF0000E94116419821A821B821C8220E030E09D
:10CB000040E05FE36091000B7091010B8091020B9C
:10CB10009091030B0F9458146D837E838F839887B5
:10CB20009E012F5F3F4FAE014B5F5F4F6CEF7AE08E
:10CB300088EF9AE00E94BECA19821A821B821C8268
:10CB400020E030E040E05FE360918A0A70918B0A58
:10CB500080918C0A90918D0A0F9458146D837E8376
:10CB60008F8398879E012F5F3F4FAE014B5F5F4FD2
:10CB7000B801C1010E94BECA19821A821B821C829E
:10CB80009E012F5F3F4F4AE85AE0B801C1010E9461
:10CB9000BECA2DEC3CEC4CEC5CE3C501B4010F9437
:10CBA000BA0D9B01AC0160918E0A70918F0A809141
:10CBB000900A9091910A0F94BA0D69837A838B83BE
:10CBC0009C830E943D649E012F5F3F4F4AE85AE0DC
:10CBD0006B857C8589859A850E94BECAA0960FB612
:10CBE000F894DEBF0FBECDBFDF91CF911F910F91A3
:10CBF000FF90EF90DF90CF90BF90AF909F908F907D
:10CC00007F906F905F904F903F902F9008954F923C
:10CC10005F926F927F928F929F92AF92BF92CF92CC
:10CC2000DF92EF92FF920F931F93CF93DF93CDB7D5
:10CC3000DEB74DB65EB66090E90A7090EA0A84E805
:10CC4000E82E81E1F82E8DB69EB66AE070E0C7014D
:10CC50000F94970C6C01009721F08C010E191F099D
:10CC600004C0C7010F94A20C8C01C80101962DB716
:10CC70003EB7281B390B0FB6F8943EBF0FBE2DBF31
:10CC80008DB79EB701965C01A801B7010F94C30C44
:10CC9000F501E00FF11F1082C5010E94D49381E0DD
:10CCA0000E94BE35C114D10451F076019FEFE91AFC
:10CCB000F90A0FB6F8949EBE0FBE8DBEC4CF0FB654
:10CCC000F8949EBE0FBE8DBEC3010E94D4930FB6D2
:10CCD000F8945EBE0FBE4DBEDF91CF911F910F91B4
:10CCE000FF90EF90DF90CF90BF90AF909F908F908C
:10CCF0007F906F905F904F900895CF93DF93282F90
:10CD000030E0F901E25CFE4E8491F901E850FF4EFB
:10CD1000D491F901EE54FF4EC491CC2391F08111CE
:10CD20000E941C5EEC2FF0E0EE0FFF1FE856FF4E56
:10CD3000A591B491EC91ED2381E090E021F480E0A5
:10CD400002C080E090E0DF91CF9108951F93CF93D0
:10CD5000DF93282F30E0F901E25CFE4E8491F90167
:10CD6000E850FF4ED491F901EE54FF4EC491CC230C
:10CD7000C1F0162F81110E941C5EEC2FF0E0EE0F27
:10CD8000FF1FE258FF4EA591B4919FB7F89411117F
:10CD900004C08C91D095D82302C0EC91DE2BDC939B
:10CDA0009FBFDF91CF911F910895CF93DF9390E0C4
:10CDB000FC01E850FF4E2491FC01EE54FF4E84919B
:10CDC000882361F190E0880F991FFC01EC59FF4E18
:10CDD000C591D491FC01E258FF4EA591B491611127
:10CDE00009C09FB7F8948881209582238883EC91AD
:10CDF0002E230BC0623061F49FB7F8948881322FE4
:10CE0000309583238883EC912E2B2C939FBF06C0F3
:10CE10008FB7F894E8812E2B28838FBFDF91CF91B5
:10CE200008951F93CF93DF93182FEB0161E00E94C9
:10CE3000D566209711F460E004C0CF3FD10539F4E6
:10CE400061E0812FDF91CF911F910C94A666E12FB5
:10CE5000F0E0E25CFE4EE4918E2F90E0FC01319711
:10CE6000E231F10508F09DC08827EA54FF4F8F4F4B
:10CE70000D94431484B5806884BDC7BD97C084B544
:10CE8000806284BDC8BD92C080918000806880931C
:10CE90008000D0938900C093880088C08091800072
:10CEA000806280938000D0938B00C0938A007EC004
:10CEB00080918000886080938000D0938D00C09323
:10CEC0008C0074C08091B00080688093B000C093E3
:10CED000B3006CC08091B00080628093B000C093BA
:10CEE000B40064C080919000806880939000D093DB
:10CEF0009900C09398005AC08091900080628093FE
:10CF00009000D0939B00C0939A0050C080919000F5
:10CF1000886080939000D0939D00C0939C0046C091
:10CF20008091A00080688093A0008091A0008F7BFA
:10CF30008093A000D093A900C093A80037C080912F
:10CF4000A00080628093A000D093AB00C093AA00A1
:10CF50002DC08091A00088608093A000D093AD0088
:10CF6000C093AC0023C08091200180688093200191
:10CF7000D0932901C093280119C0809120018062BB
:10CF800080932001D0932B01C0932A010FC0809180
:10CF90002001886080932001D0932D01C0932C0143
:10CFA00005C0C038D1050CF04BCF45CFDF91CF91F4
:10CFB0001F910895863308F0865390917B00282FA7
:10CFC0002870977F922B90937B008770806480936A
:10CFD0007C0080917A00806480937A0080917A004E
:10CFE00086FDFCCF809178002091790090E0922B13
:10CFF00008958F929F92AF92BF92CF92DF92EF925D
:10D00000FF926B017C010E94725E4B015C01C114B6
:10D01000D104E104F104F1F00E94725EDC01CB0165
:10D0200088199909AA09BB09883E9340A105B10551
:10D0300070F321E0C21AD108E108F10888EE880EE9
:10D0400083E0981EA11CB11CC114D104E104F104B9
:10D0500019F7DDCFFF90EF90DF90CF90BF90AF90AA
:10D060009F908F9008952FB7F8946091820A7091E5
:10D07000830A8091840A9091850A2FBF0895809138
:10D08000911A9091921A891B8F7019F480E090E0A8
:10D09000089590918E1A992351F0833030F48FEFD8
:10D0A000890F19F080938E1AF1CF10928E1AE091A9
:10D0B000921A84E5E89FF0011124EC55FF4E80811F
:10D0C00080FDE4CF8091921A8F5F8F7080938F1ACA
:10D0D0009091921A8091901A981304C080918F1A9F
:10D0E0008093901ACF0108950F930FB70F9300917B
:10D0F0006E000F930B7F00936E0000916F000D7F09
:10D1000000936F000F930BB70F930CB70F921F9202
:10D110002F933F934F935F936F937F938F939F933F
:10D12000AF93BF93EF93FF9311240E94E568FF91A3
:10D13000EF91BF91AF919F918F917F916F915F918F
:10D140004F913F912F911F900F900CBF0F910BBFEC
:10D150000F910260F89400936F000F9100936E009E
:10D160000F910FBF0F91189580917A0880FF03C02F
:10D1700089988FEF02C0899A81E08093E5158091AC
:10D180007A08869580FF03C08F9A8FEF02C08F9830
:10D1900081E08093E61580917A088695869580FFD8
:10D1A00008C080910B0180958270809309018FEFF8
:10D1B00006C080910B0182708093090181E0809309
:10D1C000E71500000000000008952F923F924F9253
:10D1D0005F926F927F928F929F92AF92BF92CF9207
:10D1E000DF92EF92FF920F931F93CF93DF93CDB710
:10D1F000DEB72D970FB6F894DEBF0FBECDBF8FEF11
:10D200009FEF90938900809388002AE02987212C42
:10D21000312C44244A94542C320178948091331652
:10D2200090913416A0913516B0913616892B8A2B21
:10D230008B2B09F0D9C18091121D8823E1F0109247
:10D24000121D8091101D9091111D892B09F4CCC1E4
:10D250001092E4151092111D1092101D9091911AC8
:10D260008091921A981709F4BFC18091921A8F5F2A
:10D270008F708093921A8091101D9091111D892BAF
:10D2800009F4B2C1C0902F16D0903016E09031163C
:10D29000F090321640912B1650912C1660912D165D
:10D2A00070912E1600911E1610E020E030E0DB0198
:10D2B000CA018C199D09AE09BF09081719072A0769
:10D2C0003B0710F4D901C801482F8C0D9D1DAE1DE0
:10D2D000BF1D80932F1690933016A0933116B093F4
:10D2E00032162091840030918500225E3F4FC0901D
:10D2F0000416D0900516E0900616F090071680915F
:10D30000F4159091F515A091F615B091F7158C0DC7
:10D310009D1DAE1DBF1D8093041690930516A0930E
:10D320000616B0930716B7FD1CC0889AC0901F1D43
:10D33000D090201DE090211DF090221D8091E515D8
:10D34000082E000C990BAA0BBB0B8C0D9D1DAE1D5E
:10D35000BF1D80931F1D9093201DA093211DB0938E
:10D36000221DC0900816D0900916E0900A16F09081
:10D370000B168091F8159091F915A091FA15B091BE
:10D38000FB158C0D9D1DAE1DBF1D8093081690933F
:10D390000916A0930A16B0930B16B7FD1CC08E9AFF
:10D3A000C090231DD090241DE090251DF090261DD7
:10D3B0008091E615082E000C990BAA0BBB0B8C0D67
:10D3C0009D1DAE1DBF1D8093231D9093241DA09312
:10D3D000251DB093261DC0900C16D0900D16E09020
:10D3E0000E16F0900F168091FC159091FD15A091EE
:10D3F000FE15B091FF158C0D9D1DAE1DBF1D8093B8
:10D400000C1690930D16A0930E16B0930F16B7FD41
:10D4100021C080910B018095887080930901C09094
:10D42000271DD090281DE090291DF0902A1D809185
:10D43000E715082E000C990BAA0BBB0B8C0D9D1D3C
:10D44000AE1DBF1D8093271D9093281DA093291DFD
:10D45000B0932A1DC0901016D0901116E0901216AD
:10D46000F09013168091001690910116A09102166B
:10D47000B09103168C0D9D1DAE1DBF1D809310161F
:10D4800090931116A0931216B0931316B7FD3AC0DD
:10D4900080902B1D90902C1DA0902D1DB0902E1DC6
:10D4A000C090E8150C2C000CDD08EE08FF08C80C35
:10D4B000D91CEA1CFB1CC0922B1DD0922C1DE092A3
:10D4C0002D1DF0922E1DC090F015D090F115E0901A
:10D4D000F215F090F3158C199D09AE09BF098093E0
:10D4E000101690931116A0931216B09313169091E4
:10D4F0007A0880911C1693FF02C0815001C08F5F93
:10D5000080931C1680918400909185008217930768
:10D51000C8F38091041690910516A0910616B0915B
:10D520000716B7FD15C0C090F015D090F115E0902A
:10D53000F215F090F3158C199D09AE09BF0980937F
:10D54000041690930516A0930616B09307168898B4
:10D550008091081690910916A0910A16B0910B16A9
:10D56000B7FD15C0C090F015D090F115E090F21500
:10D57000F090F3158C199D09AE09BF098093081628
:10D5800090930916A0930A16B0930B168E9880916B
:10D590000C1690910D16A0910E16B0910F16B7FDB6
:10D5A00019C0C090F015D090F115E090F215F090F0
:10D5B000F3158C199D09AE09BF0980930C16909341
:10D5C0000D16A0930E16B0930F1680910B01887064
:10D5D00080930901415041F0809184009091850031
:10D5E00082179307C8F381CE809121029091220285
:10D5F000A0912302B0912402892B8A2B8B2B09F056
:10D60000A7C080911D16882309F452C080902F1660
:10D6100090903016A0903116B0903216C090181627
:10D62000D0901916E0901A16F0901B1680911C16D7
:10D63000C814D904EA04FB0488F42091ED15309154
:10D64000EE154091EB155091EC154217530730F44D
:10D65000815080931C162150310915C08C149D04F3
:10D66000AE04BF04E8F42091ED153091EE15409121
:10D67000E9155091EA152417350790F48F5F8093D0
:10D680001C162F5F3F4F3093EE152093ED15409100
:10D690001D0250911E0260911F02709120020BC06A
:10D6A00040921D0250921E0260921F027092200250
:10D6B0004FEF5FEFBA0190911C168091EF1597FD27
:10D6C00006C0811102C0169A07C0439805C0811197
:10D6D00002C0169801C0439A2091840030918500C1
:10D6E000225E3F4F80911C16882351F18091EF15E7
:10D6F000811102C0149A01C0419A809184009091D6
:10D70000850082179307C8F380911C1687FF02C01B
:10D710008F5F01C0815080931C168091EF1581119D
:10D7200002C0149801C0419880911C168823D1F240
:10D73000809184009091850082179307C8F3D0CF21
:10D74000409321025093220260932302709324029B
:10D750008091331690913416A0913516B0913616FB
:10D76000892B8A2B8B2B09F091C3A091101DB091AE
:10D77000111D109709F4A2C5C0902F16D090301635
:10D78000E0903116F090321640912B1650912C16E5
:10D7900060912D1670912E16C416D506E606F70672
:10D7A000D0F01092E4151092111D1092101D90915E
:10D7B000911A8091921A981709F480C58091921A53
:10D7C0008F5F8F708093921A00ED802E07E0902E6D
:10D7D000A12CB12C8AC14091271650912816609136
:10D7E000291670912A164C155D056E057F0508F403
:10D7F0006DC04091231650912416609125167091AA
:10D800002616D2960D911D912D913C91D597EE271C
:10D81000419FF12D529FC001629F900D619F800D2D
:10D82000911D429FF00D811D9E1F519FF00D811D86
:10D830009E1F609FF00D811D9E1F509FF10D8E1F3A
:10D840009E1FF6958E1F9E1F349F800D911D359F44
:10D85000900D1124FD01EA5BFF4F008111812281AF
:10D860003381080F191F211D311D00931F161093BE
:10D87000201620932116309322163497C080D18031
:10D88000E280F380C016D106E206F30640F4C092AF
:10D890001F16D0922016E0922116F0922216C09008
:10D8A0001F16D0902016E0902116F09022168EEBD5
:10D8B00099E121E0FC0185909590A590B4908C149D
:10D8C0009D04AE04BF0408F45BC365C32091181621
:10D8D0003091191640911A1650911B1629833A83DC
:10D8E0004B835C832C153D054E055F0508F070C029
:10D8F00040911416509115166091161670911716D6
:10D900004A875B876C877D87D2960D911D912D91FB
:10D910003C91D597EE27419FF12D529FC001629F08
:10D92000900D619F800D911D429FF00D811D9E1FE6
:10D93000519FF00D811D9E1F609FF00D811D9E1F48
:10D94000509FF10D8E1F9E1FF6958E1F9E1F349FB8
:10D95000800D911D359F900D11248C0120E030E049
:10D9600080901F1690902016A0902116B09022163D
:10D97000FD01E65BFF4F081519052A053B05A0F4DC
:10D9800040815181628173814D835E836F8378878B
:10D99000801A910AA20AB30A84169506A606B7064B
:10D9A00038F44A015B0104C080809180A280B3807A
:10D9B0008EEB99E151E05D83FC0105911591259174
:10D9C0003491081519052A053B0508F468C374C38A
:10D9D00080911C168823D9F0D8964D915C91D997E7
:10D9E00060E070E000911D0210911E0220911F0264
:10D9F00030912002401751076207730741F01092DF
:10DA000021021092220210922302109224024091CD
:10DA1000190250911A0260911B0270911C0277FF4B
:10DA20005CC0AE5BBF4F8D919D910D90BC91A02DC0
:10DA30002EEB39E141E0F901C590D590E590F490E5
:10DA4000C816D906EA06FB0658F4B695A795979529
:10DA50008795440F2C5F3F4F69E12A3D360759F700
:10DA600040931E1680329105A105B10520F480E295
:10DA700090E0A0E0B0E08097A109B109811538E0FD
:10DA80009307A105B10508F4D3C344E0949F900126
:10DA9000112422543A4EF901329645915491EE27C1
:10DAA000859FB001849F610D7E1F06946E1F7E1FAF
:10DAB0001124CB01A0E0B0E0F9014591549160E060
:10DAC00070E0481B590B6A0B7B0B40931902509373
:10DAD0001A0260931B0270931C02809019029090AE
:10DAE0001A02A0901B02B0901C028091101D909110
:10DAF000111D892B09F0C2C10E943F689093111D2E
:10DB00008093101D892B09F4B9C1E091101DF0918B
:10DB1000111D808183FF3EC085899689A789B08DBC
:10DB200080931F1D9093201DA093211DB093221D53
:10DB3000818D928DA38DB48D8093231D9093241D90
:10DB4000A093251DB093261D858D968DA78DB0A120
:10DB50008093271D9093281DA093291DB0932A1D03
:10DB600081A192A1A3A1B4A180932B1D90932C1D00
:10DB7000A0932D1DB0932E1D9091911A8091921A11
:10DB8000981709F4B9CF8091921A8F5F8F708093A4
:10DB9000921AB2CFC588D688E788F08C81E0C1148C
:10DBA000D104E104F10409F480E0018D128D238D8C
:10DBB000348D011511052105310509F08260458D6F
:10DBC000568D678D70A1411551056105710509F0EC
:10DBD00084608093E415109214161092151610921A
:10DBE00016161092171610922316109224161092E1
:10DBF00025161092261685A196A1A7A1B0A58093FF
:10DC00002B1690932C16A0932D16B0932E168824C5
:10DC100099245401881A990AAA0ABB0A80921016FC
:10DC200090921116A0921216B092131680920C16B2
:10DC300090920D16A0920E16B0920F1680920816B2
:10DC400090920916A0920A16B0920B1680920416B2
:10DC500090920516A0920616B0920716CC0CDD1C09
:10DC6000EE1CFF1CC092F415D092F515E092F6154B
:10DC7000F092F715000F111F221F331F0093F815A4
:10DC80001093F9152093FA153093FB15440F551F87
:10DC9000661F771F4093FC155093FD156093FE158A
:10DCA0007093FF1541A152A163A174A1440F551FA8
:10DCB000661F771F4093001650930116609302165B
:10DCC00070930316880F991FAA1FBB1F8093F0152E
:10DCD0009093F115A093F215B093F31510922F16AF
:10DCE00010923016109231161092321682A593A51A
:10DCF000A4A5B5A58093271690932816A09329165E
:10DD0000B0932A1686A597A5A0A9B1A98093181645
:10DD100090931916A0931A16B0931B1681A58093A1
:10DD2000EF1520911802821721F01092EE15109233
:10DD3000ED1597A990931D16992309F144AD55ADA2
:10DD40005093EC154093EB1542AD53AD5093EA154B
:10DD50004093E915109221021092220210922302A0
:10DD60001092240240AD51AD60E070E040931D027E
:10DD700050931E0260931F027093200208C04092CD
:10DD80001D0250921E0260921F027092200296A9FC
:10DD900030917A08931302C0821731F090937A0879
:10DDA000809318020E94B4688091790881110E94C2
:10DDB0008AE54092190250921A0260921B027092F8
:10DDC0001C02E091101DF091111DEA5BFF4F808154
:10DDD0009181A281B38180931F1690932016A09306
:10DDE0002116B09322162EEB39E141E0F901C590DE
:10DDF000D590E590F490C816D906EA06FB0660F4C3
:10DE0000B695A79597958795440F2C5F3F4FEAED00
:10DE1000F9E1E217F30751F740931E16803291059E
:10DE2000A105B10520F480E290E0A0E0B0E0809789
:10DE3000A109B109811558E09507A105B10508F4BC
:10DE40001AC264E0969F9001112422543A4EF901BF
:10DE5000329645915491EE27859FB001849F610DC4
:10DE60007E1F06946E1F7E1F1124F90185909490E9
:10DE7000A12CB12C861A970AA108B10880923316FA
:10DE800090923416A0923516B09236160091331641
:10DE9000109134162091351630913616409121029A
:10DEA000509122026091230270912402F02E198376
:10DEB000F22FE32F401751076207730720F4F42E67
:10DEC0005983F62FE72F8F2D9981AF2FBE2F009703
:10DED000E1E0AE07B10520F08FEF9FEFA0E0B0E0EA
:10DEE000081B190B2A0B3B0B0093331610933416A7
:10DEF00020933516309336164F3FFFEF5F076F07BD
:10DF00007F0761F0481B590B6A0B7B0B4093210282
:10DF1000509322026093230270932402F89420917C
:10DF2000840030918500205F3F4F498541504987EB
:10DF3000442339F0280E391E2216330608F46DC921
:10DF400001C01901309289002092880078942D96A2
:10DF50000FB6F894DEBF0FBECDBFDF91CF911F91FA
:10DF60000F91FF90EF90DF90CF90BF90AF909F9078
:10DF70008F907F906F905F904F903F902F9008957B
:10DF8000F694E794D794C794220F0496E9E18A3D6A
:10DF90009E0709F08FCC20931E16F0E2CF16D10415
:10DFA000E104F10428F410E2C12ED12CE12CF12C73
:10DFB00030E2C31AD108E108F108C11488E0D8069C
:10DFC000E104F104F8F0E4E0DE9EC0011124825483
:10DFD0009A4EFC01329625913491FC2DEE27F39F49
:10DFE0008001F29F010D1E1F06940E1F1E1F11249B
:10DFF000FC0185909490A12CB12C801A910AA10863
:10E00000B10822C097018601369527951795079587
:10E01000F801EC7F9F0122543E4EF90185909490C7
:10E02000F901329685919491EC2DE770E89F90016B
:10E03000E99F300D1124F3E036952795FA95E1F725
:10E04000821A930AA12CB12C480D591D6A1D7B1D03
:10E05000409323165093241660932516709326162A
:10E0600090911D1680911C16992309F473C0882382
:10E0700009F43BCDD8968D919C91D997A0E0B0E062
:10E0800040911D0250911E0260911F02709120026A
:10E0900084179507A607B70709F05FC026CDB69489
:10E0A000A794979487942D81220F2D83049639E1AC
:10E0B0008A3D930709F080CC4D8140931E1650E2B3
:10E0C00085169104A104B10428F450E2852E912C08
:10E0D000A12CB12C60E2861A9108A108B108811424
:10E0E00078E09706A104B10408F440C0E4E09E9EE5
:10E0F000C001112482549A4EFC013296259134912C
:10E10000F82DEE27F39F8001F29F010D1E1F06944C
:10E110000E1F1E1F1124FC0185909490A12CB12C80
:10E12000801A910AA108B1084A855B856C857D85B6
:10E13000480D591D6A1D7B1D4093141650931516EA
:10E14000609316167093171680911D16811132C0B8
:10E1500080911C16882309F4C8CC109221021092D9
:10E1600022021092230210922402BFCC9501840156
:10E170003695279517950795F801EC7F9F01225456
:10E180003E4EF90185919491F901329605911491D1
:10E19000E82DE770E09F9001E19F300D112443E0EE
:10E1A000369527954A95E1F74C01821A930AA12CDE
:10E1B000B12CBACF49815A816B817C812D81420F6C
:10E1C000511D611D711D4C155D056E057F05C8F45F
:10E1D00080911C16882309F488CCD8964D915C91C7
:10E1E000D99760E070E000911D0210911E0220910D
:10E1F0001F0230912002401751076207730709F48C
:10E2000074CC1092210210922202109223021092DA
:10E210002402D8968D919C91D997A0E0B0E080938C
:10E220001D0290931E02A0931F02B09320025DCCAA
:10E23000AC01BD017695679557954795FA01EC7F3E
:10E240009F0122543E4EF90145915491F9013296B5
:10E25000659174918770869F9001879F300D11247E
:10E26000C901F3E096958795FA95E1F7481B590B9C
:10E2700060E070E02ACCAC01BD01769567955795BA
:10E280004795FA01EC7F9F0122543E4EF90185909B
:10E290009490F9013296459154918770849F900132
:10E2A000859F300D1124C901A3E096958795AA9505
:10E2B000E1F7881A990AA12CB12CE0CD80ED882EC7
:10E2C00087E0982EA12CB12C17CCCF930E943BC194
:10E2D000C0919F100E943BC1C13081F1C23059F4FE
:10E2E0000E94B4DD609397107093981080939910FA
:10E2F00090939A1002C00E94E8DD81E080939F1005
:10E300000E943368609393107093941080939510DB
:10E3100090939610C230A1F080916808909169089E
:10E32000019690936908809368081092A01010924B
:10E33000A1101092A2101092A31002C080E001C0A0
:10E3400081E0CF910895CF93DF9300D01F92CDB796
:10E35000DEB7809167088823A9F083E390E09C836F
:10E360008B831A8219829E012F5F3F4F40E150E05C
:10E3700068E678E0CE0103960E94C04D89EA96E0F7
:10E380000E94EE4F0F900F900F900F90DF91CF9162
:10E390000895CF92DF92EF92FF920F931F930E9406
:10E3A000EEC00E94EEC080919F108150823010F02C
:10E3B00080E05DC010929F100E94336860939B10B4
:10E3C00070939C1080939D1090939E1080916A088A
:10E3D00090916B08019690936B0880936A08C090A7
:10E3E000A010D090A110E090A210F090A3100E9475
:10E3F000B4DD6093A0107093A1108093A21090934D
:10E40000A31000916C0810916D0820916E08309156
:10E410006F080C191D092E093F09DC01CB01800F83
:10E42000911FA21FB31F80936C0890936D08A09357
:10E430006E08B0936F080E94B4DD009170081091CF
:10E440007108209172083091730806171707280782
:10E45000390750F40E94B4DD60937008709371081E
:10E4600080937208909373080E94A37181E01F91BA
:10E470000F91FF90EF90DF90CF900895CF93DF93AF
:10E4800000D01F921F92CDB7DEB781E0809367085E
:10E49000E8E6F8E080E1DF011D928A95E9F70E9445
:10E4A000A37186E18D8382E390E09C838B831A8243
:10E4B00019829E012F5F3F4F41E050E0BE016B5F2C
:10E4C0007F4FCE0103960E94C04D0F900F900F908A
:10E4D0000F900F90DF91CF9108952F923F924F921E
:10E4E0005F926F927F928F929F92AF92BF92CF92E4
:10E4F000DF92EF92FF920F931F93CF93DF93CDB7ED
:10E50000DEB7CA59D1090FB6F894DEBF0FBECDBF32
:10E510004B015A011901E096EFAEE097C057DF4F6B
:10E52000D982C882C059D040DC012D913D914D91D6
:10E530005C91E8962CAF3DAF4EAF5FAFE89720916E
:10E54000AC163091AD164091AE165091AF16E896CC
:10E550006CAD7DAD8EAD9FADE8970F94BA0D0F9465
:10E56000C5162B013C0125966CAF7DAF8EAF9FAFDA
:10E570002597D4012D913D914D915C91E4962CAF5E
:10E580003DAF4EAF5FAFE4972091B0163091B1161A
:10E590004091B2165091B316E4966CAD7DAD8EAD40
:10E5A0009FADE4970F94BA0D0F94C516A7966CAF64
:10E5B0007DAF8EAF9FAFA79729966CAF7DAF8EAF23
:10E5C0009FAF2997D5012D913D914D915C91AF96CB
:10E5D0002CAF3DAF4EAF5FAFAF972091B4163091E7
:10E5E000B5164091B6165091B716AF966CAD7DAD8D
:10E5F0008EAD9FADAF970F94BA0D0F94C5166B01FA
:10E600007C012D966CAF7DAF8EAF9FAF2D97D10162
:10E610002D913D914D915C91AB962CAF3DAF4EAF9E
:10E620005FAFAB972091B8163091B9164091BA16EA
:10E630005091BB16AB966CAD7DAD8EAD9FADAB97DB
:10E640000F94BA0D0F94C5164B015C0161966CAF27
:10E650007DAF8EAF9FAF6197E8962CAD3DAD4EADCF
:10E660005FADE89765962CAF3DAF4EAF5FAF659756
:10E67000E4968CAD9DADAEADBFADE49769968CAF21
:10E680009DAFAEAFBFAF6997AF962CAD3DAD4EAD70
:10E690005FADAF976D962CAF3DAF4EAF5FAF6D974F
:10E6A000AB968CAD9DADAEADBFADAB97A1968CAF2B
:10E6B0009DAFAEAFBFAFA1978091E91683FF16C0A3
:10E6C0008092C31A9092C41AA092C51AB092C61A28
:10E6D000AB962CAD3DAD4EAD5FADAB972093B31A6D
:10E6E0003093B41A4093B51A5093B61A8091961687
:10E6F00090919716892B09F0A3C3D801BC91ED9690
:10E70000BFAFED97F801F181C058DF4FF883C058D3
:10E71000D040D8011296BC91CC57DF4FB883C45873
:10E72000D040F801F381C857DF4FF883C858D04074
:10E730008091911A9091921A891B8F708F3021F4D9
:10E7400080E00E94AA50F4CF2091911AC856DF4F62
:10E750002883C859D0408091911A282E312C80915D
:10E76000B71A9091B81AA091B91AB091BA1A481A6A
:10E77000590A6A0A7B0A8091BB1A9091BC1AA0912F
:10E78000BD1AB091BE1AA7962CAD3DAD4EAD5FAD92
:10E79000A797281B390B4A0B5B0BA7962CAF3DAFF5
:10E7A0004EAF5FAFA7978091BF1A9091C01AA0910A
:10E7B000C11AB091C21AA7019601281B390B4A0B46
:10E7C0005B0BE4962CAF3DAF4EAF5FAFE49780910B
:10E7D000C31A9091C41AA091C51AB091C61AA50186
:10E7E0009401281B390B4A0B5B0BE8962CAF3DAF0D
:10E7F0004EAF5FAFE897232B242B252B09F492C053
:10E800008091E816811133C060913A0870913B08FD
:10E8100080913C0890913D080F94C41520915D02B1
:10E8200030915E026217730714F58092C31A9092BA
:10E83000C41AA092C51AB092C61AAB968CAD9DAD03
:10E84000AEADBFADAB978093B31A9093B41AA093BB
:10E85000B51AB093B61A0E94BC4D8DEF99E10E9493
:10E860001F4DE8961CAE1DAE1EAE1FAEE897E0969B
:10E87000AFADE09794E0A99F800111240F5C1D4F7C
:10E88000E8966CAD7DAD8EAD9FADE8970F945B0DB6
:10E89000F80120813181428153810F94BA0D6B01BF
:10E8A0007C0120E030E0A9010F94B81687FF04C076
:10E8B000F7FAF094F7F8F09420E030E04AEF53E4F0
:10E8C0006091B8167091B9168091BA169091BB16E6
:10E8D0000F94BA0DA70196010F94540D87FF22C023
:10E8E0008092C31A9092C41AA092C51AB092C61A06
:10E8F000AB962CAD3DAD4EAD5FADAB972093B31A4B
:10E900003093B41A4093B51A5093B61A0E94BC4D76
:10E910008EED99E10E941F4DE8961CAE1DAE1EAE15
:10E920001FAEE897D301C2018827B7FD83959927C9
:10E93000AA27BB27B82EA7962CAD3DAD4EAD5FAD37
:10E94000A79757FF03C0382F3260B32EE4968CADE3
:10E950009DADAEADBFADE497B7FF03C09B2D9460F6
:10E96000B92EE8962CAD3DAD4EAD5FADE89757FFA3
:10E9700003C03B2D3860B32EE0965FADE09744E0D6
:10E98000549F800111240F5C1D4FE8966CAD7DAD46
:10E990008EAD9FADE8970F945B0DD8012D913D9101
:10E9A0004D915C910F94BA0D6B017C0120E030E039
:10E9B000A9010F94B81687FF04C0C701B60190588B
:10E9C00002C0C701B60120E030E040E05FE30F94F1
:10E9D00058140F94CB15AF966CAF7DAF8EAF9FAF31
:10E9E000AF9784E5829DF001839DF00D1124EC55D5
:10E9F000FF4E1082B6AA5301420177FE07C0882459
:10EA00009924540184189508A608B70884E5829DC6
:10EA1000F001839DF00D1124EC55FF4E858A968AF6
:10EA2000A78AB08EA7962CAD3DAD4EAD5FADA79732
:10EA3000AB962CAF3DAF4EAF5FAFAB9757FF0DC05E
:10EA400050954095309521953F4F4F4F5F4FAB9676
:10EA50002CAF3DAF4EAF5FAFAB9784E5829DF00129
:10EA6000839DF00D1124EC55FF4EAB968CAD9DAD02
:10EA7000AEADBFADAB97818F928FA38FB48FE4966D
:10EA80002CAD3DAD4EAD5FADE497EC962CAF3DAFF8
:10EA90004EAF5FAFEC9757FF0DC050954095309546
:10EAA00021953F4F4F4F5F4FEC962CAF3DAF4EAF90
:10EAB0005FAFEC9784E5829DF001839DF00D1124FA
:10EAC000EC55FF4EEC968CAD9DADAEADBFADEC9769
:10EAD000858F968FA78FB0A3C301B2010F945B0DF2
:10EAE00020915B1630915C1640915D1650915E1638
:10EAF0000F94BA0DC457DF4F688379838A839B8351
:10EB0000CC58D04069AB7AAB8BAB9CABA7966CADC5
:10EB10007DAD8EAD9FADA7970F945B0D20915F16D5
:10EB20003091601640916116509162160F94BA0DA3
:10EB30002B013C016DAB7EAB8FAB98AFE4966CAD17
:10EB40007DAD8EAD9FADE4970F945B0D2091631664
:10EB50003091641640916516509166160F94BA0D67
:10EB6000A7966CAF7DAF8EAF9FAFA79769AF7AAF17
:10EB70008BAF9CAF20916716309168164091691653
:10EB800050916A16C701B6010F94BA0D6B017C0152
:10EB900021966CAF7DAF8EAF9FAF219796E089161F
:10EBA0009104A104B1041CF5AB962CAD3DAD4EAD66
:10EBB0005FADAB972630310541055105C4F4EC96A5
:10EBC0008CAD9DADAEADBFADEC970697A105B1057F
:10EBD00074F420E030E0A901C701B6010F94B81623
:10EBE00087FF18C0F7FAF094F7F8F09413C0C057F5
:10EBF000DF4FA881B981C059D040CD90DD90ED9014
:10EC0000FC9020E030E0A901C701B6010F94540D3B
:10EC1000882369F084E5829DF001839DF00D112425
:10EC2000EC55FF4EC586D686E786F08A3AC0C457B3
:10EC3000DF4F288139814A815B81CC58D040CA019D
:10EC4000B9010F94BA0D6B017C01A3019201C301BC
:10EC5000B2010F94BA0D9B01AC01C701B6010F942C
:10EC600058146B017C01A7962CAD3DAD4EAD5FAD48
:10EC7000A797CA01B9010F94BA0D9B01AC01C70156
:10EC8000B6010F9458140F94061724E5229DF00145
:10EC9000239DF00D1124EC55FF4E658776878787FD
:10ECA000908B84E5829DF001839DF00D1124EC553D
:10ECB000FF4EAF962CAD3DAD4EAD5FADAF9721A3EE
:10ECC00032A343A354A3582D492D3A2D2B2DAB9697
:10ECD0008CAD9DADAEADBFADAB9788169906AA06BB
:10ECE000BB0660F4A8965FADA897A9964FADA9970B
:10ECF000AA963FADAA97AB962FADAB97852F942FD1
:10ED0000A32FB22FEC962CAD3DAD4EAD5FADEC9781
:10ED100082179307A407B50710F4DA01C901AF966B
:10ED20002CAD3DAD4EAD5FADAF9782179307A407F5
:10ED3000B50710F4DA01C90124E5229DF001239DF5
:10ED4000F00D1124EC55FF4E85A396A3A7A3B0A701
:10ED50000697A105B10510F40C944484DF01AE5A66
:10ED6000BF4F8091E6168C9311968091E7168C9395
:10ED7000E0963FADE09731A789288A288B2809F0D3
:10ED80005F9884E5829DF001839DF00D1124EC5580
:10ED9000FF4E818D928DA38DB48D892B8A2B8B2B69
:10EDA00009F08A9884E5829DF001839DF00D11247D
:10EDB000EC55FF4E858D968DA78DB0A1892B8A2BA2
:10EDC0008B2B29F080910801817080930601AF960A
:10EDD0008CAD9DADAEADBFADAF97892B8A2B8B2B84
:10EDE00091F180917B16882319F0815080937B16D6
:10EDF00080917C16882399F0815080937C16E09650
:10EE00009FADE097992319F0913081F025C08111D1
:10EE100001C0479A129880E280937B161DC0E0964D
:10EE2000FFADE097FF23A9F3F130B1F480917B1699
:10EE3000811101C0129A479880E280937C160CC021
:10EE400080E00C94CD84E090DC16F090DD1600910B
:10EE5000DE161091DF1608C0E090D816F090D91693
:10EE60000091DA161091DB169701A801ED966FADAF
:10EE7000ED97C058DF4F7881C058D040CC57DF4F56
:10EE80008881C458D040C857DF4F9881C858D040B7
:10EE90000F94540D87FF12C0ED96EFAEED97C0585A
:10EEA000DF4FF882C058D040CC57DF4F0883C4589A
:10EEB000D040C857DF4F1883C858D04084E5829DA2
:10EEC000F001839DF00D1124EC55FF4E45845684CE
:10EED00067847088A301920160E070E080E89FE39E
:10EEE0000F945215EC966CAF7DAF8EAF9FAFEC9741
:10EEF000ED962FADED97C058DF4F3881C058D04008
:10EF0000CC57DF4F4881C458D040C857DF4F588195
:10EF1000C858D0400F94BA0D4B015C018091911AF2
:10EF200090918F1A891B8F70C857DF4F8883C858FC
:10EF3000D040A501940160E074E284E799E40F9465
:10EF400052150F94C5166B017C01C857DF4F88819D
:10EF5000C858D04082508630D0F58091A816909144
:10EF6000A916A091AA16B091AB16C816D906EA0642
:10EF7000FB0668F58C199D09AE09BF09BC01CD01DE
:10EF8000660F771F881F991FC857DF4FA881C85881
:10EF9000D0400A2F10E020E030E0A90198010F9442
:10EFA000AA13CA01B9010F94590D0F94C5166C0D1F
:10EFB0007D1D8E1D9F1D0F94590D9B01AC0160E0BE
:10EFC00074E284E799E40F9452154B015C01A501AA
:10EFD0009401C301B2010F94BA0D9B01AC010F94CF
:10EFE000BA0DC457DF4F688379838A839B83CC58DB
:10EFF000D04084E5829D8001839D100D11240C5525
:10F000001F4EC457DF4F288139814A815B81CC581C
:10F01000D040D80111962D933D934D935C93149756
:10F0200095962D913D914D915C919897C458DF4FE5
:10F03000288339834A835B83CC57D040CA01B90106
:10F040000F94590DC058DF4F688379838A839B835F
:10F05000C058D0409B01AC01C501B4010F94BA0D5A
:10F060000F9436150F94CB15C057DF4F6883798303
:10F070008A839B83C059D040F801EE5BFF4F6083C9
:10F080007183828393838E010F5C1F4FFE01B196C3
:10F09000CC57DF4FF983E883C458D0402CEB36E1DE
:10F0A000CA56DF4F39832883C659D040A801405F34
:10F0B0005F4FC756DF4F59834883C959D040CC565C
:10F0C000DF4FF983E883C459D040A4961FAEA497BC
:10F0D000A8961FAEA89750E8E0965FAFE0978FE341
:10F0E000E1968FAFE197D8012D913D914D915D91C2
:10F0F0008D01C501B4010F94BA0D6B017C01CC5692
:10F10000DF4FE881F981C459D040619371938193B5
:10F110009193CC56DF4FF983E883C459D04020E067
:10F1200030E0A9010F94B81687FF04C0F7FAF094F5
:10F13000F7F8F094CA56DF4FA881B981C659D0407C
:10F140004D905D906D907D90CA56DF4FB983A88336
:10F15000C659D040A7019601C301B2010F94540DC6
:10F1600087FF24C0A7019601C301B2010F94521575
:10F170007B016C01A4962FADA497A8963FADA897EC
:10F18000E0964FADE097E1965FADE1970F94540D97
:10F1900087FF0CC0A496EFAEA497A896FFAEA897E1
:10F1A000E096CFAEE097E196DFAEE197C756DF4F2E
:10F1B000E881F981C959D040E017F10709F093CFF0
:10F1C00020E030E040E85FE3A4966FADA497A896F6
:10F1D0007FADA897E0968FADE097E1969FADE19760
:10F1E0000F94540D87FF84C08E010F5C1F4FA496AF
:10F1F0002FADA497A8963FADA897E0964FADE097A6
:10F20000E1965FADE197CC57DF4FA881B981C45833
:10F21000D0406D917D918D919C910F94BA0DCC57FA
:10F22000DF4FE881F981C458D04061937193819395
:10F230009193CC57DF4FF983E883C458D0400E1721
:10F240001F07A9F624E5229DC001239D900D1124DE
:10F250009C012C553F4E790189010E5B1F4FC05711
:10F26000DF4F688179818A819B81C059D0400F949A
:10F27000590DA4962FADA497A8963FADA897E096F8
:10F280004FADE097E1965FADE1970F94BA0D0F9403
:10F29000CB15D8016D937D938D939C931397A49672
:10F2A0002FADA497A8963FADA897E0964FADE097F5
:10F2B000E1965FADE197A4966FADA497A8967FAD58
:10F2C000A897E0968FADE097E1969FADE1970F94F8
:10F2D000BA0DC457DF4F288139814A815B81CC58F0
:10F2E000D0400F94BA0DF7016183728383839483B6
:10F2F000C058DF4F288139814A815B81C058D04096
:10F30000EC966CAD7DAD8EAD9FADEC970F94BA0DC4
:10F31000A7966CAF7DAF8EAF9FAFA79784E5829D18
:10F320008001839D100D11240C551F4ED801559658
:10F330008D909D90AD90BC90589781149104A1043C
:10F34000B10469F559968D919D910D90BC91A02DB8
:10F35000892B8A2B8B2B19F5F801858D968DA78D1E
:10F36000B0A1892B8A2B8B2BD1F42091D016309110
:10F37000D1164091D2165091D316A7966CAD7DADA3
:10F380008EAD9FADA7970F94BA0D0F9436150F94BD
:10F39000CB152B013C01D801D7961C9247C3AF96E1
:10F3A0002CAD3DAD4EAD5FADAF97232B242B252B60
:10F3B00049F02091CC163091CD164091CE16509147
:10F3C000CF1608C02091D4163091D5164091D6168C
:10F3D0005091D716A7966CAD7DAD8EAD9FADA7971A
:10F3E0000F94BA0D0F9436150F94CB152B013C01D9
:10F3F000AF968CAD9DADAEADBFADAF97892B8A2BCF
:10F400008B2BF9F0E091F70A94E0E99FF0011124C9
:10F41000ED5AF94E20E030E0A901608171818281CE
:10F4200093810F94540D882361F081E0E8962CAD10
:10F430003DAD4EAD5FADE8971216130614061506E6
:10F440000CF080E094E5929D8001939D100D1124B5
:10F450000C551F4ED801D7968C93882309F4D0C041
:10F460002091A71A3091A81A4091A91A5091AA1A6E
:10F4700065966CAD7DAD8EAD9FAD65970F945714BD
:10F48000AB966CAF7DAF8EAF9FAFAB972091AB1AB1
:10F490003091AC1A4091AD1A5091AE1A69966CAD8C
:10F4A0007DAD8EAD9FAD69970F945714E8966CAF04
:10F4B0007DAF8EAF9FAFE8972091AF1A3091B01A11
:10F4C0004091B11A5091B21A6D966CAD7DAD8EAD72
:10F4D0009FAD6D970F9457146B017C01AB962CADCB
:10F4E0003DAD4EAD5FADAB97CA01B9010F94BA0DFA
:10F4F000AB966CAF7DAF8EAF9FAFAB97E8962CAD60
:10F500003DAD4EAD5FADE897CA01B9010F94BA0D9C
:10F510009B01AC01AB966CAD7DAD8EAD9FADAB9755
:10F520000F945814AB966CAF7DAF8EAF9FAFAB9777
:10F53000A7019601C701B6010F94BA0D9B01AC015A
:10F54000AB966CAD7DAD8EAD9FADAB970F9458145F
:10F550000F9406176B017C012091B31A3091B41AF5
:10F560004091B51A5091B61AA1966CAD7DAD8EAD95
:10F570009FADA1970F945714A70196010F945215B0
:10F580006B017C01F801FE96608371838283938313
:10F5900020E030E040E450E40F94B81618161CF454
:10F5A000F80117AA2DC0E091F70A24E0E29FF001CC
:10F5B0001124ED5AF94E2081318142815381C701D6
:10F5C000B6010F94BA0D9B01AC0160914F1670917A
:10F5D000501680915116909152160F945215A7967D
:10F5E0002CAD3DAD4EAD5FADA7970F94BA0D0F9406
:10F5F000CB15641575058605970510F42B013C01A4
:10F6000080914B1690914C16A0914D16B0914E16CC
:10F61000C458DF4F288139814A815B81CC57D04063
:10F6200082179307A407B50708F4DCC0811491047E
:10F63000A104B10411F160913B1670913C168091C8
:10F640003D1690913E166415750586059705A8F43C
:10F650000F949A136B017C01A5019401C301B201BF
:10F660000F949A13C616D706E806F90630F4C701B8
:10F67000B6010F94AA1329013A0184E5829DF00195
:10F68000839DF00D1124EC55FF4EC18CD28CE38C80
:10F69000F48CC114D104E104F10451F160913F16DE
:10F6A000709140168091411690914216641575052F
:10F6B00086059705E8F4C458DF4F288139814A81CF
:10F6C0005B81CC57D0400F949A134B015C01A7018A
:10F6D0009601C301B2010F949A1386169706A806E5
:10F6E000B90630F4C501B4010F94AA1329013A01F7
:10F6F00084E5829DF001839DF00D1124EC55FF4EB1
:10F70000C58CD68CE78CF0A0C114D104E104F104BF
:10F7100051F1609143167091441680914516909175
:10F7200046166415750586059705E8F4C458DF4F3D
:10F73000288139814A815B81CC57D0400F949A133C
:10F740004B015C01A7019601C301B2010F949A130A
:10F7500086169706A806B90630F4C501B4010F94C1
:10F76000AA1329013A0184E5829DF001839DF00DE1
:10F770001124EC55FF4EC1A0D2A0E3A0F4A0C11407
:10F78000D104E104F10409F451C16091471670916C
:10F7900048168091491690914A166415750586059C
:10F7A000970508F043C1C458DF4F288139814A8149
:10F7B0005B81CC57D0400F949A134B015C01A70199
:10F7C0009601C301B2010F949A1386169706A806F4
:10F7D000B90608F02BC1C501B4010F94AA13290181
:10F7E0003A0124C181149104A104B104D9F16091BA
:10F7F0003B1670913C1680913D1690913E16641513
:10F8000075058605970570F50F94590DC058DF4FA3
:10F81000288139814A815B81C058D0400F94BA0D4C
:10F820006B017C01C501B4010F94590D4B015C01C2
:10F83000C301B2010F94590DA50194010F94BA0DA3
:10F840009B01AC01C701B6010F94540D87FF0AC09C
:10F85000A5019401C701B6010F9452150F94CB1561
:10F860002B013C0184E5829DF001839DF00D112464
:10F87000EC55FF4E818C928CA38CB48C8114910436
:10F88000A104B104D9F160913F16709140168091A6
:10F89000411690914216641575058605970570F519
:10F8A0000F94590DC058DF4F288139814A815B81FF
:10F8B000C058D0400F94BA0D6B017C01C501B40152
:10F8C0000F94590D4B015C01C301B2010F94590D06
:10F8D000A50194010F94BA0D9B01AC01C701B601BB
:10F8E0000F94540D87FF0AC0A5019401C701B6010A
:10F8F0000F9452150F94CB152B013C0184E5829D8A
:10F90000F001839DF00D1124EC55FF4E858C968CF3
:10F91000A78CB0A081149104A104B104D9F1609125
:10F9200043167091441680914516909146166415C1
:10F9300075058605970570F50F94590DC058DF4F72
:10F94000288139814A815B81C058D0400F94BA0D1B
:10F950006B017C01C501B4010F94590D4B015C0191
:10F96000C301B2010F94590DA50194010F94BA0D72
:10F970009B01AC01C701B6010F94540D87FF0AC06B
:10F98000A5019401C701B6010F9452150F94CB1530
:10F990002B013C0184E5829DF001839DF00D112433
:10F9A000EC55FF4E81A092A0A3A0B4A081149104B5
:10F9B000A104B104D9F16091471670914816809165
:10F9C000491690914A16641575058605970570F5D8
:10F9D0000F94590DC058DF4F288139814A815B81CE
:10F9E000C058D0400F94BA0D6B017C01C501B40121
:10F9F0000F94590D4B015C01C301B2010F94590DD5
:10FA0000A50194010F94BA0D9B01AC01C701B60189
:10FA10000F94540D87FF0AC0A5019401C701B601D8
:10FA20000F9452150F94CB152B013C0184E5829D58
:10FA30008001839D100D11240C551F4EF801E25BCF
:10FA4000FF4F4082518262827382C301B2010F94E0
:10FA5000590D6B017C01A7962CAD3DAD4EAD5FAD50
:10FA6000A7970F945215E4966CAF7DAF8EAF9FAF02
:10FA7000E497D80151966D937D938D939C93549701
:10FA80002DEB37E346E051E4C701B6010F94BA0D00
:10FA90000F94CB15F80162AB73AB84AB95AB87A920
:10FAA0008823A9F1E091F70A24E0E29FF0011124F4
:10FAB000ED5AF94ED801DE962D913D914D915C9114
:10FAC00060817181828193810F94BA0DE4962CAD8F
:10FAD0003DAD4EAD5FADE4970F94BA0D2091B816D1
:10FAE0003091B9164091BA165091BB160F94BA0DC9
:10FAF0009B01AC0160E074E284EF99E40F9452152D
:10FB00000F94CB15D801D9967C936E93D89729A9D9
:10FB10003AA94BA95CA9EC966CAD7DAD8EAD9FADBD
:10FB2000EC970F94BA0DAF966CAF7DAF8EAF9FAFD1
:10FB3000AF97698B7A8B8B8B9C8B2DA93EA94FA994
:10FB400058ADEC966CAD7DAD8EAD9FADEC970F943E
:10FB5000BA0D2B013C016D8B7E8B8F8B988F29AD5D
:10FB60003AAD4BAD5CADEC966CAD7DAD8EAD9FAD61
:10FB7000EC970F94BA0D4B015C01698F7A8F8B8FD4
:10FB80009C8F21962CAD3DAD4EAD5FAD2197EC968F
:10FB90006CAD7DAD8EAD9FADEC970F94BA0DEC962C
:10FBA0006CAF7DAF8EAF9FAFEC976D8F7E8F8F8FD9
:10FBB00098A3C857DF4FB881C858D040BB2309F479
:10FBC000DBC2E091931AA496EFAFA497F091941A38
:10FBD000A896FFAFA8972091951AE5962FAFE597C5
:10FBE0003091961AE0963FAFE0972DEB37E346E869
:10FBF00055E3BF01E5968FADE597E0969FADE097A1
:10FC00000F94540D87FDB8C280916B1690916C16BD
:10FC1000A0916D16B0916E16C458DF4F88839983FA
:10FC2000AA83BB83CC57D04020916F1630917016B9
:10FC30004091711650917216C058DF4F2883398356
:10FC40004A835B83C058D04080917316909174169C
:10FC5000A0917516B0917616CC57DF4F88839983A3
:10FC6000AA83BB83C458D040209177163091781670
:10FC70004091791650917A16C857DF4F28833983FF
:10FC80004A835B83C858D040C458DF4F688179816C
:10FC90008A819B81CC57D0409058AF962CAD3DAD1A
:10FCA0004EAD5FADAF970F94BA0D6B017C01C0589C
:10FCB000DF4F288139814A815B81C058D040C30120
:10FCC000B2010F94BA0D9B01AC01C701B6010F94AC
:10FCD00057146B017C01CC57DF4F288139814A8151
:10FCE0005B81C458D040C501B4010F94BA0D9B018B
:10FCF000AC01C701B6010F9457146B017C01C857C2
:10FD0000DF4F288139814A815B81C858D040EC9609
:10FD10006CAD7DAD8EAD9FADEC970F94BA0D9B0190
:10FD2000AC01C701B6010F9457146B017C012FEE93
:10FD30003FEF4FE75FE30F94B81618160CF4BEC1FF
:10FD40002FEE3FEF4FE75FEBC701B6010F94540D65
:10FD500087FF08C03FEEC32EDD24DA943FE7E32E91
:10FD60003FEBF32EC458DF4F288139814A815B81F4
:10FD7000CC57D040AF966CAD7DAD8EAD9FADAF97FB
:10FD80000F94571469837A838B839C83C058DF4F09
:10FD9000288139814A815B81C058D040C301B201BA
:10FDA0000F9457146D837E838F839887CC57DF4FD2
:10FDB000288139814A815B81C458D040C501B40192
:10FDC0000F94571469877A878B879C87C857DF4FB2
:10FDD000288139814A815B81C858D040EC966CAD4E
:10FDE0007DAD8EAD9FADEC970F9457146D877E87D8
:10FDF0008F87988BAE014F5F5F4FAD965FAF4EAF71
:10FE0000AD97CE014196A3969FAF8EAFA3978A017F
:10FE1000812C912C5401D8014D905D906D907D9076
:10FE20008D0120E030E0A901C301B2010F94540D0F
:10FE3000882371F0A3019201C301B2010F94BA0D9E
:10FE40009B01AC01C501B4010F9458144B015C0136
:10FE5000A396EEADFFADA397E017F107E1F6C5015C
:10FE6000B4010F9406179B01AC0160E070E080E8DC
:10FE70009FE30F9452154B015C01AD960EAD1FAD83
:10FE8000AD97A5019401D8016D917D918D919C91C3
:10FE90000F94BA0DF80161937193819391938F013F
:10FEA000A3962EAD3FADA3972E173F0751F708E954
:10FEB00016E1E1965FACE197E2966FACE297E396CC
:10FEC0007FACE397E4964FACE497AD96AEADBFAD93
:10FED000AD978D909D90AD90BD90AD96BFAFAEAFFC
:10FEE000AD9720E030E0A901C501B4010F94540D95
:10FEF000882331F1F80160817181828193810F94AF
:10FF0000590DA50194010F9452154B015C0120E09D
:10FF100030E0A9010F94B81687FF04C0B7FAB09477
:10FF2000B7F8B094252D362D472D542DC501B401B9
:10FF30000F94540D87FF04C0582C692C7A2C4B2C3D
:10FF40000C5F1F4FA3962EAD3FADA397AD964EAD60
:10FF50005FADAD972417350709F0B7CFA70196011C
:10FF600060E070E080E89FE30F94571420E030E0F9
:10FF700040E05FE30F94BA0D0F9406174B015C014C
:10FF800020913716309138164091391650913A1613
:10FF9000652D762D872D942D0F94BA0DA501940112
:10FFA0000F94BA0DAF966CAF7DAF8EAF9FAFAF978A
:10FFB000A501940160E070E080E89FE30F9457147E
:10FFC0009B01AC01AF966CAD7DAD8EAD9FADAF9793
:10FFD0000F945215AC966FAFAC97E9967FAFE99747
:10FFE0008C0184E5829DF001839DF00D1124EC5578
:10FFF000FF4E85849684A784B08820E030E040E8F6
:020000021000EC
:100000005FE3C501B4010F94540D87FF61C0A701E0
:100010009601C701B6010F94BA0D23EC38EB42E309
:100020005FEB0F94BA0D23EF36E64FE55FE30F94D5
:100030005714A70196010F94BA0D2BED3FE049EC40
:100040005FE30F9458142CEE31E548E35EE30F9420
:1000500057146B017C0124EE3BEC46E150E40F9415
:10006000B8161816ACF5A70196016BED7FE089E490
:1000700090E40F9457149B01AC01C501B4010F9497
:100080005215252D362D472D542D0F94BA0D6B0189
:100090007C019B01AC01AC966FADAC97E9967FAD4E
:1000A000E997C8010F94B816181694F4AC96CFAE21
:1000B000AC97E996DFAEE99787010AC05BE0AC96A2
:1000C0005FAFAC9787EDE9968FAFE99703E21BE34B
:1000D00084E5829DF001839DF00D1124EC55FF4EC7
:1000E000C180D280E380F4809601A701A4966FAD11
:1000F000A497A8967FADA897E5968FADE597E09673
:100100009FADE0970F94B816181664F4A496CFAE7E
:10011000A497A896DFAEA897E596EFAEE597E09690
:10012000FFAEE097AC962FADAC97E9963FADE9975F
:10013000A801A4966FADA497A8967FADA897E59661
:100140008FADE597E0969FADE0970F94B81618161F
:10015000FCF4AC969FADAC97A4969FAFA497E9969C
:10016000AFADE997A896AFAFA897E5960FAFE59723
:10017000E0961FAFE0970CC0A4961FAEA497A89678
:100180001FAEA897E5961FAEE597E0961FAEE097E5
:1001900080E1FE017196ABE6B6E101900D928A9581
:1001A000E1F784E5829D8001839D100D11240C559B
:1001B0001F4EA4968FADA497A8969FADA897E596DD
:1001C000AFADE597E096BFADE097F80181879287E4
:1001D000A387B487E4966CAD7DAD8EAD9FADE497FB
:1001E00090589B01AC010F945814D8011D962D9185
:1001F0003D914D915C9150970F94BA0D9B01AC01CC
:100200006BE077ED83E29BE30F9457142BE0C22E53
:1002100027EDD22E23E2E22E2BE3F22EF801C58247
:10022000D682E782F086B080C180D280E380F480FD
:10023000A70196010F94B81687FD02C083E001C0A4
:1002400081E08B2994E5929DF001939DF00D11249E
:10025000EC55FF4E808380E1FE01B196A7E9BAE13B
:1002600001900D928A95E1F7C092931AD092941A58
:10027000E092951AF092961A80E1FE01EF5BFF4F33
:10028000A7EBBAE101900D928A95E1F780E1FE01BA
:10029000EF5AFF4FA7EABAE101900D928A95E1F774
:1002A0009091911A8091921A981303C084E68093DA
:1002B0008E1AC856DF4F8881C859D0408F5F8F7023
:1002C0008093911A8091911A9091901A81508F7019
:1002D000891709F4B6C0F090911A8FEF8F0D8F70C7
:1002E000A4968FAFA497B090901A8091911AB816E7
:1002F00009F476C0C12CD12CA496FFADA497FB15B0
:1003000009F46EC06F2E712C24E5269D8001279D77
:10031000100D11240C551F4ED8018C9183FD3DC04A
:10032000AC960FAFAC97E9961FAFE9970115110591
:10033000D1F11996BC91A896BFAFA897F801F285A4
:10034000E596FFAFE597D8011B96BC91E096BFAF4D
:10035000E097F801F485E196FFAFE197D801159693
:100360002D903D904D905C901897A2019101A89618
:100370006FADA897E5967FADE597E0968FADE097D6
:100380009F2F0F94540D8111F0C1C114D10459F065
:10039000F601808180FDE9C106C0AC96CFAEAC9776
:1003A000E996DFAEE997A4968FADA49781508F7040
:1003B000A4968FAFA4978091901A8B1107C0AC962A
:1003C000CFACAC97E996DFACE99796CFA496FFAD9A
:1003D000A497FB1529F081E08B0D8F70B82EEBCF21
:1003E0002091901AA4962FAFA497C12CD12C809164
:1003F000911AA4963FADA497831719F1832E912CDF
:1004000044E5489D8001499D100D11240C551F4E57
:10041000D8018C9183FD0AC05801C114D10439F070
:10042000C6010E9401FA811102C035C25601A4968C
:100430008FADA4978F5F8F70A4968FAFA49765013F
:10044000D6CF4091921AA4964FAFA4975091911A8B
:10045000A8965FAFA89724E5A4968FADA497A89619
:100460009FADA897891779F0892F81508F70289FA9
:10047000F0011124EC55FF4E908193FF04C0A89623
:100480008FAFA897E9CF812C912CA12CB12CE596A8
:100490001FAEE597E0961FAEE097E1961FAEE1979D
:1004A000AC961FAEAC97212C312C00E010E0A89642
:1004B000AFADA897A496BFADA497AB1709F4D4C06D
:1004C000E4E5EB9FC00111249C012C553F4E19011E
:1004D000D9018C9183FD19C015966D917D918D91F7
:1004E0009C9118970F940617F62EE72ED82EC92E3A
:1004F0000115110509F49EC0F801808180FD12C02C
:10050000D1018C9180FD0EC095C0E596FFACE597BA
:10051000E096EFACE097E196DFACE197AC96CFAC1C
:10052000AC978DC0F801808181608083C8010E94F2
:1005300001FA81117BC0F80161817281838194810C
:100540000F9406172B013C019B01AC0160E070E0A9
:1005500080E89FE30F9452154B015C019B01AC01B5
:100560006F2D7E2D8D2D9C2D0F94BA0D69837A836E
:100570008B839C83E5962FADE597E0963FADE097A2
:10058000E1964FADE197AC965FADAC97C501B40174
:100590000F94BA0D698B7A8B8B8B9C8BAE014F5F5E
:1005A0005F4FBE016F5E7F4FC8010E94D5D6D80154
:1005B000D7968C918823D1F1E091F70AB4E0EB9FB4
:1005C000F0011124ED5AF94ED801DE962D913D919E
:1005D0004D915C9160817181828193810F94BA0DFC
:1005E0002091B8163091B9164091BA165091BB16A9
:1005F0000F94BA0D4B015C019B01AC01C301B20128
:100600000F94BA0D0F94CB15F80173AF62AFA5012B
:1006100094016F2D7E2D8D2D9C2D0F94BA0D0F946E
:10062000CB15D801DD967C936E93DC97F801808121
:100630008E7F80838F2C9E2CAD2CBC2C8101A496A8
:100640008FADA4978F5F8F70A4968FAFA497E59618
:10065000FFAEE597E096EFAEE097E196DFAEE1976B
:10066000AC96CFAEAC9723CF2114310409F40CC162
:10067000D1018C9181608C93C8010E9401FA811193
:100680006FC0F10161817281838194810F9406179B
:100690006B017C019B01AC0160E070E080E89FE3AE
:1006A0000F9452152B013C012DEC3CEC4CE45DE326
:1006B0000F94BA0D69837A838B839C839401A5017F
:1006C000C301B2010F94BA0D698B7A8B8B8B9C8B13
:1006D000AE014F5F5F4FBE016F5E7F4FC1010E9451
:1006E000D5D6D101D7968C918823D1F1E091F70A24
:1006F000B4E0EB9FF0011124ED5AF94ED101DE96E2
:100700002D913D914D915C916081718182819381A8
:100710000F94BA0D2091B8163091B9164091BA16BF
:100720005091BB160F94BA0D4B015C019B01AC01BB
:10073000C701B6010F94BA0D0F94CB15F10173AF39
:1007400062AF2DEC3CEC4CE45DE3C501B4010F94C9
:10075000BA0D0F94CB15D101DD967C936E93DC9787
:10076000F10180818E7F80838FC024E5269DF0017A
:10077000279DF00D1124EC55FF4E808181FD4BC06B
:10078000C114D10441F0D6011596CD90DD90ED90C5
:10079000FC90189708C08BE0C82E87EDD82E83E216
:1007A000E82E8BE3F82EB4E5B69DF001B79DF00D71
:1007B0001124EC55FF4E81899289A389B489BC012B
:1007C000CD0190589B01AC010F945814F801258578
:1007D0003685478550890F94BA0D9B01AC01C7013E
:1007E000B6010F945714E62E872E982EA92E262F89
:1007F000372F482F592FA8966FADA897E5967FAD54
:10080000E597E0968FADE097E1969FADE1970F9465
:10081000540D87FF0CC0A896EFACA897E5968FAC57
:10082000E597E0969FACE097E196AFACE1972E2D6F
:10083000382D492D5A2DC201B1010F94540D882332
:1008400009F4B1CDF4E5F69DC001F79D900D11249A
:100850009C012C553F4E6901D9018C9181608C938C
:10086000C8010E9401FA882329F0F60180818E7F59
:10087000808399CD8E2D982DA92DBA2DF6018583D3
:100880009683A783B0878FCD80916F00826080931D
:100890006F0081E082C0D6018C9181FD58C0D601E5
:1008A00015962D913D914D915C911897AB962CAF7B
:1008B0003DAF4EAF5FAFAB971501B5E02B0E311CCE
:1008C000F8014580568067807084A3019201AB9641
:1008D0006CAD7DAD8EAD9FADAB970F94540D87FF82
:1008E00036C0F60181899289A389B489BC01CD0102
:1008F00090589B01AC010F945814D6011D962D9170
:100900003D914D915C9150970F94BA0D9B01AC01B4
:10091000AB966CAD7DAD8EAD9FADAB970F9457147C
:100920006B017C019B01AC01C301B2010F94B816AD
:1009300018166CF4D8018C9181608C93C5010E94CB
:1009400001FA8823F1F0F80180818E7F808324E50D
:10095000289DF001299DF00D1124EC55FF4E2185B5
:1009600032854385548565817681878190850F9492
:10097000540D81115CCDA4963FADA4973093901A8D
:1009800056CDD101CD92DD92ED92FC921397A496B3
:10099000BFADA497B093901ADACFC656DF4F0FB60B
:1009A000F894DEBF0FBECDBFDF91CF911F910F91A5
:1009B000FF90EF90DF90CF90BF90AF909F908F907F
:1009C0007F906F905F904F903F902F9008950F937E
:1009D0001F93CF93DF930CEA16E1CBE5D6E1F80144
:1009E00021913191419151918F0160E070E080E857
:1009F0009FE30F9452156993799389939993F6E144
:100A0000CB36DF0761F70E94A662DF91CF911F917D
:100A10000F910C94F2D2EF92FF920F931F93CF930A
:100A20007C018B014F3F11F4C2E401C0C4E580E2B8
:100A30000E940D4D8C2F0E940D4D8AE30E940D4D9A
:100A4000F701608171818281938142E00E94C84EEA
:100A5000F80140815181628173818FED9AE10E949A
:100A6000D74F62E070E080E090E0CF911F910F914E
:100A7000FF90EF900C94F96760913E0870913F08E9
:100A8000072E000C880B990B0F945B0D20913A08F0
:100A900030913B0840913C0850913D080F94B816A6
:100AA00018161CF08BEE9AE102C088EF9AE160E024
:100AB0000C9404DF1F93CF93DF93CDB7DEB7289755
:100AC0000FB6F894DEBF0FBECDBF182F60913E0861
:100AD00070913F08072E000C880B990B0F945B0D4B
:100AE0006D837E838F83988780913A0890913B082D
:100AF000A0913C08B0913D0889839A83AB83BC8365
:100B00004CEFBE016B5F7F4FCE0101960E940B85BB
:100B10006091550870915608072E000C880B990BB0
:100B20000F945B0D6D837E838F839887809151082E
:100B300090915208A0915308B091540889839A83E8
:100B4000AB83BC834FEFBE016B5F7F4FCE0101963D
:100B50000E940B851F3F41F087E11802F00111242C
:100B6000EA5CF74F628502C06091570870E087EE3B
:100B70009AE10E94BB4E6091570870E082EE9AE1C4
:100B80000E94BB4E28960FB6F894DEBF0FBECDBFB5
:100B9000DF91CF911F9108952F923F924F925F92D4
:100BA0006F927F928F929F92AF92BF92CF92DF927D
:100BB000EF92FF920F931F93CF93DF93CDB7DEB7E2
:100BC00063970FB6F894DEBF0FBECDBF898B81E06F
:100BD000809317021A821B821C821D8219861A8634
:100BE0001B861C8619821D862CE32E873CE13F87DD
:100BF00046E4488B312C212C50E85A8B8FEB8B8BA1
:100C000091E09887812C912C540160915508709146
:100C10005608072E000C880B990B0F945B0D7B0177
:100C20008C019B01AC01632D722D8A899B890F94E5
:100C3000540D882361F160915108709152088091A0
:100C4000530890915408A989A1110EC0B1E0B9834D
:100C50009701A8010F94B81618160CF019823E2CB3
:100C60002F2C0A8B1B8B13C09701A8010F94B81669
:100C7000181644F480911702882309F4F1C00E94E9
:100C800088DFEEC03E2C2F2C0A8B1B8B19820E9412
:100C900033686B017C01DC01CB0129853A854B85EA
:100CA0005C85821B930BA40BB50BB7FD34C0D70139
:100CB000C60188519C4FAF4FBF4F89879A87AB873A
:100CC000BC878091F70A0E945A8589E09BE10E94C7
:100CD0001F4D81149104A104B104B9F0D501C401E0
:100CE000805F984DAF4FBF4FBC01CD016C197D099E
:100CF0008E099F0928EE33E040E050E00F94AA13DC
:100D0000CA01B9010E949F4E03C08FE30E940D4D9E
:100D10008AE00E940D4D80E00E94AA500E94336834
:100D2000609374197093751980937619909377195D
:100D3000909151089E83A0915208AF83009153086F
:100D400010915408292F3A2FA801632D722D8A89FA
:100D50009B890F9457142B013C0120E030E0A9013E
:100D60000F94B81687FF04C077FA709477F87094E0
:100D700081149104A104B104B1F420E030E040E812
:100D80005FE3C301B2010F94540D87FF18C0B8850B
:100D900046015701BB2399F020E1820E27E2921E03
:100DA000A11CB11C0CC020E030E040E450E4C301C1
:100DB000B2010F94B816181614F446015701398180
:100DC0003323A9F18A819B81AC81BD81892B8A2B38
:100DD0008B2B61F0D701C6012A813B814C815D815B
:100DE000821B930BA40BB50BB7FD21C02E813F8155
:100DF000A8016D857E858F8598890F94571420E012
:100E000030E040EC5FE30F94540D87FD33CFD70102
:100E1000C601805A9541AF4FBF4F8A839B83AC83F5
:100E2000BD839E819D87AF81AE870F87188B809190
:100E30001702882309F41ECF81149104A104B10480
:100E400011F41886E2CEB0E1CB1AB7E2DB0AE10872
:100E5000F108C818D908EA08FB08F7FCF2CF0ACF56
:100E60008091170263960FB6F894DEBF0FBECDBF18
:100E7000DF91CF911F910F91FF90EF90DF90CF9076
:100E8000BF90AF909F908F907F906F905F904F90AA
:100E90003F902F9008952F923F924F925F926F92C2
:100EA0007F928F929F92AF92BF92CF92DF92EF92FA
:100EB000FF920F931F93CF93DF93CDB7DEB7649765
:100EC0000FB6F894DEBF0FBECDBF898B6A8B81E071
:100ED000809317021A821B821C821D8219861A8631
:100EE0001B861C8621E0288719821D863CE33E87ED
:100EF0004CE14F8756E4588B312C212C80E88B8BAA
:100F00009FEB9C8B812C912C540160913E08709139
:100F10003F08072E000C880B990B0F945B0D7B018B
:100F20008C019B01AC01632D722D8B899C890F94E0
:100F3000540D882361F160913A0870913B088091CB
:100F40003C0890913D08AA89A1110EC0B1E0B98377
:100F50009701A8010F94B81618160CF019823E2CB0
:100F60002F2C0B8B1C8B13C09701A8010F94B81664
:100F7000181644F480911702882309F4F0C00E94E7
:100F800088DFEDC03E2C2F2C0B8B1C8B19820E940E
:100F900033686B017C01DC01CB0129853A854B85E7
:100FA0005C85821B930BA40BB50BB7FD33C0D70137
:100FB000C60188519C4FAF4FBF4F89879A87AB8737
:100FC000BC8789890E945A8585E09BE10E941F4D5C
:100FD00081149104A104B104B9F0D501C401805F6A
:100FE000984DAF4FBF4FBC01CD016C197D098E09E3
:100FF0009F0928EE33E040E050E00F94AA13CA01A5
:10100000B9010E949F4E03C08FE30E940D4D8AE0FC
:101010000E940D4D80E00E94AA500E9433686093A8
:10102000741970937519809376199093771990912C
:101030003A089E83A0913B08AF8300913C08109131
:101040003D08292F3A2FA801632D722D8B899C8989
:101050000F9457142B013C0120E030E0A9010F94BC
:10106000B81687FF04C077FA709477F870948114EB
:101070009104A104B104B1F420E030E040E85FE362
:10108000C301B2010F94540D87FF18C0B885460103
:101090005701BB2399F020E1820E27E2921EA11C8A
:1010A000B11C0CC020E030E040E450E4C301B201C8
:1010B0000F94B816181614F44601570139813323DA
:1010C000A9F18A819B81AC81BD81892B8A2B8B2BD5
:1010D00061F0D701C6012A813B814C815D81821B71
:1010E000930BA40BB50BB7FD21C02E813F81A80146
:1010F0006D857E858F8598890F94571420E030E0A8
:1011000040EC5FE30F94540D87FD34CFD701C60147
:10111000805A9541AF4FBF4F8A839B83AC83BD8379
:101120009E819D87AF81AE870F87188B80911702B4
:10113000882309F41FCF81149104A104B10411F490
:101140001886E3CEB0E1CB1AB7E2DB0AE108F1087A
:10115000C818D908EA08FB08F7FCF2CF0BCF80913A
:10116000170264960FB6F894DEBF0FBECDBFDF91B5
:10117000CF911F910F91FF90EF90DF90CF90BF9094
:10118000AF909F908F907F906F905F904F903F9027
:101190002F9008952F923F924F925F926F927F927D
:1011A0008F929F92AF92BF92CF92DF92EF92FF9277
:1011B0000F931F93CF93DF93CDB7DEB729970FB669
:1011C000F894DEBF0FBECDBFF82E762E0E9469D3F5
:1011D00081E08F1598F40E94BC4D84E50E940D4D6E
:1011E0006F2D70E080E090E00E949F4E80E20E94B0
:1011F0000D4D8DE09BE10E941F4DF7C1711008C09D
:101200008091A60A877077247394873009F4712C33
:101210009090F70A81E087258987882389F08824C0
:10122000839420E030E0A9016091EA167091EB16FA
:101230008091EC169091ED160F94540D811101C020
:10124000812C8091E91683FD53C18091E8168111AC
:101250004FC120913E0830913F0880915D029091EE
:101260005E02281739070CF043C1882049F00E941C
:10127000BC4D81E39BE10E941F4DF092F70AB5C17E
:1012800066246394F91409F424C120905902309023
:101290005A0240905B0250905C0280E090E0A8EC23
:1012A000B2E48093590290935A02A0935B02B093E8
:1012B0005C0280E00E9476E381E00E9476E382E0B7
:1012C0000E9476E30E94B4CA8985882309F470C01D
:1012D0002091FE163091FF16409100175091011792
:1012E0006091000B7091010B8091020B9091030BA8
:1012F0000F9458146093000B7093010B8093020BB2
:101300009093030BA0905502B0905602C0905702E4
:10131000D0905802A60195010F94B816181644F4FF
:10132000A092000BB092010BC092020BD092030B63
:10133000A12CB12C6501E090F70A04EC16E124E041
:101340003BE040E05BE06CEF7AE088EF9AE00E94DF
:10135000EAD58091F6169091F716A091F816B09103
:10136000F9168093F80A9093F90AA093FA0AB093B9
:10137000FB0A8091FA169091FB16A091FC16B09191
:10138000FD168093FC0A9093FD0AA093FE0AB09389
:10139000FF0AE92C09E512E024E03BE040E05BE0D5
:1013A0006CEF7AE088EF9AE00E94EAD50E9469D358
:1013B00020E030E0A9016091F80A7091F90A80916B
:1013C000FA0A9091FB0A0F9458146093F80A7093EC
:1013D000F90A8093FA0A9093FB0A20E030E0A90111
:1013E0006091FC0A7091FD0A8091FE0A9091FF0ABB
:1013F0000F9458146093FC0A7093FD0A8093FE0AC0
:101400009093FF0A20E030E0A9016091000B7091F9
:10141000010B8091020B9091030B0F945814609371
:10142000000B7093010B8093020B9093030BF092CF
:10143000F70A0E94D7E4711044C0809140028823CB
:1014400009F43FC0892D90E0FC01EC51F94E209148
:10145000E61620836F2D70E0FB01EC51F94E2081E0
:101460002093E61620913E0830913F08880F991F7F
:10147000FC01E052F94E31832083660F771FFB0198
:10148000E052F94E80819181009761F02817390769
:1014900049F00E944BA180E00E943C8560E080E022
:1014A0000E944B87811050C086E99AE00E940AE0B2
:1014B0008985882331F064EC76E18EE99AE00E9418
:1014C0009CE42092590230925A0240925B02509260
:1014D0005C020E9469D30E94BC4D6091F70A70E0E3
:1014E0008FE19BE10E94BB4E8AE00E940D4D7DC0C2
:1014F000882041F16091F4167091F516072E000CCA
:10150000880B990B0F945B0D20E030E040E752E42C
:101510000F9452156D837E838F8398878091EA168E
:101520009091EB16A091EC16B091ED16B05889830E
:101530009A83AB83BC83BE016B5F7F4FCE01019664
:101540000E944ACD612C9ECE6110AECF6091F21602
:101550007091F316072E000C880B990B0F945B0DFE
:1015600020E030E040E752E40F94521569837A831B
:101570008B839C83BE016F5F7F4F8AEE96E10E9452
:101580004ACD80E090E0A0E4B0E489839A83AB8305
:10159000BC83BE016F5F7F4F8EEE96E10E944ACD05
:1015A0000E9469D320E030E040E050E46091040BF9
:1015B0007091050B8091060B9091070B0F945714B7
:1015C0006093040B7093050B8093060B9093070BAD
:1015D0006093A20A7093A30A8093A40A9093A50A29
:1015E00082EA9AE00E947AD35FCF29960FB6F894E8
:1015F000DEBF0FBECDBFDF91CF911F910F91FF9046
:10160000EF90DF90CF90BF90AF909F908F907F90A2
:101610006F905F904F903F902F900895EF92FF92C0
:101620000F931F93CF93DF9380913F028F37A0F0EA
:101630008F579091400890931017992311F02C9A8E
:1016400001C02C982091570820930F179091020108
:10165000222369F090950BC090911017891708F01C
:101660002C9890910F17891728F090910201907291
:10167000909300018F5F80933F0290910E1781E05D
:10168000892780930E1780913E0285301CF411E06B
:10169000180F01C010E0823009F4B9C054F4882357
:1016A00001F1813009F0E8C088E080937B0085E497
:1016B000C5C0843009F4CAC00CF4BCC0853009F040
:1016C000DBC090910D17911102C080930D1780918E
:1016D0000D17815080930D17882309F4CDC015E0B4
:1016E000CBC080913D028F5F80311CF480933D021E
:1016F000C3C010923D0280919416811113C0809155
:101700003608909137089093390880933808809173
:101710004D0890914E089093500880934F0881E0B7
:1017200080939416109237081092360810924E0843
:1017300010924D08E0903808F0903908F194E19447
:10174000F10880913E0890913F0801E018161906B3
:101750002CF080914008811101C000E080911102BD
:10176000909112029195819591098E159F053CF4F7
:101770004FE45AE160E77AE180E00E946BF50023D4
:1017800089F080910F0290911002919581959109B5
:10179000E816F9063CF442E85AE163EA7AE180E0AF
:1017A0000E946BF5809155089091560801E018163B
:1017B00019062CF080915708811101C000E020919A
:1017C0004F08309150088091650890916608821703
:1017D00093073CF04FE55AE160E77AE18FEF0E9412
:1017E0006BF5002309F448C020914F083091500850
:1017F00080910D0290910E0228173907ECF142E911
:101800005AE163EA7AE18FEF0E946BF535C080916F
:101810007A0086FD2EC08091780090917900209109
:10182000360830913708820F931F909337088093C2
:10183000360822C088E080937B0086E480937C0099
:1018400080917A00806480937A0016C080917A003B
:1018500086FD11C0809178009091790020914D080B
:1018600030914E08820F931F90934E0880934D083D
:1018700003C012E001C014E010933E0220917819D9
:10188000309179192115310509F43AC0F8949091F5
:101890000901927080910801817080930601809106
:1018A0000B01121613060CF08095827080930901CB
:1018B00000000000000080910B01809588708093EB
:1018C000090184E08A950000E9F780910B01887096
:1018D0008093090180910B01911180958270809312
:1018E000090178948091781990917919121613064C
:1018F00014F4019701C00196909379198093781997
:1019000080919516882309F44DC080913C028E5F2A
:101910008F7780933C02811145C08CB185FB88276D
:1019200080F9C82F80E0D82F8091030181FDC2602B
:101930004B99C46000910B1710910C170C271D27B1
:101940000115110579F100FF07C0BE01617077270D
:101950008AEC9AE10E94BB4E01FF08C06C2F66958D
:10196000617070E081EC9AE10E94BB4E02FF08C0FA
:10197000C2FB662760F970E088EB9AE10E94BB4EDB
:1019800085EB9AE10E941F4D10910A17612F70E0BC
:101990008DE00E941167109510930A17D0930C17D1
:1019A000C0930B178091790881110E948AE580917C
:1019B000961690919716009769F001979093971655
:1019C00080939616892B31F483ED9AE190938A08DF
:1019D00080938908DF91CF911F910F91FF90EF9035
:1019E00008950F930FB70F9300916E000B7F009334
:1019F0006E0078940F930BB70F930CB70F921F9252
:101A00002F933F934F935F936F937F938F939F9306
:101A1000AF93BF93EF93FF9311240E940E8BFF911E
:101A2000EF91BF91AF919F918F917F916F915F9156
:101A30004F913F912F911F900F900CBF0F910BBFB3
:101A40000F910460F89400936E000F910FBF0F91F7
:101A500018952F923F924F925F926F927F928F9242
:101A60009F92AF92BF92CF92DF92EF92FF920F932D
:101A70001F93CF93DF93CDB7DEB729970FB6F894B6
:101A8000DEBF0FBECDBF1C017B836A8329831F830A
:101A90000E83FD82EC8227FD10C0022E000C330B5A
:101AA00039872887398185E03802F0011124E2570F
:101AB000F94E84818823E1F008C080918D16882337
:101AC00099F0E1E0F0E0F987E887F1011482E88518
:101AD000F985EE0FFF1FEE0FFF1FEE5FF84E10822D
:101AE0001182128213822EC021E030E039872887CC
:101AF000FA01C080D180E280F38008851985000F4B
:101B0000111F000F111F0E5F184EA7019601F8015B
:101B100060817181828193810F94540D882391F0AB
:101B2000F801C082D182E282F38211E020E030E04D
:101B3000A901C701B6010F94B81618160CF010E0F1
:101B4000F1011483F10184818230F9F0833009F4CA
:101B500001C1813009F023C1E885F985EE0FFF1F2F
:101B6000EE0FFF1FEE5FF84E2081318142815381DD
:101B7000EA81FB8160817181828193810F94540D90
:101B800087FD0DC182E0F101848380913B028823AF
:101B900009F493C0F981F7FD90C08F2FFF0F990BC7
:101BA0008C011816190614F401E010E0F801EA514E
:101BB000F94E2081222371F1EA81FB81C080D1801E
:101BC000E280F380880F991F880F991FFC01EE5F58
:101BD000F84E80809180A280B3802C813D81B90134
:101BE00080E090E00F94590D2B013C0120E030E0A3
:101BF00040E85EE30F94BA0D9B01AC01C501B4014E
:101C00000F9457149B01AC01C701B6010F94B8168D
